:100000000C9461100C9492100C9492100C94921019
:100010000C9492100C9492100C9492100C949210D8
:100020000C9492100C9492100C9492100C949210C8
:100030000C9492100C9492100C9492100C949210B8
:100040000C9492100C9492100C9492100C949210A8
:100050000C9492100C9492100C9492100C945EAF2D
:100060000C9492100C94418E0C94178E0C94921058
:100070000C9492100C9492100C9492100C94921078
:100080000C9492100C9492100C9492100C94921068
:100090000C94ED8D0C94C38D0C9492100C94FC294F
:1000A0000C9492100C9492100C9492100C94921048
:1000B0000C9492100C9492100C9492100C94921038
:1000C0000C9492100C9492100C9492100C94998DA4
:1000D0000C946F8D0C9492100C94458D0C941B8D88
:1000E0000C94921007634236B79BD8A71A3968560A
:1000F00018AEBAAB558C1D3CB7CC5763BD6DEDFD4A
:10010000753EF6177231BF000000803F0800000006
:10011000BE922449123EABAAAA2ABECDCCCC4C3EFC
:1001200000000080BEABAAAAAA3E00000000BF00EB
:100130000000803F0000000000084178D3BB4387E7
:10014000D1133D190E3CC3BD4282AD2B3E68EC82FB
:1001500076BED98FE1A93E4C80EFFFBE01C4FF7F80
:100160003F00000000000C94157B0C943E390C9469
:1001700015120C944BA80C9482150C94CC3D0C9445
:10018000E33B0C9476490C9447A80C946E260C948F
:100190006A820C94F23A0C940A150C94EE650C9455
:1001A00028130C945E170C94AE610C94A43D0C942F
:1001B000B8390C9429880C942BA80C94B5310C9464
:1001C00098480C9458650C94497F0C9437140C94FF
:1001D00062900C94B6820C94B6140C94A9480C94BA
:1001E000D3540C9491280C941F120C942A360C941E
:1001F0003F140C9421420C94FC200C9407120C9494
:10020000C1610C94001A0C9481120C94CF100C94C0
:1002100030620C9403130C942BA90C94F7C50C9426
:10022000F5610C9413A80C94E2150C948D260C9493
:1002300019A80C94E7610C94FC150C94F2610C94D1
:10024000D14D0C9481660C94C03D0C9413280C94F1
:10025000303A0C94CF6C0C94B3140C94061F0C948D
:100260006F120C94A2380C9463390C9468160C9499
:100270001DA80C9403610C94894D0C9445390C9481
:100280002B200C94E32E0C9479170C94041A0C94E4
:1002900011A90C94CB280C9412220C9449120C94A2
:1002A000153D0C94883A0C9458A90C94397F0C9401
:1002B000493A0C9440BB0C945F160C94061A0C94AB
:1002C000E4610C9468740C946B7F0C9432820C94EF
:1002D0001B4A0C94AA100C9431A80C940B130C9488
:1002E00014390C9405C60C944AC50C9463290C94DB
:1002F000FBBF0C9471650C9466800C94B9140C943B
:1003000049A90C94F0A80C94A6120C94993A0C9458
:10031000AE100C9439A80C94313C0C9454480C94B5
:1003200070180C941E120C948E120C9485180C9458
:1003300085760C9483120C94183C0C947E2B0C94B0
:10034000C4100C94FDA80C9467390C94FF800C9495
:10035000A0260C9435A80C94C36F0C94B23D0C9459
:100360006D800C94D13D0C94E23D0C94253D0C9491
:10037000FE6F0C940BA80C94CD160C94554D0C9458
:100380001B3C0C94B0140C9465340C9408210C9410
:10039000E5490C948AA90C9476800C9423A80C94BB
:1003A0001A390C94191F0C94A6810C9448490C948A
:1003B00076A90C94ED3C0C940FA80C94DB3A0C94A9
:1003C00073120C94D0180C94113E0C94E23A0C94D5
:1003D000F7640C94AC130C944E4A0C94D5390C94DD
:1003E000ED4D0C944AA80C94031E0C945F3D0C94A4
:1003F00086120C94BF810C9411390C94C03C0C945F
:10040000D3150C9448380C94E68F0C94EE3A0C9467
:1004100046120C947E660C9470800C9405A80C9483
:10042000F37E0C9414210C94C3210C9423660C9439
:10043000683E0C9460120C94F31E0C94C07F0C94D4
:10044000B3650C948A3D0C944B390C94D2C40C9433
:10045000FC140C943FA90C9462A90C9447210C94B1
:10046000A7770C94E07E0C9443A80C940E3E0C9459
:1004700040170C944E150C9440120C94A9380C940F
:1004800017390C94AA1A0C9498C70C946A120C94FD
:100490008E180C948E290C9445380C9464330C946B
:1004A0009F3C0C9445160C94F0910C941BA90C9451
:1004B000946C0C949A610C94B04D0C94A8640C94B8
:1004C000DD3C0C942D220C9496120C944C800C94D0
:1004D00021830C94C4400C9416120C946CA90C94B7
:1004E0008A130C9438240C941B160C94441C0C9402
:1004F000FE3B0C9423A90C94783A0C94E31F0C94C3
:10050000D8610C94741E0C94BAC70C94E13D0C9401
:1005100050C50C942B650C942A150C940E150C9454
:1005200010150C94B3800C9472640C94BA180C944B
:100530006E3A0C94D5650C945F7B0C94493D0C94F9
:1005400063120C94021A0C94F78F0C9442480C948A
:100550000C890C945F120C94803D0C9452820C9484
:10056000E6800C941E240C943FA80C945EC50C9459
:1005700080A90C94D91E0C94263B0C94F27E0C940A
:1005800075760C9417900C94843A0C9454390C940E
:1005900092120C94C0140C943F4E0C94061E0C94B2
:1005A00007800C941A370C945D7F0C9419120C94EC
:1005B000515B0C94F2140C9445120C94E93C0C948D
:1005C000863A0C940B4D0C941F140C94C7170C9482
:1005D00094100C94D8200C9428BE0C94C6150C943E
:1005E000D5550C9477120C94A7C00C9446140C9417
:1005F000A5170C94DCC50C9400900C94AA3C0C94A8
:1006000001620C947B660C9435A90C94483E0C94C2
:10061000D2140C94084E0C94FE390C94AD210C9419
:100620006D810C9428140C9451810C94A2660C9446
:10063000FE190C9413150C9433290C94F9B80C94EE
:1006400074900C94AD900C9471160C94FC280C943E
:1006500049220C947C810C947FC50C9433480C94F3
:10066000B8810C94B2400C944D1F0C94DE640C9431
:100670004E120C9485150C9427A80C944E380C94AB
:1006800040610C941F390C94803A0C9434130C94F0
:10069000081A0C9407A90C9451120C94F8A80C9405
:1006A00046BB0C949F186364696E6F7073757858BD
:1006B0005B004E414E494E495459494E46CDCCCC33
:1006C0003D0AD7233C17B7D13877CC2B329595E626
:1006D000241FB14F0A000020410000C84200401C06
:1006E0004620BCBE4CCA1B0E5AAEC59D74556E6BDF
:1006F0006E6F776E207375666669782000556E6B35
:100700006E6F776E20636D642000636C7243747249
:100710003A20002F00496E3A20003D00494E3A0031
:100720003D004C454741435920494E3A00000020C6
:10073000002300260029002C002F003200000100B9
:10074000000301060109012D3E00200023002D3E7B
:1007500000200050656E6465643A20230072617762
:100760000076616C0074656D70007361740068756B
:10077000650066616E0052474200485356006D6F37
:10078000646500536574436D643A0053746F726519
:1007900064204558543A00737566666978436F64FF
:1007A000653A00584F4E0048414C54002074696D22
:1007B000653A004374726C205265733A00205453BA
:1007C0003A0020543A003D0050696E3A004F4E3ACC
:1007D000416C7265616479204163746976650A00D1
:1007E00048414C543A416C726561647920496E61AC
:1007F00063746976650A00584F4E3A416C726561C0
:100800006479204163746976650A00584F46462032
:10081000736B69707065642E205072657620636D0D
:10082000643A005475726E6564206F666620667265
:100830006F6D3A00526573746F7265642066726FF3
:100840006D3A0049676E6F7265642C206368616E53
:100850006E656C20636D643D0020457865633A00E9
:100860004163746976653A0048414C543A416C7270
:100870006561647920496E6163746976650A005820
:100880004F4E3A416C7265616479204163746976B8
:10089000650A00584F464620736B69707065642E78
:1008A000205072657620636D643A005475726E65EF
:1008B00064206F66662066726F6D3A0052657374CD
:1008C0006F7265642066726F6D3A004E6F742065BA
:1008D0006E6F756768206D656D6F727920666F72D7
:1008E0002067726F7570206F7065726174696F6ECA
:1008F00000206D73203A0041726D656420666F724E
:1009000020002044697361726D656400536B6970E7
:1009100070656420686F6D69652073747566660024
:100920004F75744F664D656D6F7279210A00200016
:10093000205375623D00204974656D3D0052414D64
:100940003D00282D292000282B2920002076616CCD
:100950007565206973200020756E6B6E6F776E0A67
:10096000005D3D005B0020696E76616C696400206B
:1009700000206F6B003A00206661696C6564003A84
:10098000005265747279696E67206D6F6462757369
:1009900020434D440A00207365632072656D6169D0
:1009A0006E696E6700537461747573206465666662
:1009B000657265640A002D3E005075623A2000633E
:1009C0006D640046414E5F4F4E4C590044525900F1
:1009D000434F4F4C0048454154004155544F002D62
:1009E0003E005075623A20007365740064656C00C7
:1009F0002D3E005075623A20002D3E005075623A3F
:100A00002000556E6B6E6F776E20636D64200A0058
:100A10004F4646004F4E0020002D3E00436F6E763D
:100A2000657274696E6720002D3E0057726F6E67A5
:100A30002041737369676E6D656E74200052474282
:100A4000783A200020764C6576656C3A0020436F3A
:100A50006E76563A0020436F6E76533A0020486F08
:100A6000743A00436F6C643A0020436F6E7665728F
:100A700074656420563A00436F6E766572746564DF
:100A800020533A002D3E0057726F6E6720417373FA
:100A900069676E6D656E7420002D3E0057726F6E33
:100AA000672041737369676E6D656E7420005361D2
:100AB0007665643A0020537566663A002041543AE0
:100AC00000436F6E666967206368616E67656420C6
:100AD0006C6F63616C6C792C20706F7274616C2028
:100AE00064697361626C6564002F636F6E66696729
:100AF0002E6A736F6E007265626F6F742000436DB3
:100B0000643A20002F636F6D6D616E642F002F7249
:100B1000616D2F002F6974656D2F002F6974656DED
:100B20002F004C6F636174696F6E3A206874747043
:100B30003A2F2F6C617A79686F6D652E72752F7000
:100B40007761003F6D61633D002669703D0026704E
:100B50006F72743D00266E616D653D002F002000B0
:100B6000436F6D706C6574652E2052656D6F766590
:100B700020746F706963200024636F6D6D616E6413
:100B800000536B697070696E672E2E00436C65614F
:100B90006E55702072657461696E656420746F7043
:100BA00069632000220022004F75744F664D656D09
:100BB0006F727921005D20003A5B000A005D0045FC
:100BC0006D7074793A205B000A003A004D41433A57
:100BD00000554450205379736C6F6720696E6974B7
:100BE00069616C697A65642E0A005379736C6F676A
:100BF00020706172616D733A0043757272656E7434
:100C0000204C414E20636F6E6669672869702C64C2
:100C10006E732C67772C7375626E6574293A000ABF
:100C200055736520746865736520636F6D6D616EC3
:100C300064733A202768656C7027202D20746869DA
:100C40007320746578740A276D61632064653A6166
:100C5000643A62653A65663A66653A3030272073D1
:100C6000657420616E642073746F7265204D41431A
:100C70002D6164647265737320696E20454550521E
:100C80004F4D0A276970205B69705B2C646E735B43
:100C90002C67775B2C7375626E65745D5D5D5D2797
:100CA000202D20736574207374617469632049502A
:100CB0000A277361766527202D207361766520638E
:100CC000757272656E7420636F6E66696720696EF7
:100CD000204E5652414D3B204F4E7C4F4646202DD4
:100CE00020656E61626C652F64697361626C65205A
:100CF0006175746F736176650A2767657427205B79
:100D0000636F6E66696720616464725D27202D20C1
:100D100067657420636F6E6669672066726F6D2009
:100D20007072652D636F6E666967757265642055B4
:100D3000524C20616E642073746F7265206164642C
:100D4000722C204F4E7C4F4646202D20656E6162EE
:100D50006C652F64697361626C6520646F776E6C7B
:100D60006F6164206F6E20737461727475700A27EE
:100D70006C6F616427202D206C6F616420636F6E3F
:100D80006669672066726F6D204E5652414D0A2784
:100D900070776427202D20646566696E6520616E1A
:100DA000642073746F7265204D51545420706173C8
:100DB00073776F72640A276F746170776427202DD0
:100DC00020646566696E6520616E642073746F725D
:100DD0006520485454502041504920706173737706
:100DE0006F72640A276C6F67205B73657269616C50
:100DF0005F6C6F676C6576656C5D205B7564705FBA
:100E00006C6F676C6576656C5D27202D2064656668
:100E1000696E65206C6F67206C6576656C20283084
:100E20002E2E37290A276B696C6C27202D207465BC
:100E30007374207761746368646F670A27636C65F5
:100E4000617227202D20636C6561722045455052E8
:100E50004F4D0A277265626F6F7427202D207265CF
:100E6000626F6F7420636F6E74726F6C6C6572006A
:100E7000536F6674207265626F6F74696E672E2E91
:100E80002E0052414D3D000A5379736C6F6720006C
:100E90000A6D71747420000A696E70757473200095
:100EA0000A6974656D7320000A436F6E6669677521
:100EB0007265643A003B003D0050696E3A003B00A9
:100EC0003D4C4F5700546865726D6F3A0041707029
:100ED0006C79696E6720636F6E666967004C6F613D
:100EE00064656420455441473A004E6F2073746F27
:100EF00072656420636F6E666967004C6F6164653C
:100F0000642066726F6D20454550524F4D006C6FE6
:100F10006164206661696C6564004C6F6164696E30
:100F20006720436F6E6669672066726F6D20454566
:100F300050524F4D00436F6E666967206175746F44
:100F4000736176653A000A5379736C6F6720646544
:100F5000627567206C6576656C3A005365726961ED
:100F60006C206465627567206C6576656C3A005329
:100F7000617665640A005365742064796E616D69F9
:100F8000632049500A00454550524F4D20636C651F
:100F9000617265640A004D51545420506173737737
:100FA0006F726420757064617465640A004F544107
:100FB0002050617373776F7264207570646174651B
:100FC000640A00636F756C64206E6F7420706172C8
:100FD00073653A2000557064617465640A004E6F51
:100FE000204950206164726573730052656C6561BD
:100FF00073696E6720736F636B657420616E642024
:10100000726574727900205361766564004C6F617B
:1010100064696E67204854545020636F6E66696738
:10102000206F6E20737461727475703A004F46467B
:10103000004F4E002B002D00455461673A200047B9
:10104000657420455441473A2000485454502F318C
:101050002E312025690025733A2025730D0A0020C2
:10106000485454502F312E310D0A486F73743A2072
:1010700025730D0A4163636570743A202A2F2A0D87
:101080000A436F6E6E656374696F6E3A20636C6FAE
:1010900073650D0A0025730020000D0A00474554B2
:1010A000006661696C656420746F20636F6E6E65A5
:1010B00063740A004552524F523A20536572766566
:1010C000722072657475726E65642000436F6E667F
:1010D0006967206E6F74206368616E6765640A00DB
:1010E000446F6E652E0A00436F6E666967207061FB
:1010F0007273696E67206661696C65640A00676F68
:101100007420436F6E6669670A0066726565200029
:10111000436F6E666967205552493A20687474704F
:101120003A2F2F002044656661756C7420636F6EE2
:101130006669672073657276657220757365643AB7
:1011400020006C617A79686F6D652E7275000A28CF
:101150002B29454C455641544F52000A282B294D06
:10116000554C544956454E54000A282B2950574D8A
:101170005F52454C4159000A282D294D444E5300D9
:101180000A282D2955415254425249444745000AE4
:10119000282B295359534C4F47000A282D295049D1
:1011A00044000A282D294D43503233303137000A8C
:1011B000282D294152544E4554000A282B294F54BA
:1011C00041000A282D29535049204C4544000A2843
:1011D0002D294D4F544F5220435452000A282B2999
:1011E0004143204841494552206F6E205365726942
:1011F000616C33000A282D294343533831312026AE
:101200002048444331303830000A282B29524553B6
:10121000544152545F4C414E5F4F4E5F4D515454B8
:101220005F4552524F5253000A282D2948415244DB
:1012300052455345542C207573696E6720736F6651
:1012400074000A282D29434F554E544552000A2850
:101250002D29444854000A282D294F57495245004A
:101260000A282D294D4F44425553000A282D294460
:101270004D58000A282B2957697A6E6574357830E5
:1012800030000A282B294672656552616D20707204
:10129000696E74696E67000A282B295741544348C8
:1012A000444F47000A4669726D77617265204D416F
:1012B0004320416464726573732064653A30313A47
:1012C00032333A30303A30303A3031006C617A792A
:1012D000686F6D652E7275000A436F6E66696720D0
:1012E0007365727665723A003230313730334C00B4
:1012F00020432B2B2076657273696F6E3A00383964
:1013000031373031635F323032322D31302D30326F
:10131000000A4C617A79686F6D652E7275204C6990
:1013200067687448756220636F6E74726F6C6C6569
:10133000722000204F464600204F4E002042595058
:1013400041535300757074696D6500667265656818
:10135000656170002054696D65723A00204C6F63BE
:101360006B733A002000204C6F636B733A000A5293
:10137000414D3D0020457870697265640A00202D5A
:10138000746172676574207A6F6E652D0020416C00
:1013900061726D20457870697265640A0020636D22
:1013A000643A00204375723A00205365743A005342
:1013B0006176656420746F20454550524F4D00534F
:1013C0006176696E6720636F6E66696720746F204F
:1013D000454550524F4D2E2E002069732000446524
:1013E0006C6574696E6720636F6E662E2052414D86
:1013F000207761733A0053746F70706564005374A2
:101400006F7070696E67206368616E6E656C7320C3
:101410002E2E2E004E6F7420756E6C6F636B65649C
:1014200020696E20313073202D20636F6E74696ED9
:101430007565202E2E2E00556E6C6F636B696E677E
:1014400020636F6E666967202E2E2E00414320496F
:101450006E69740041432044652D496E69740045EE
:101460005252004452590046414E5F4F4E4C590073
:101470004845415400434F4F4C00506F6C6C696EAF
:1014800067004C4F57004D454449554D004849476A
:1014900048004155544F0072617700717565697459
:1014A000007377696E67006C6F636B0044656661FB
:1014B000756C742073657269616C206D6F64652052
:1014C0004E38312075736564003845310026003888
:1014D0004E31000600384532002E00384E32000EE4
:1014E00000384F31003600384F32003E003745316A
:1014F000002400374532002C00374F3100340037CC
:101500004F32003C00374E31000400374E32000CA1
:1015100000203D3E002C002C002C002C00456C656A
:101520007661746F723A20636F6E666967206661D8
:10153000696C65643A00456C657661746F7220630E
:101540006F6E666967206572726F7200456C6576B2
:1015500061746F7220636F6E666967206C6F61647F
:1015600065642000456C657661746F723A204F7532
:1015700074206F66206D656D6F727900456C6576BD
:1015800061746F722044652D496E6974004030307B
:1015900052523030303030313030334630303431E8
:1015A0003043303034322A00403030525230303004
:1015B0003030323030374630303032313030303306
:1015C000302A0040303052523030303030343030F9
:1015D0003346303038343134303033382A003C0030
:1015E0003E00556E6B6E6F776E2073756666697818
:1015F0002000556E6B6E6F776E20636D6420005314
:101600006574206E6F7420696D706C656D656E74A5
:10161000656400466F726365642065786563757400
:10162000696F6E00454C45563A20004D756C7469E3
:1016300056656E7420636F6E666967206661696CBB
:101640006564004D756C746956656E7420696E69C9
:1016500074004D756C746976656E742044652D490F
:101660006E697400204F75743A00206D3300206657
:10167000726F6D2000204D61782072657175657301
:10168000743A002066616E253A00206163746976C1
:101690006520563A00546F74616C20563A002069F8
:1016A0006E69740050574D2D4F75742023002073C0
:1016B000746F700050574D2D4F75742023003D00FE
:1016C00050696E3A0020696E69740052656C6179E8
:1016D0002D4F75742023002073746F700052656C59
:1016E00061792D4F75742023003D3E003A007075DE
:1016F0006220616374696F6E200069646C65006FBD
:1017000066660068656174696E670066616E006494
:101710007279696E6700636F6F6C696E670020692C
:101720007320004F75742000556E6B6E6F776E20BE
:101730007375666669782000556E6B6E6F776E20E4
:10174000636D642000616374696F6E0072656C6123
:10175000794374723A20005B305D3A2000202D20DE
:101760002D202D20EFBBBF003E003E31202D20005C
:1017700020002E00696E00735F6F7574006D7968CC
:101780006F6D6500202D3E2000456D69743A200084
:10179000202D3E20004974656D436D643A20002081
:1017A0002D3E20004974656D3A20003E3E200049E0
:1017B0006E76616C696420636F6D6D616E64003E6E
:1017C0003E3E004E6F204D414320636F6E66696759
:1017D000757265643A20736574206669726D77610D
:1017E00072652773204D41430A004E6F2076616C6D
:1017F000696420454550524F4D20646174612E202C
:10180000496E697469616C697A696E672E00476F09
:101810007420495020616464726573733A002769CB
:1018200070205B69705B2C646E735B2C67775B2C3C
:101830007375626E65745D5D5D5D27202D20736537
:1018400074207374617469632049500A00466169A9
:101850006C656420746F20636F6E6669677572656E
:101860002045746865726E6574207573696E6720B3
:10187000444843502E20596F752063616E20736574
:1018800074206970206D616E75616C6C7921000A3D
:101890007573657320444843500A00204D41534BF3
:1018A0003A002047573A0020444E533A004C6F61AB
:1018B0006465642066726F6D20666C617368204990
:1018C000503A005374617274696E67206C616E00E7
:1018D0004142434445464748494A4B4C4D4E4F5080
:1018E0005152535455565758595A6162636465664C
:1018F0006768696A6B6C6D6E6F7071727374757600
:101900007778797A303132333435363738392B2F8E
:101910003D004261736963200061726475696E6F96
:101920003A004F544120696E697469616C697A6547
:10193000640A0044454641554C54207061737377E6
:101940006F726420666F72204F5441204150492EBF
:1019500020557365206F746170776420636F6D6DBF
:10196000616E6420746F20736574007061737377A7
:101970006F726400757074696D652C667265656858
:1019800065617000247374617473003839313730C5
:1019900031635F323032322D31302D3032004C69BC
:1019A0006768744875622000246E616D6500726519
:1019B00061647900546F6F206D616E79204D5154D0
:1019C0005420636F6E6E656374696F6E206572720A
:1019D0006F72732E2052657374617274204C414E85
:1019E000002074727920616761696E20696E20350C
:1019F000207365636F6E6473006661696C65642C47
:101A00002072633D004177616974696E6720666F7B
:101A1000722072657461696E656420746F706963A9
:101A20007300636F6E6E656374656420617320007C
:101A3000202E2E2E0020757365723A003A000A415E
:101A40007474656D7074696E67204D5154542063D1
:101A50006F6E6E656374696F6E20746F20002473FF
:101A60007461746500646973636F6E6E6563746539
:101A700064005573696E67204D5154542070617332
:101A800073776F72642066726F6D20636F6E666924
:101A90006700446576696365204E616D653A004173
:101AA00074206C6561737420646576696365206E6B
:101AB000616D6520616E642062726F6B6572204992
:101AC00050206D75737420626520636F6E66696760
:101AD0007572656400526562696E64207375636334
:101AE0006573732E20495020616464726573733A84
:101AF000004572726F723A20726562696E64206688
:101B000061696C0052656E65776564207375636307
:101B10006573732E20495020616464726573733A53
:101B2000004572726F723A2072656E657765642047
:101B30006661696C000A4E6F206C696E6B005265BD
:101B400073746F72696E6720636F6E666967206673
:101B5000726F6D20454550524F4D00416363657073
:101B600074696E6720636F6D6D616E64732E2E2EC7
:101B70000A004E6F204D51545420636F6E666967A2
:101B800075726564004C6F6164696E6720636F6E87
:101B90006669672066726F6D20706F7274616C2069
:101BA00064697361626C65642E2075736520676576
:101BB00074204F4E20746F20656E61626C65004327
:101BC0006F6E6669672069732076616C6964004393
:101BD0006F6E74696E7565207769746820707265C0
:101BE00076696F75736C79206C6F616465642063CE
:101BF0006F6E6669670000002100240027002A003C
:101C00002D003000330001010000040107010A012A
:101C100000002200250028002B002E003100340097
:101C200002010000050108010B0105050505070576
:101C300008080808020202020A0A08080404040448
:101C40000101010101010101030303030303030374
:101C5000040707070C0C0C0C0C0C0C0C0202020203
:101C600006060606060606060B0B0B0B0B0B0B0BEC
:101C7000050505080807070404040A0A0A0A0A0AEF
:101C8000010210202008081020401020408002018E
:101C90000201080402010102040810204080804073
:101CA0002010080402018004020180402010080472
:101CB0000201080402010102040810204080010210
:101CC0000408102040800440800480081010204048
:101CD00004081020408000000B0C030A0D0E0F09B1
:101CE00008040502000000000000000000000000E1
:101CF00000000000000000000000000000000000E4
:101D0000000013121100000000000000000000009D
:101D100000000000000000000000000000000000C3
:101D20000000000000000000000000002F6461744B
:101D300061002F736B65746368004163636573733F
:101D40002D436F6E74726F6C2D526571756573746F
:101D50002D507269766174652D4E6574776F726B64
:101D60003A2074727565004163636573732D436F28
:101D70006E74726F6C2D416C6C6F772D4865616469
:101D80006572733A202A004163636573732D436F54
:101D90006E74726F6C2D416C6C6F772D4D6574682D
:101DA0006F64733A20504F53542C4745542C4F5076
:101DB00054494F4E53004163636573732D436F6EF7
:101DC00074726F6C2D416C6C6F772D437265646516
:101DD0006E7469616C733A2074727565004F50546B
:101DE000494F4E530044454C45544500505554000E
:101DF00047455400504F535400617574686F7269C1
:101E00007A6174696F6E3A2000417574686F726907
:101E10007A6174696F6E3A2000436F6E74656E74F8
:101E20002D4C656E6774683A20006F637465742F7B
:101E300073747265616D00696D6167652F6A7065A5
:101E40006700696D6167652F6769660074657874FE
:101E50002F68746D6C006170706C69636174696F78
:101E60006E2F6A736F6E00746578742F706C616981
:101E70006E00436F6E74656E742D547970653A20F0
:101E800000436F6E6E656374696F6E3A20636C6FAA
:101E90007365004163636573732D436F6E74726F76
:101EA0006C2D416C6C6F772D4F726967696E3A20AB
:101EB000687474703A2F2F6C617A79686F6D652E33
:101EC000727500556E6B6E6F776E004E6F74204D9D
:101ED0006F646966696564004F4B004D6F76656499
:101EE000207065726D616E656E746C7900496E74F8
:101EF00065726E616C2053657276657220457272F0
:101F00006F72005061796C6F616420546F6F204C68
:101F100061726765004E6F7420666F756E6400575E
:101F200057572D41757468656E7469636174653ABD
:101F3000204261736963207265616C6D3D2241636B
:101F40006365737320726573747269637465642268
:101F500000556E617574686F72697A6564005061CE
:101F6000796C6F61642073697A652077726F6E6730
:101F70000042616420726571756573740048545441
:101F8000502F312E31200020000000000000000002
:101F900000004F4E000000000000004F46460000C9
:101FA00000000000524553540000000000544F4709
:101FB000474C4500000048414C54000000000058C8
:101FC0004F4E000000000000584F46460000000041
:101FD00000494E4352454153450044454352454113
:101FE000534500484541540000000000434F4F4C0A
:101FF00000000000004155544F0000000000464121
:102000004E5F4F4E4C5900445259000000000000F2
:1020100053544F500000000000484947480000005A
:1020200000004D454449554D0000004C4F570000FD
:1020300000000000454E41424C4500000044495319
:1020400041424C45000054525545000000000046F6
:10205000414C534500000000524742000000000080
:102060000048535600000000000057726F6E672052
:102070007061796C616400202D3E2041543A004328
:1020800068616E20747970653A004E6F2073746FCA
:102090007265642076616C756573202D20646566B9
:1020A00061756C743A200053617665642045544133
:1020B000473A0053657420455441473A2000BAC757
:1020C00098C711241FBECFEFD1E2DEBFCDBF00E025
:1020D0000CBF16E0A0E0B2E0EAECFCEB01E00BBFC5
:1020E00002C007900D92AC3EB107D9F720E1ACEEEB
:1020F000B6E001C01D92A637B207E1F710E1C0E6D5
:10210000D0E100E006C021970109802FFE010E9466
:102110001BD9CF35D10780E00807A9F70E9454B733
:102120000C9453DE0C940000CF93DF931F92CDB735
:10213000DEB76983DC01ED91FC910280F381E02D33
:1021400041E050E0BE016F5F7F4F19950F90DF9126
:10215000CF910895FC01818D928D0895CF93DF93E7
:102160001F92CDB7DEB76983DC01ED91FC9102804F
:10217000F381E02D41E050E0BE016F5F7F4F199584
:102180000F90DF91CF910895FC019485FB01848528
:10219000981303C081E0983008F080E00895CF9351
:1021A000DF931F92CDB7DEB76983DC01ED91FC911F
:1021B0000280F381E02D41E050E0BE016F5F7F4F70
:1021C00019950F90DF91CF91089585ED8093BC0014
:1021D0008091BC0084FDFCCF10927408089520917A
:1021E0005008260F3327331F21323105ECF420919C
:1021F0007408FC0190E080E0243069F082E00895EA
:10220000A09150082191AC01405D574FA40FB52F0C
:10221000B11D2C930196861798F380915008680F92
:102220006093500880E0089581E008958FEF9FEF5C
:1022300008958FEF9FEF089580912F0890E091957A
:10224000819591090895CF93DF93CB01EA01642F23
:102250000E94EF10CE01DF91CF910895CF93DF93CD
:102260001F92CDB7DEB7698361E0CE0101960E946F
:10227000EF1081E090E00F90DF91CF91089590E012
:10228000FC01E65DF34EE491F0E0EE0FFF1FE05F2E
:10229000F34EA591B4912C918058934EFC018491FA
:1022A000822391E009F490E0892F08958F929F9204
:1022B000AF92BF92CF92DF92EF92FF920F931F9354
:1022C000CF93DF9300D000D000D01F921F92CDB7E4
:1022D000DEB77C018E010F5F1F4F68018AE0882EF8
:1022E000912CA12CB12CC601801B910B41155105DD
:1022F0006105710581F0CB01BA01A50194010E942D
:1023000090D8942F852F605DF60161936F01A9012C
:10231000692F782FE8CFF801E80FF91FD701015096
:10232000110922912D93E017F107D9F7E80EF91E54
:10233000F70110822B960FB6F894DEBF0FBECDBF0B
:10234000DF91CF911F910F91FF90EF90DF90CF9091
:10235000BF90AF909F908F900895FC01DC018D910C
:102360008111FDCF30E020E050E040E08AE0919123
:10237000992301F1443051055CF59E3271F42F3FF1
:10238000310509F02CF5DB01A40FB51F12962C9333
:102390004F5F5F4F30E020E0EACF829FD001839F04
:1023A000B00D1124292F990F330B205331092A0F17
:1023B0003B1FDDCF2F3F310509F054F44430510568
:1023C0003CF4640F751FFB01228381E090E00895C7
:1023D00090E080E00895CF93DF931F921F92CDB7D6
:1023E000DEB780916A1090916B10009711F486E728
:1023F00090E1BE016F5F7F4F681B790B072E000CC9
:10240000880B990B0F900F90DF91CF910895DC010D
:1024100015968D919C91009739F0DC01ED91FC911E
:102420000680F781E02D19940895089583E090E0E7
:1024300008958091D7079091D80708950895DC01F9
:102440001296ED91FC9113973097B9F016968D91F5
:102450009C918430910541F08530910541F00397BE
:1024600049F482E090E0089581E090E0089581E1F0
:1024700090E00895808590E0089590E080E00895D0
:102480008091D5079091D6070895089590E080E057
:1024900008958091D3079091D407089584E090E047
:1024A0000895DC011496ED91FC91309729F080811C
:1024B000082E000C990B089590E080E0089508958F
:1024C00085E090E0089580911C0790911D07817030
:1024D0009927089580910B0790910C070895FC01AE
:1024E000848195810895FC01768765870895DC01D4
:1024F000ED91FC91068CF78DE02D199591E08927DF
:102500000895862F089581E08627089521E0FC0133
:102510008485883008F020E0822F0895FC018485AE
:1025200095850895FC0184899589089522E334E016
:10253000FC0131832083FB014089518962897389C1
:10254000FC0142835383648375830895DC01ED911C
:10255000FC91048CF58DE02D1994CF93DF9300D07E
:1025600000D01F921F92CDB7DEB7FC016F3F7105FF
:1025700019F014F06FEF70E077FD60E09181892F22
:1025800082958F7081508230C8F4648388E0DE01C8
:10259000119601900D928A95E1F729813A814B813C
:1025A0005C816D817E818F81988528960FB6F89425
:1025B000DEBF0FBECDBFDF91CF9108959F709061B8
:1025C0009183E3CF0F931F93CF93DF93DC01C62F4B
:1025D0001196EC911197E295EF70EC3008F0BCC0C9
:1025E000F0E08827E950FD4E8F4F0C941BD9031360
:1025F00028132813AC13AC13AC138A133413AC1385
:10260000AC130B130B1370E060E0CB01DF91CF91A3
:102610001F910F91089514968D919D910D90BC91ED
:10262000A02D8F3F9105A105B10529F024F08FEF72
:1026300090E0A0E0B0E0B7FF03C080E090E0DC01F4
:102640006FEF70E0681B790BC111DFCFBC01DDCFEC
:1026500014966C9170E0CC23C1F28FEF90E09C0156
:10266000261B370BB901D1CF862F14960C911497E6
:1026700015961C9115971696DC9116971796CC9186
:1026800020E030E0A901B801882331F18D2F9C2F83
:102690000E9446D787FD1BC020E030E04FE753E49F
:1026A000B8018D2F9C2F0E944EDA181624F400E0FA
:1026B00010E0DFE7C3E498014D2F5C2F60E070E08D
:1026C0008FE793E40E9439D90E9418DA9ECF00E088
:1026D00010E0D0E0C0E0EFCF8D2F9C2F0E9446D7B6
:1026E00087FD13C020E030E04FE753E4B8018D2FA1
:1026F0009C2F0E944EDA181624F400E010E0DFE769
:10270000C3E4B8018D2F9C2FDFCF00E010E0D0E0B4
:10271000C0E0F7CF14966D917D918D919C911797A4
:1027200024E630E040E050E00E94B2D82F3F31056F
:102730004105510529F024F02FEF30E040E050E052
:1027400057FF03C020E030E0A9016FEF70E0621B8B
:10275000730BC1115ACF86CF6FEF7FEF56CFCF9358
:10276000DF93EC01DB01898182958F708630E1F186
:1027700028F481508230C8F080E014C0873009F11D
:102780008A508230C8F72FEF30E00E9432D924E619
:1027900030E040E050E00E94B2D82C833D834E836D
:1027A0005F8381E0DF91CF9108952FEF30E00E94A9
:1027B00032D924E630E040E050E00E94B2D82C83C9
:1027C000F0CF2FEF30E00E9432D924E630E040E035
:1027D00050E00E94B2D8CA01B9010E944DD76C8363
:1027E0007D838E839F83DDCF2CE933E60E9432D92F
:1027F00024E630E040E050E00E94B2D82C833D83D4
:102800004E835F83B9CFDC011196EC911197E2956D
:10281000EF70E150EB3008F039C0F0E08827EC5E53
:10282000FB4E8F4F0C941BD93714371446141F14CA
:102830001F1428143F143F143F141F141F14149620
:102840006D917D918D919C9117970E944DD7089520
:1028500014966D917D918D919C91179724E630E0AF
:1028600040E050E00E94B2D8CA01B901EECF149600
:102870006C9170E090E080E00E944BD70895149630
:102880006D917D918D919C911797089560E070E016
:10289000CB010895FC01A7812A2F2E7FD1F08181E1
:1028A00082958F7081508330A0F4A695A150BB0B08
:1028B0002BE531E00E9432D924E630E040E050E0E0
:1028C0000E94B2D8DA01C90187569F4FAF4FBF4F60
:1028D00008958FEF9FEF0895DC01ED91FC91309703
:1028E00029F090859F7081E0953009F080E008958F
:1028F000FC01A481B581109721F118969C9118973D
:102900009F708EEF890F823010F091111AC01996C6
:102910004D935D936D937C931C97A481B58118961C
:102920009C911897907F926018969C930480F581F3
:10293000E02D8085982F907F903619F48F70806AF3
:1029400080870895DC0119968D919C91009739F04C
:10295000DC01ED91FC910280F381E02D1994089542
:102960008AE090E0089581E090E0089588E090E0AA
:102970000895DC01ED91FC91008CF18DE02D19940E
:10298000CF93DF93EC01E881F9810484F585E02D94
:10299000199529893A892F5F3F4F3A8B298BDF910F
:1029A000CF910895CF93DF93EC018E8581110DC0F7
:1029B00081E090E049895A892C853D85421753076B
:1029C00008F080E0DF91CF910895E881F9810484D7
:1029D000F585E02DCE0119958F3F910549F780E0EF
:1029E00090E0F0CFFC01848595856817790708F49D
:1029F000CB01928B818B0895DC011E962C911E9742
:102A0000222339F0ED91FC910190F081E02D6FEFE0
:102A100019940895FC0187859089089581E00895AF
:102A200090E080E00895FC0122813381232B49F05E
:102A3000868197818130910539F01CF003970397C7
:102A400030F090E080E0089581E090E0089582E029
:102A500090E00895CF93DF93CDB7DEB760970FB6C0
:102A6000F894DEBF0FBECDBF19821A821B821C8272
:102A70001D821E821F8218868A818F708A836FEF63
:102A800070E0CE0101960E94AD1260960FB6F894E8
:102A9000DEBF0FBECDBFDF91CF910895CF92DF9201
:102AA000EF92FF920F931F93CF93DF93CDB7DEB7D3
:102AB00060970FB6F894DEBF0FBECDBF7C016B01EF
:102AC000BA01A901CE0101960E945611D701ED91DC
:102AD000FC910288F389E02D9801AE014F5F5F4FB2
:102AE000B601C701199560960FB6F894DEBF0FBE08
:102AF000CDBFDF91CF911F910F91FF90EF90DF90AD
:102B0000CF90089590E080E00895CF92DF92EF9209
:102B1000FF920F931F93CF93DF9300D000D0CDB7D8
:102B2000DEB78C016B017A01FC01808D883010F4D6
:102B30000E947C9782E394E09A838983F6018281E4
:102B40009381A481B5818B839C83AD83BE83B701C0
:102B5000CE0101960E9403A7F801808F8830A0F46F
:102B6000F586E486128E118E81E026960FB6F894D3
:102B7000DEBF0FBECDBFDF91CF911F910F91FF90B0
:102B8000EF90DF90CF90089580E0EFCFCF93DF9369
:102B9000EC01888D883020F40E947C9788E0888F33
:102BA000DF91CF910895FC01808D883040F4218D14
:102BB000328D232B21F00E944E9690E008958FEFE6
:102BC0009FEF0895CF93DF93FC012485283028F0F0
:102BD0008FEF9FEFDF91CF910895EC010190F0818D
:102BE000E02D0084F185E02D1995892B89F38C85E2
:102BF0000E944E9690E0EECFCF93DF93FC01218DA3
:102C0000328D2115310529F48FEF9FEFDF91CF91A0
:102C10000895EC01808D4217530708F0A9010E9426
:102C20009D961816190684F7298D3A8D281B390BA5
:102C30003A8F298FEBCF0F931F93CF93DF931F9280
:102C4000CDB7DEB7FC01218D328D232B41F48FEF00
:102C50009FEF0F90DF91CF911F910F9108958C01FD
:102C600041E050E0BE016F5F7F4FFC01808D0E940C
:102C70009D96181619065CF7F801818D928D0197C3
:102C8000928F818F898190E0E4CFCF93DF931F9261
:102C9000CDB7DEB741E050E0BE016F5F7F4FFC0172
:102CA00084850E949D961816190634F4898190E057
:102CB0000F90DF91CF9108958FEF9FEFF9CFFC0137
:102CC0008485883010F40C949D9690E080E00895FF
:102CD000FC018485883010F40C94769690E080E0B6
:102CE00008950F931F93CF93DF9300D000D01F92CE
:102CF0001F92CDB7DEB78C01D80159964D915C91EA
:102D00005A974115510551F0ED91FC91048CF58DC8
:102D1000E02D70E060E0C8011995EECFF801808DDC
:102D20000E947696892BB1F148E050E0BE016F5FBA
:102D30007F4FD80158968C910E949D9618161906BF
:102D4000F4F4D801509684E0FE01319601900D9282
:102D50008A95E1F78D8190E0982F88272E81820F48
:102D6000911DF801958B848B8F81282F30E0322FB5
:102D700022278885820F932F911D928F818F28960D
:102D80000FB6F894DEBF0FBECDBFDF91CF911F917C
:102D90000F91089590E080E0F2CFCF92DF92EF9212
:102DA000FF920F931F93CF93DF93CDB7DEB7AF970B
:102DB0000FB6F894DEBF0FBECDBF7C016A0102E3FF
:102DC00014E01A8309831C861B8688EE93E0A0E03A
:102DD000B0E08D879E87AF87B88B88E094E09A87B4
:102DE0008987188F0F8B198E1A8E1B8E1C8E88E088
:102DF00089A31BA70AA71CA61DA61EA61FA6809115
:102E0000740D9091750DA091760DB091770D8EA3F4
:102E10009FA3A8A7B9A78B839C83AD83BE83188685
:102E20001F82AE01465D5F4FCE0101960E94F9AC54
:102E300081309105B1F4D701ED91FC910488F589B9
:102E4000E02D1DA30CA38CA59DA5AEA5BFA58EA3AB
:102E50009FA3A8A7B9A7A601BE016C5D7F4FC701BC
:102E60001995AF960FB6F894DEBF0FBECDBFDF91B8
:102E7000CF911F910F91FF90EF90DF90CF90089529
:102E80000F931F93CF93DF93EC018B01888D8830D4
:102E900010F40E947C97B80182E00E94C597888F49
:102EA000883050F41D870C871A8E198E81E0DF91CF
:102EB000CF911F910F91089580E0F9CF0F931F9349
:102EC000CF93DF938C01EA01FC018485883048F4BC
:102ED0000E94EC95892B39F481E090E0F80193830E
:102EE0008283D0E0C0E0CE01DF91CF911F910F919E
:102EF0000895EF92FF920F931F93CF93DF937C017E
:102F00008091E309D4E0833309F0D8E003ED19E0C0
:102F1000C0E0F801219131918F01F7018481958101
:102F20002817390729F0CF5FDC13F3CF80E006C004
:102F30008C2F0E948A978431B1F781E0DF91CF9185
:102F40001F910F91FF90EF900895CF93DF93EC01C5
:102F50008C858830D0F40E948A97843189F0882348
:102F600079F0883169F021E08C3159F4E881F981F8
:102F70000084F185E02DCE01199521E0892B09F41B
:102F800020E0822FDF91CF91089580E0FBCFCF9298
:102F9000DF92EF92FF920F931F93CF93DF93CDB702
:102FA000DEB7AF970FB6F894DEBF0FBECDBF8C0172
:102FB0006B017A0182E394E09A8389831B821C82ED
:102FC0001D821E821C861B8648EE53E060E070E086
:102FD0004D875E876F87788B28E034E03A872987B2
:102FE000988F8F8B198E1A8E1B8E1C8E28E029A32A
:102FF0009BA78AA71CA61DA61EA61FA6D8011C96C5
:103000008C91883060F40E948A97882321F0F8011F
:1030100084850E946E9788E0D8011C968C938091DD
:10302000740D9091750DA091760DB091770D8EA3D2
:103030009FA3A8A7B9A78B839C83AD83BE83188663
:103040001F82AE01465D5F4FB601CE0101960E9420
:10305000F9AC0097C1F0D801ED91FC910684F78599
:10306000E02D82E394E09DA38CA38CA59DA5AEA545
:10307000BFA58EA39FA3A8A7B9A7A701BE016C5D9A
:103080007F4FC8011995AF960FB6F894DEBF0FBEFB
:10309000CDBFDF91CF911F910F91FF90EF90DF9007
:1030A000CF9008950F931F93182F0E9406AA04C073
:1030B00096958795779567951A95D2F78B019C0120
:1030C00001501109210931090E3F1F4F2F4F3F4F6A
:1030D00020F061E070E080E090E01F910F91089592
:1030E000CF93DF93EC018C85883060F40E948A973F
:1030F000873111F08C3131F48C850E94CF95811588
:10310000984088F3DF91CF910895FC018485883041
:1031100010F40C94CF9590E080E0089562E576E19C
:103120008FE29FE00E94B4898FE29FE00E941E8898
:103130001092D4071092D30781E090E0089564E5DF
:1031400074E18FE29FE00E94B4898FE29FE00E94C9
:103150001E8810920C0710920B0781E090E00895F2
:1031600064E370E1811102C066E370E18EEF9DE0DF
:103170000C94B48960E77EE08EEF9DE00E94B489F4
:10318000F0E0E0E0199584EF91E0089567E479E0DC
:10319000811102C062E479E08FE29FE00C94B4896F
:1031A0004F925F926F927F92AF92BF92DF92EF92B7
:1031B000FF920F931F93CF93DF9300D000D0CDB732
:1031C000DEB77C01D62E80912B08882309F4BEC07F
:1031D000D70114969C9180912A02891708F4B6C0F1
:1031E0008091290890912A08BAE06B13F0C08752A9
:1031F000984FFC011082D70118960D911C91011572
:10320000110509F49FC0F80161857285611571058A
:1032100091F4458056806780708480916E0D909106
:103220006F0DA091700DB091710D481659066A0688
:103230007B0609F487C0D8011B964D915C911C97C1
:103240004115510509F47EC0F701248153968C91F4
:10325000539790E0322F377002C0959587953A9535
:10326000E2F780FF6FC0A22EB12CC501887F93705A
:10327000892B39F451968D919C91887F9370A82A5F
:10328000B92AD8018D919C91DC01ED91FC916115D9
:10329000710509F486C00688F789E02D1995019714
:1032A00009F050C06CE3F801808191810E94BD88D3
:1032B000A50170E060E02AE0D8018D919C910E9408
:1032C000D287F8012281808191816AE677E1222309
:1032D00011F068E677E10E94B489D8011D966D91DE
:1032E0007C911E978D919C910E944E8960E2F8011D
:1032F000808191810E94BD88D8011F966D917C913B
:1033000050978D919C910E944E89F8012281808175
:1033100091816DE577E1222311F067E577E10E9465
:10332000B48969ED77E0D8018D919C910E944E8916
:10333000F80180819181DC01ED91FC91008CF18D8F
:10334000E02D199510922A0810922908D701159698
:103350008D919C911697009709F44DC014963C915D
:1033600020912B02231708F446C0DC01ED91FC915B
:103370000190F081E02D6D2D199526960FB6F894E9
:10338000DEBF0FBECDBFDF91CF911F910F91FF9098
:10339000EF90DF90BF90AF907F906F905F904F90D5
:1033A00008950488F589E02D22E334E03A832983E7
:1033B000D80115964D905D906D907C9018974B823A
:1033C0005C826D827E82BE016F5F7F4F67CF8F34DC
:1033D00091050CF0BBCFBDE06B1709F4B7CF9C0192
:1033E0002F5F3F4F30932A08209329088752984F28
:1033F000FC016083ABCF81E090E0BFCF0C94D0CBD9
:103400000C94D0CB0C94D0CB0C94D0CB0C94D0CBD0
:10341000CF93C1E068EE73E080E090E00E94D4A911
:103420004AE050E06C2F8EEF9DE00E942288CF5F33
:10343000C43181F784EF91E0CF910895CF93DF936A
:10344000009709F484C0FC012081222309F47FC085
:10345000EC0168EE79E00E9470CE892B09F456C029
:103460006FEB79E0CE010E9470CE892B09F451C038
:103470006EE777E0CE010E9470CE892B09F44CC034
:103480006AE777E0CE010E9470CE892B09F447C02D
:1034900066E777E0CE010E9470CE892B09F442C026
:1034A00062E777E0CE010E9470CE892BF1F16EE6E3
:1034B00077E0CE010E9470CE892BD1F16AE677E0E9
:1034C000CE010E9470CE892BB1F165E677E0CE0186
:1034D0000E9470CE892B91F161E677E0CE010E94C7
:1034E00070CE892B71F16CEE79E0CE010E9470CE26
:1034F000892B51F16DE577E0CE010E9470CE892BCA
:1035000031F58CE090E0DF91CF91089582E090E07A
:10351000FACF81E090E0F7CF88E090E0F4CF85E04B
:1035200090E0F1CF86E090E0EECF87E090E0EBCF47
:1035300089E090E0E8CF8AE090E0E5CF8BE090E092
:10354000E2CF83E090E0DFCF84E090E0DCCF90E05A
:1035500080E0D9CFCF93DF93EC016DED76E18FE280
:103560009FE00E94B4896C817D818FE29FE00E9480
:10357000799C67ED76E18FE29FE00E94B4898FE24B
:103580009FE00E941E8860E08C810E947CA81092BF
:10359000D8071092D70781E090E0DF91CF9108958E
:1035A000EF92FF921F93CF93DF93192F7B01C82FC8
:1035B000D92FD7FF03C0D195C195D10961E08C2FD8
:1035C0000E947CA882E0E816F10499F460E08C2F58
:1035D0000E944EA86CE373E18FE29FE00E94B489E1
:1035E0008FE29FE0DF91CF911F91FF90EF900C94BD
:1035F0001E88612FEF2851F46095661F6627661FAD
:103600008C2F0E944EA868E373E1E6CF661F662701
:10361000661F8C2F0E944EA863E373E1DDCFCF932A
:10362000DF93EC01FB01248135814081518162816E
:1036300073810E94C488CE01DF91CF910895EF92EB
:10364000FF920F931F93CF93DF93EC018B011D82A9
:103650001C821A821B82E880F980E114F10409F4CB
:103660005DC08091060790910707892B09F456C029
:10367000672B09F48701F80180858F708630A9F4E3
:1036800060E474E0C8010E94F79B009719F0FC0108
:1036900081858A836DED76E0C8010E94F79B0097D3
:1036A00009F443C0FC0181858B8362E474E0C701A7
:1036B0000E94F79B009779F565E177E08FE29FE044
:1036C0000E94B4894AE050E06B818FE29FE00E9443
:1036D000228863E177E08FE29FE00E94B4894AE0AC
:1036E00050E06A818FE29FE00E9422888FE29FE093
:1036F0000E941E8820E030E0A90162E474E0888125
:1037000099810E94ACA062E474E0888199810E9452
:10371000F79B009719F009969D838C83DF91CF91D9
:103720001F910F91FF90EF900895F8018081918192
:103730000E9404CEB9CFCF93DF9300D000D01F9268
:103740001F92CDB7DEB7E9EEFDE0128A118A80E064
:1037500090E19587848784E890E0948B838B81E067
:10376000868780E090E2908B87871C821B8282E2B2
:1037700093E09A838983FE83ED838FEF9FEF988791
:103780008F836FEB73E18EEF9DE00E94B4896091AF
:10379000060770910707CE0101960E94B88F89EE47
:1037A0009DE00E94B9146FEA73E18EEF9DE00E94E4
:1037B000B4898EEF9DE00E941E880E94A8AF2896D3
:1037C0000FB6F894DEBF0FBECDBFDF91CF91089545
:1037D000FC0186819781009799F0FC0120852F706C
:1037E000223029F46185728583859485089525307A
:1037F00039F460E00E946C9C009711F0FC01F2CF5C
:1038000060E070E0CB0108950F931F93CF93DF9397
:10381000FC01C281D3812097F9F088858F708230B6
:1038200049F4672BC9F489859A85DF91CF911F915F
:103830000F910895853081F48B01CE010E94819C07
:103840008017110649F044F0602FCE010E946C9C55
:10385000FC0181859285E9CF90E080E0E6CFFC0114
:103860006115710519F48481958108958681978188
:10387000681779072CF084819581860F971F08952A
:10388000828193810C94041CCF93DF93EC0164EB51
:1038900076E18FE29FE00E94B4896C817D818FE2A6
:1038A0009FE00E94799C6EEA76E18FE29FE00E94A1
:1038B000B4898FE29FE00E941E88E881F981028C22
:1038C000F38DE02DCE0119958130910529F00297F5
:1038D00059F060E08C811AC063E070E0CE010E9474
:1038E0002F1C60E00E947CA860E08C810E947CA874
:1038F00061E070E0CE010E942F1C60E00E947CA875
:1039000062E070E0CE010E942F1C60E00E947CA863
:103910001092D6071092D50781E090E0DF91CF9109
:103920000895CF93DF93EB0163E0FC0180819181E7
:103930000E946C9CFC01892BA9F080858D7091F40C
:10394000C095D095CF6FAE0170E060E08185928523
:10395000A385B4858C239523A623B72381879287DB
:10396000A387B487DF91CF910895CF93DF93EB01C5
:1039700063E0FC01808191810E946C9CFC01892B99
:10398000B9F09085892F8D7099F4907F926090871F
:10399000CC27CE01B0E0A0E04185528563857485D7
:1039A000842B952BA62BB72B81879287A387B4876F
:1039B000DF91CF910895CF93DF93EB0163E0FC019A
:1039C000808191810E946C9C009761F0FC012085B0
:1039D0002F70223039F4818592858C239D23DF91CD
:1039E000CF91089590E080E0FACFCF93C62F63E0A7
:1039F000FC01808191810E946C9CFC01892B29F142
:103A00009085892F8D7009F5907F926090878185D0
:103A10009285A385B4858827AA27BB278C2B81870D
:103A20009287A387B48763E877E08FE29FE00E94E4
:103A3000B4894AE050E06C2F8FE29FE00E94228818
:103A40008FE29FE0CF910C941E88CF91089563E0A0
:103A5000FC01808191810E946C9C009719F0FC010F
:103A6000818508958FEF0895FF920F931F93CF9351
:103A7000DF93CDB7DEB764970FB6F894DEBF0FBE05
:103A8000CDBF8C01F62E8FE290E09A838983FE01F0
:103A9000339688E0DF011D928A95E9F7F801668187
:103AA000FF2011F081E06827D80114968C910E94C4
:103AB0004EA8F80187819085A185B285883E934004
:103AC000A105B10508F48BC063E277E18FE29FE0C6
:103AD0000E94B489D80114966D917C918FE29FE089
:103AE0000E94799C6EE177E18FE29FE00E94B489A9
:103AF0006F2D70E08FE29FE00E94799C8FE29FE043
:103B00000E941E8865E477E1CE0101960E9465CE91
:103B1000F801828193810E94271DFF2009F46BC068
:103B20006BE077E18D3051F06FE077E18E3031F06E
:103B300066E177E18B3011F063E077E1CE010B961F
:103B40000E9479CE6EEE76E18FE29FE00E94B4890A
:103B5000D8011296ED91FC9113970190F081E02D20
:103B600060817181ED91FC910288F389E02D9E01C5
:103B70002F5F3F4FAE01455F5F4FC8011995BC01F4
:103B80008FE29FE00E94799C6CEE76E18FE29FE0ED
:103B90000E94B489D8011296ED91FC910190F081B8
:103BA000E02D608171818FE29FE00E944E89BE010D
:103BB0006F5F7F4F8FE29FE00E944E8969EE76E152
:103BC0008FE29FE00E94B489BE01655F7F4F8FE264
:103BD0009FE00E944E898FE29FE00E941E886496BB
:103BE0000FB6F894DEBF0FBECDBFDF91CF911F910E
:103BF0000F91FF9008956FEF76E1823009F49ECF28
:103C00006AEF76E19BCF81E090E00895CF93DF9358
:103C1000EC0164EA76E18FE29FE00E94B4896C8156
:103C20007D818FE29FE00E94799C6EE976E18FE2D0
:103C30009FE00E94B4898FE29FE00E941E888A81E3
:103C40009B81892B09F44DC08C819D81892B09F0C2
:103C500048C0E881F981028CF38DE02DCE011995E1
:103C60008130910529F0029759F061E08C811AC0EA
:103C700063E070E0CE010E942F1C61E00E947CA8EE
:103C800061E08C810E947CA861E070E0CE010E941E
:103C90002F1C61E00E947CA862E070E0CE010E94CF
:103CA0002F1C61E00E947CA88091A100887F8093F6
:103CB000A10080919100887F809391008091A10064
:103CC00082608093A1008091910082608093910036
:103CD00081E090E09093D6078093D507DF91CF9154
:103CE000089590E080E0FACFCF93DF93DC01149643
:103CF000ED91FC91309709F44FC0C681D781209790
:103D0000C1F1E881F981309781F18081882369F1DF
:103D100064ED74E0CE010E94F79B892B41F42FEFF4
:103D20003FEFA90164ED74E0CE010E94ACA065EE06
:103D300074E0CE010E94F79B892B41F42FEF3FEFF7
:103D4000A90165EE74E0CE010E94ACA065E474E0C8
:103D5000CE010E94F79B892B41F42FEF3FEFA90181
:103D600065E474E0CE010E94ACA00A80DB81C02D26
:103D7000C6CF63E476E18FE29FE00E94B4898FE2D0
:103D80009FE00E941E8881E090E09093D40780938A
:103D9000D307DF91CF9108956BE276E18FE29FE048
:103DA0000E94B4898FE29FE00E941E8890E080E02C
:103DB000F0CF6CE474E18FE29FE00E94B4898FE25F
:103DC0009FE00E941E8826E040E855E260E070E037
:103DD00086EF99E00E946B8E81E090E090930C0753
:103DE00080930B070895892B71F0FB0182819381E9
:103DF0000E949E9D6DEA7FE08EEF9DE00E94B48957
:103E000088EC90E0089590E080E0F2CF892B71F08B
:103E1000FB01828193810E943B9D66E97FE08EEFEA
:103E20009DE00E94B48988EC90E0089590E080E0E5
:103E3000F2CF8091DB0D9091DC0D892B51F00E9427
:103E4000D2B0882331F066E87FE08EEF9DE00E94DB
:103E5000B4891092FB0D1092FA0D80E090E19093DE
:103E6000F60D8093F50D84E890E09093FD0D80931E
:103E7000FC0D81E08093F70D80E090E29093F90DC6
:103E80008093F80D89EE9DE00E94FC1489EE9DE080
:103E90000E94B91488EC90E00895EF92FF920F937E
:103EA0001F93CF93DF93CDB7DEB72C970FB6F8945F
:103EB000DEBF0FBECDBF8C017B0182E394E09A830D
:103EC00089831B821C821D821E8298878F8319869C
:103ED0001A861B861C8605301105ECF0BE01695F51
:103EE0007F4FF701808591850E94AD11892B99F054
:103EF000CE0107960E946C9EBE01695F7F4FF7015D
:103F0000868197810E94AD11892B61F0CE010796C1
:103F10000E94429F0EC0CE0101960E946C9E04300A
:103F2000110554F7CE0101960E94429F03301105FE
:103F30008CF1BE01695F7F4FF701848195810E94FA
:103F4000AD11892B39F1CE0107960E94D79EBE0193
:103F5000695F7F4FF701828193810E94AD11892BA8
:103F600001F1CE0107960E94019E6FE67FE08EEF81
:103F70009DE00E94B48988EC90E02C960FB6F894EE
:103F8000DEBF0FBECDBFDF91CF911F910F91FF908C
:103F9000EF900895CE0101960E94D79E0230110540
:103FA000B4F6CE0101960E94019E01301105E9F69A
:103FB000CE0101960E94019E66E77FE08EEF9DE0B4
:103FC0000E94B489D2CF0F931F93CF93DF938C01BC
:103FD000EB010297C4F08A819B810E9404CE8093FA
:103FE0002B0299270E947AA00230110549F08C819A
:103FF0009D810E9404CE80932A0299270E9484A06A
:10400000C8ECD0E002C0C0E9D1E06BE57FE08EEF04
:104010009DE00E94B4894AE050E060912B028EEF4F
:104020009DE00E94228866E47FE08EEF9DE00E9482
:10403000B4894AE050E060912A028EEF9DE00E9430
:1040400022888EEF9DE00E941E88CE01DF91CF91E5
:104050001F910F910895CF93DF93EB010297A4F185
:1040600061E370E18A819B810E9452CE892B29F401
:104070000E94AD9F6F770E940AA06DE270E18A8175
:104080009B810E9452CE892B29F40E94AD9F6068CB
:104090000E940AA065E37FE08EEF9DE00E94B48954
:1040A0000E94AD9F6095661F6627661F70E08EEFC9
:1040B0009DE00E94799C8EEF9DE00E941E8888EC16
:1040C00090E0DF91CF9108950E949B1BF8CF2F9233
:1040D0003F924F925F926F927F928F929F92AF9298
:1040E000BF92CF92DF92EF92FF920F93CF93DF9325
:1040F00000D01F92CDB7DEB77C017A8369835C83E1
:104100004B83DB011C92FC016081662309F44DC0E6
:1041100030FF4BC0F9E06F9FB00111246757704E1C
:10412000CD010E94A7CED70111968C91807F41F0DE
:104130004B815C8169E474E089819A810E948CDD05
:10414000E981FA8101900020E9F7319789819A810C
:10415000E81BF90B1C012E0E3F1EAB81BC81AE1B70
:10416000BF0B1197BC83AB83D7011196EC911197CC
:104170008E2F807F09F4BCC0E295EF70E150EC30E7
:1041800008F0B6C0F0E08827E753FF4D8F4F0C943E
:104190001BD9D8204721AD2112222D221421C32161
:1041A000C321C3210821FC20492229803A80DCCF89
:1041B000F7018481282F30E050E040E0002359F0DF
:1041C00030E0A4E6B0E00E94E4D82FEF30E040E019
:1041D00050E00E94B2D85F934F933F932F938BE4AC
:1041E00094E09F938F93FC81FF938B818F933F92F9
:1041F0002F920E94C4DD77C0F70187818F9386815B
:104200008F9385818F9384818F938EE494E0E9CF9F
:10421000F70187818F9386818F9385818F93848126
:104220008F9382E594E0DDCFF701C480D580E680EE
:10423000F780C701B60124E630E040E050E00E947C
:10424000B2D897FF07C090958095709561957F4F84
:104250008F4F9F4F9F938F937F936F93C701B601AB
:1042600024E630E040E050E00E94B2D85F934F93E4
:104270003F932F9386E594E09F938F93FC81FF9368
:104280008B818F933F922F920E94C4DD2CC0C70177
:104290000E944A14BC01F701C680D780D0FADD2401
:1042A000D0F89481F580EB80BC80292F30E050E07D
:1042B00040E077FD35C0011135C07F936F931F92A9
:1042C0001F921F929F931F92FF92DF92CF928FE5D2
:1042D00094E09F938F939C819F93AB81AF933F9288
:1042E0002F920E94C4DD0FB6F894DEBF0FBECDBF83
:1042F00089819A810F900F900F900F90DF91CF914D
:104300000F91FF90EF90DF90CF90BF90AF909F9074
:104310008F907F906F905F904F903F902F90089577
:10432000002361F0292F30E0A4E6B0E00E94E4D839
:104330002FEF30E040E050E00E94B2D85F934F93FF
:104340003F932F931F92FF92DF92CF9282E694E0E9
:104350009F938F93BF92EF9295CF15968C9115975F
:104360001F928F9316969C91169717968C91817039
:104370008F939F9385E694E09F938F93BC81BF9327
:10438000EB81EF9334CF14968D909D90AD90BC90BF
:10439000179720E030E0A901C501B4010E9446D77B
:1043A0002401350187FF04C077FA709477F8709480
:1043B000C301B2010E9418DA6B01072E000C880BB2
:1043C000990B0E944DD79B01AC01C301B2010E9421
:1043D00039D920E030E04AE754E40E94ACD70E948B
:1043E000A3DA0E9418DA062F772E20E030E0A90128
:1043F000C501B4010E9446D787FF07C07F920F9383
:10440000DF92CF928BE694E0B7CF7F920F93DF924B
:10441000CF928CE694E09F938F939C819F93AB8186
:10442000AF93E5CE14968C9114971F928F931596A7
:104430008C9115971F928F9316968C911F928F9344
:1044400082E694E09F938F93BC81BF93EB81EF93BF
:104450003F922F920E94C4DD46CF17968C911797FA
:104460001F928F9314968C9114971F928F93159689
:104470008C9115971F928F9316968C911F928F9304
:104480008FE594E09F938F93BC81BF93EB81EF9373
:10449000F9CE14966D917C914B815C81C1010E9493
:1044A000AADD26CFCF92DF92EF92FF920F931F9358
:1044B000CF93DF93EC01888199810E94819C082F22
:1044C00010E0043011059CF40E94BD91009739F072
:1044D000DC0118962C911897207F18962C93BC011C
:1044E000888199810E9490A00F5F1F4FEACFC880FA
:1044F000D98060E0C6010E946C9CFC01F184F886C2
:1045000061E0C6010E946C9C8C019B838A8362E0FF
:10451000C6010E946C9C9D838C8364E0C6010E944E
:104520006C9C6C019F838E83F0E1FF1609F48AC0B6
:10453000FF1580F083E0F81689F1AAE0FA1609F475
:1045400073C0DF91CF911F910F91FF90EF90DF909B
:10455000CF900895B2E1FB1609F4F3C0E3E1FE1237
:10456000F0CF86E090E00E9434CBFC01D383C2837D
:104570008CE392E091838083C114D10409F4FCC0E0
:10458000D60118968C9118978F70823009F0F4C07C
:1045900016968D919C9195838483EBC08AE090E080
:1045A0000E9434CB7C01DC011396DC93CE931297EE
:1045B0008EE592E08D939C9370E060E0CE010E94C6
:1045C000041C97FD22C0F701958384830115110512
:1045D00041F1F80180858F70823001F1853009F555
:1045E000C8010E94819C90E0D70117969C938E93FE
:1045F000169782E892E011969C938E9319961C92DE
:104600001E921897FA86E9869CCF9195819591091B
:10461000D70115969C938E931497D8CF81E090E0A4
:10462000E3CF90E080E0E0CF84E090E00E9434CBE4
:10463000FC01D383C2832AEE32E0318320839A8740
:1046400089877FCF8BE090E00E9434CB7C01DC0136
:104650001396DC93CE93129788EC92E011969C937C
:104660008E9316961C9270E060E0CE010E94041CAE
:1046700097FD46C0F70195838483F7018481958176
:10468000009719F0863591053CF080E290E0D70163
:1046900015969C938E9314970115110509F443C048
:1046A000F80180858F708530F1F5C8010E94819CEA
:1046B0008230C8F161E0C8010E946C9CFC01892B2A
:1046C00091F180858F70823039F56185728583859F
:1046D00094850E944DD720E030E04AE754E40E94E0
:1046E000ACD70E941FDA6115710581059105F9F0BB
:1046F000D70117966D937D938D939C931A9782CFD4
:10470000919581959109D70115969C938E93149755
:1047100081E016968C93B1CF833029F46185728540
:1047200083859485D8CF60E070E0CB01D4CF88E852
:1047300093E1A0E0B0E0F70187839087A187B2877B
:1047400061CF86E090E00E9434CBFC01D383C2832A
:1047500086EA92E091838083158214820115110507
:1047600041F0D80118968C918F70863011F4158322
:104770000483FA87E987E5CE90E080E00CCFCF9301
:10478000DF93EC01798368831A8619861B861C8E59
:104790001B8E0E946C14882329F0CE01DF91CF91EB
:1047A0000C945222DF91CF910895EF92FF920F93D4
:1047B0001F93CF93DF93EC017B018E819F81892B27
:1047C000D9F4888199810E94819C082F10E00530DE
:1047D000110594F40E94BD91009721F0FC01208501
:1047E000207F20879F838E83BC01888199810E94CE
:1047F00090A00F5F1F4FEBCFEE81FF813097D9F074
:104800008085982F9F70A9F4807F82608087EE81D9
:10481000FF811186128613861486EE81FF81F7824E
:10482000E682C701DF91CF911F910F91FF90EF902A
:104830000895923061F3F12CE12CF3CFCF93DF9305
:10484000EC016CE775E18FE29FE00E94D8898C81D2
:104850009D810E94D0CB70E060E08A819B810E94A4
:10486000D5231D821C8281E090E0DF91CF910895D5
:10487000CF92DF92EF92FF920F931F93CF93DF932C
:10488000EC018C819D81892B61F40A811B8185E07B
:1048900090E00E9434CBBC01C8010E94D5239D83C7
:1048A0008C83EC80FD80E114F104A9F464E675E1E9
:1048B00088E09EE00E94B48988E09EE00E941E8805
:1048C00090E080E0DF91CF911F910F91FF90EF90EA
:1048D000DF90CF9008951092CE071092CD071092DE
:1048E000C8071092C7071092CF071092D0071092F6
:1048F000D1071092D2071092C9071092CA071092DE
:10490000CB071092CC071092450710928707EA81D7
:10491000FB81309759F082819381009739F0DC0157
:1049200018962C912F70263009F468C06DE175E15E
:1049300088E09EE00E94B48961E070E08C819D81F6
:10494000892B11F470E060E088E09EE00E94799C81
:104950006BE175E188E09EE00E94B48961E070E05F
:104960008A819B81892B11F470E060E088E09EE0F1
:104970000E94799C69E175E188E09EE00E94B4891B
:10498000EA81FB8161E070E082819381892B11F4DF
:1049900070E060E088E09EE00E94799C67E175E14C
:1049A00088E09EE00E94B489EA81FB810280F38165
:1049B000E02D80858F7061E070E0863011F470E04A
:1049C00060E088E09EE00E94799C65E175E188E006
:1049D0009EE00E94B48988E09EE00E941E8866E303
:1049E00075E188E09EE00E94B48988E09EE00E9424
:1049F0001E88EC81FD8182E0808362CF64E774E0F1
:104A00000E94F79B009709F4A8C0FC0120852F7035
:104A1000243009F0A2C0C184D284B6018FE29FE0A5
:104A20000E944E8961E175E18FE29FE00E94B489A6
:104A300010E000E0C114D10409F486C0B801675346
:104A40007B4EC6010E9470CE892B09F077C0F80119
:104A5000E353FB4E25913491922F832FD701139668
:104A60009C93139714968C93EA81FB816BE774E017
:104A7000828193810E94F79BEC81FD81009709F46C
:104A800072C0DC0118962C9118972F70223009F013
:104A90006AC019964D915D916D917C911C9741155D
:104AA00051056105710509F45EC05283418341815E
:104AB0005281052E000C660B770B238180E39CE06E
:104AC0000E946B8EEC81FD8141815281052E000C8C
:104AD000660B770B238183E19BE00E946B8EEA815A
:104AE000FB816AEF74E0828193810E94F79B0097BB
:104AF00039F0FC0181859285909386078093850724
:104B00006CE475E18EEF9DE00E94B489EA81FB813F
:104B10000190F081E02D608171818EEF9DE00E9417
:104B20004E898EEF9DE00E941E88EC81FD8181E020
:104B300080838093290281E090E0C4CE0A5F1F4FFA
:104B40000834110509F076CF6CEA74E18FE29FE03A
:104B50000E94B48996E080E081CF86E090E0F70182
:104B60009483838381CF80E09BE4928381839FCF72
:104B7000CF92DF92EF92FF920F931F93CF93DF9329
:104B8000EC016A017B018E819F81892BD9F4888198
:104B900099810E94819C082F10E00530110594F442
:104BA0000E94BD91009721F0FC012085207F208785
:104BB0009F838E83BC01888199810E9490A00F5FA2
:104BC0001F4FEBCFEE81FF81309749F18085982F01
:104BD0009F7019F5807F82608087EE81FF81C1869A
:104BE000D286E386F4866BE877E08FE29FE00E944E
:104BF000B4892AE030E0B701A6018FE29FE00E946D
:104C0000C4888FE29FE0DF91CF911F910F91FF90B9
:104C1000EF90DF90CF900C941E889230F1F2DF91EC
:104C2000CF911F910F91FF90EF90DF90CF9008955B
:104C3000EF92FF920F931F93CF93DF93EC017B01D1
:104C40008A0101501109A80186EF99E00E94F37EC4
:104C5000F701329660E0CF018E199F098017910706
:104C600018F48191680FF7CF86EF99E00E94C07F1A
:104C70000A80DB81C02D80E00E945218AB01BC018C
:104C8000CE010E94B82560E874E08FE29FE00E94A8
:104C90004E89E701CE018E199F0980179107A0F474
:104CA000688140E150E06A3048F469E874E08FE2DE
:104CB0009FE00E944E8940E150E068818FE29FE0D2
:104CC0000E9422882196E6CF8FE29FE0DF91CF916C
:104CD0001F910F91FF90EF900C941E881F93CF931C
:104CE000DF93FC01162FC389D489818992899C01A5
:104CF0002F5F3F4F328B218BC80FD91FCE010E94EF
:104D00006AD8181721F0612FCE010E9472D881E075
:104D100090E0DF91CF911F910895FC0181899289E4
:104D2000248535858217930740F423893489820FBF
:104D3000931F0E946AD890E008958FEF9FEF089527
:104D40002F923F924F925F926F927F928F929F929B
:104D5000AF92BF92CF92DF92EF92FF920F931F9389
:104D6000CF93DF93CDB7DEB762970FB6F894DEBF6F
:104D70000FBECDBF5C014B0129013A01CA01B90147
:104D80000E9418DA1B013F926F9388E694E09F938C
:104D90008F93CE0101967C019F938F930E9401DE39
:104DA0000F900F900F900F900F900F9020E030E039
:104DB000A901C301B2010E944EDA181624F077FA55
:104DC000709477F87094F70101900020E9F731971B
:104DD0006F01CE18DF088EE28083A2E0B0E0AC0F56
:104DE000BD1FAC0DBD1DBA8BA98BB10137FE03C031
:104DF000719561957109072E000C880B990B0E9423
:104E00004DD79B01AC01C301B2010E9439D920E00A
:104E100030E040E251E40E94ACD70E9418DA605DB5
:104E2000E989FA896083FE01EC0DFD1D1382D5012D
:104E3000ED91FC910288F389E02D9801A701B4015E
:104E4000C501199562960FB6F894DEBF0FBECDBFAF
:104E5000DF91CF911F910F91FF90EF90DF90CF9056
:104E6000BF90AF909F908F907F906F905F904F908A
:104E70003F902F900895DA01E0919A08F0E0FE2F1C
:104E8000EE27E60FF71F90E0982F8827A901BD01B4
:104E90008E0F9F1F0C944193CF93DF931F92CDB73A
:104EA000DEB720919A0830E0322F2227260F371FD5
:104EB00090E0982F8827498341E050E0BE016F5F62
:104EC0007F4F820F931F0E9441930F90DF91CF91EC
:104ED0000895CF93DF931F92CDB7DEB741E050E046
:104EE000BE016F5F7F4F0E94B69289810F90DF9164
:104EF000CF91089520919A0830E0322F2227620F37
:104F0000731F90E0982F8827860F971F0C946927AE
:104F100063E070E00C947A279F92AF92BF92CF9299
:104F2000DF92EF92FF920F931F93CF93DF93EC01E9
:104F30007B018091E309811121C01B821A8288EED6
:104F400093E0A0E0B0E08C839D83AE83BF838CEBC5
:104F500093E09983888388E08C8788EE93E09E872E
:104F60008D87CE01DF91CF911F910F91FF90EF9030
:104F7000DF90CF90BF90AF909F90089534E0932E34
:104F8000833311F028E0922E83EDC82E89E0D82ECD
:104F900010E098E0B92EA12CD6012D913D916D0124
:104FA000F701848195812817390791F4812F0E9498
:104FB0008A97082F873111F08C3139F5812F0E94A3
:104FC0007696892B59F50C3119F4812F0E946E9732
:104FD0001F5F9112E1CFA11008C0D701ED91FC91A4
:104FE0000084F185E02DC70119951B821A8288EE95
:104FF00093E0A0E0B0E08C839D83AE83BF838CEB15
:1050000093E099838883BC86A8CF843149F08111CD
:10501000DFCFF601329711821082DACFB12ED8CFCE
:10502000AA24A394D5CF8F929F92AF92BF92CF9292
:10503000DF92EF92FF920F931F93CF93DF93CDB741
:10504000DEB72F970FB6F894DEBF0FBECDBF5C0161
:105050004B017A018091E3098823C9F104E083338D
:1050600009F008E0B501CE0101960E948C2783ED7E
:10507000C82E89E0D82E10E0F601219131916F0100
:10508000F501848195812817390751F4812F0E94F9
:105090008A97873129F4A701B401812F0E94EC95EA
:1050A0001F5F0113E9CFC7012F960FB6F894DEBF3B
:1050B0000FBECDBFDF91CF911F910F91FF90EF9069
:1050C000DF90CF90BF90AF909F908F900895F12C7C
:1050D000E12CE9CFDA01E0919A08F0E0FE2FEE270B
:1050E000E60FF71F90E0982F8827A901BD018E0FCA
:1050F0009F1F0C94B69244E050E0BC018FE090E01A
:105100000C94419344E050E0BC0185E090E00C94A5
:10511000419344E050E0BC0181E090E00C94419365
:1051200008959F92AF92BF92CF92DF92EF92FF923B
:105130000F931F93CF93DF938C015B01942EE52E89
:10514000FC01C688D788F08C80E591E00E9440A5DC
:105150008F2D0E949295C92DDE2D8C179D0708F486
:10516000EC019E01A501B6018F2D0E940F95F8015B
:10517000868997898C0F9D1F978B868BCE01DF9137
:10518000CF911F910F91FF90EF90DF90CF90BF9044
:10519000AF909F900895CF93FC01C08D80E591E082
:1051A0000E9440A560E270E08C2F0E94A69262E00F
:1051B00070E08C2F0E947A2784FD16C062E070E0B8
:1051C0008C2F0E947A2783FF0AC048E162E070E0DA
:1051D0008C2F0E944C2780E090E0CF91089580E5CD
:1051E00091E00E9440A5E3CF40E162E070E08C2FA7
:1051F0000E944C2781E0F0CFFF920F931F93CF9333
:10520000DF93EB01FC01178A168A2A81211109C05C
:105210002B81211106C02C81211103C02D81222355
:1052200001F141155105E9F08A01FC01F08C80E59E
:1052300091E00E9440A5AE014E5F5F4F24E030E058
:105240006CE070E08F2D0E943B27B8018F2D0E94EB
:10525000999781E090E0DF91CF911F910F91FF909E
:10526000089580E0F7CF0F931F93CF938C01FC013B
:105270006481758181E20E94C597C82F8830F8F457
:1052800080E591E00E9440A58C2F0E948827833101
:1052900031F08C2FCF911F910F910C946E9762E09B
:1052A00070E08C2F0E94A692F80184819581EC2FEA
:1052B000F0E0EE0FFF1FED52F64F91838083CF9108
:1052C0001F910F9108950F931F93CF93DF931F9218
:1052D0001F92CDB7DEB7FC0124852830E0F48C01A5
:1052E00080E591E00E9440A522E030E0AE014F5FF2
:1052F0005F4F60E170E0F80184850E946A2889812F
:105300009A819827892798270F900F90DF91CF9146
:105310001F910F91089590E080E0F6CF0F931F93B7
:10532000CF93DF931F921F92CDB7DEB7FC01248588
:105330002830E0F48C0180E591E00E9440A522E055
:1053400030E0AE014F5F5F4F64E070E0F8018485AC
:105350000E946A2889819A819827892798270F9027
:105360000F90DF91CF911F910F91089590E080E011
:10537000F6CFCF93DF93EC0182E394E099838883A7
:105380001A821B821C821D8280E591E00E9440A54A
:10539000BE016E5F7F4F44E050E08FE090E00E94DE
:1053A000B692CE01DF91CF9108950E940294882396
:1053B00031F08091E309843329F0873381F090E064
:1053C00080E0089580E591E00E9440A585E390E0AB
:1053D0000E94692785FD0DC082E090E0089580E578
:1053E00091E00E9440A58EE290E00E94692780FF34
:1053F000F3CF81E090E008951F920F920FB60F92C5
:1054000011240BB60F922F933F934F935F936F939B
:105410007F938F939F93AF93BF93EF93FF9380916D
:10542000B900887F803609F44DC008F040C088324A
:1054300009F4A7C028F5803109F49BC0C8F488237B
:1054400009F4F7C0883009F494C0FF91EF91BF913F
:10545000AF919F918F917F916F915F914F913F910C
:105460002F910F900BBE0F900FBE0F901F901895AD
:10547000883109F486C0803241F78093730814C0E4
:10548000803409F49BC040F48033B9F38833E9F6E3
:105490008093730885ECAEC0803509F483C08835ED
:1054A00009F494C0883489F60E94E510CECF88397B
:1054B00009F48AC038F5883729F050F4883611F09D
:1054C000803719F683E0809374081092720855C0F3
:1054D000883809F479C0803919F0803809F0B5CFDF
:1054E00080917208803208F06FC0E091720881E00C
:1054F0008E0F809372088091BB00F0E0EE5AF74F58
:1055000080833BC0803B39F0D0F4803A09F477C007
:10551000883A09F09ACF84E0809374081092510879
:1055200010925008F0E0E0E0199580915008811148
:105530000FC081E0809350081092300809C0803C71
:1055400009F4A8CF883C09F4A5CF883B09F07DCFAA
:10555000E091510881E08E0F80935108F0E0E05D0A
:10556000F74F80818093BB00909151088091500843
:1055700029C0809199088093BB0085EC8093BC0082
:1055800064CF9091980880919708981758F5E0910A
:10559000980881E08E0F80939808F0E0E958F74F63
:1055A0008081E9CFE091980881E08E0F8093980880
:1055B0008091BB00F0E0E958F74F80839091980804
:1055C000809197089817C8F285E8D8CFE09198089D
:1055D00081E08E0F809398088091BB00F0E0E9583D
:1055E000F74F80838091760881115ECF81E08093B0
:1055F000750884EA8093BC001092740826CF85EC6D
:105600008093BC001092740880917208803230F44C
:10561000E0917208F0E0EE5AF74F10826091720844
:1056200070E082E598E0F0E0E0E0199510927208F1
:105630000CCF1092730838CF4F925F926F927F9287
:10564000AF92BF92CF92DF92EF92FF920F931F9390
:10565000CF93DF9300D01F92CDB7DEB72B013C0173
:1056600029833A834B835C83A6019501C801B70166
:10567000640D751D861D971D2115310541055105C8
:1056800011F00E9490D829813A814B815C81621788
:10569000730784079507D0F424153505460557058B
:1056A00030F521E0822F0F900F900F900F90DF9137
:1056B000CF911F910F91FF90EF90DF90CF90BF900F
:1056C000AF907F906F905F904F9008954616570669
:1056D0006806790650F421E089819A81AB81BC810A
:1056E00084159505A605B705E8F220E0DBCF21E09B
:1056F0004616570668067906A8F2F7CF8F929F9252
:10570000AF92BF92CF92DF92EF92FF920F931F93CF
:10571000CF93DF9300D000D000D01F92CDB7DEB77B
:105720006130710509F07BC24C010E9406AA9B0101
:10573000AC01609118077091190780911A07909138
:105740001B07A12CB12C650118E8E12E13E1F12E05
:1057500000E010E00E941C2B8823C1F080E00E9432
:105760005218609318077093190780931A07909343
:105770001B076AE774E18FE29FE00E94D8894DE041
:1057800050E062E072E0C4010E94182686EF99E0C2
:105790000E946B7F8597ACF481E090E02A960FB66B
:1057A000F894DEBF0FBECDBFDF91CF911F910F9157
:1057B000FF90EF90DF90CF90BF90AF909F908F9031
:1057C000089545E250E06EE177E086EF99E00E94AF
:1057D000A08786EF99E00E946B7F892B59F062E0E9
:1057E00070E080E090E00E94D4A986EF99E00E94EA
:1057F000497FEFCF8091420790911707891761F297
:10580000809317078091410790E09C01205F3F4FF4
:105810003093440720934307499708F0BDCF809108
:105820002B0790E09093160780931507809135071A
:1058300090E090931407809313078091370790E0CE
:1058400090931207809311078091390790E090930D
:10585000100780930F0780913B0790E090931D07FE
:1058600080931C0780913A0790E090930E078093F5
:105870000D07D401ED91FC9111970288F389E02D79
:1058800012968D919C91DC018D919C91DC016D9122
:105890007C9180913D072BE834E04AE655E080FD9D
:1058A00002C045E755E0C401199580910D0790911C
:1058B0000E0780389105A9F4D4011296ED91FC9160
:1058C00013970190F081E02D60817181ED91FC9141
:1058D0000288F389E02D22E934E04AE655E0C4016C
:1058E000199580910D0790910E07892BA9F4D40189
:1058F0001296ED91FC9113970190F081E02D60815B
:105900007181ED91FC910288F389E02D22E934E068
:1059100045E755E0C401199568E974E08FE29FE01E
:105920000E944E8960911C0770911D078FE29FE0D5
:105930000E94799C8FE29FE00E941E8880911C0744
:10594000F40120813181A281B3810D90BC91A02D01
:105950006D917C91D9015296ED91FC912FE934E043
:105960004AE655E083FD02C045E755E0C4011995BC
:10597000D401ED91FC9111970288F389E02D1296E4
:105980008D919C91DC018D919C91DC016D917C91BC
:1059900080911C0726EA34E04AE655E081FD02C00A
:1059A00045E755E0C401199520910F073091100784
:1059B000032E000C440B550BD4011296ED91FC9173
:1059C00013970190F081E02D60817181ED91FC9140
:1059D0000684F785E02D02EB14E0C401199580914F
:1059E000110790911207892BA9F4D4011296ED9119
:1059F000FC9113970190F081E02D60817181ED9110
:105A0000FC910288F389E02D29EB34E04EEB54E061
:105A1000C401199580911107909112070197A9F47B
:105A2000D4011296ED91FC9113970190F081E02D35
:105A300060817181ED91FC910288F389E02D29EB61
:105A400034E043EC54E0C401199580911107909122
:105A500012070297A9F4D4011296ED91FC911397C5
:105A60000190F081E02D60817181ED91FC910288BF
:105A7000F389E02D29EB34E04AEC54E0C401199598
:105A800080911107909112070397A9F4D4011296FF
:105A9000ED91FC9113970190F081E02D608171816F
:105AA000ED91FC910288F389E02D29EB34E04EEC76
:105AB00054E0C4011995D401ED91FC91119702882D
:105AC000F389E02D12968D919C91DC018D919C9132
:105AD000DC016D917C9180910F079091100722EB72
:105AE00034E045E755E0892B11F04AE655E0C40162
:105AF00019952091430730914407032E000C440B65
:105B0000550BD4011296ED91FC9113970190F08101
:105B1000E02D60817181ED91FC910684F785E02D87
:105B200003ED14E0C4011995209115073091160773
:105B30002F3F3105B9F0032E000C440B550BD40157
:105B40001296ED91FC9113970190F081E02D608108
:105B50007181ED91FC910684F785E02D08ED14E04C
:105B6000C40119951982809113079091140762E975
:105B700074E10097C9F065E774E181309105A1F007
:105B800060E774E18230910579F067E674E1833073
:105B9000910551F063E674E18430910529F08D366A
:105BA000910531F46FE574E1CE0101960E9479CE42
:105BB0002091130730911407032E000C440B550B52
:105BC000D4011296ED91FC9113970190F081E02D94
:105BD00060817181ED91FC910684F785E02D0EEDD9
:105BE00014E0C401199580911C07F40120813181D2
:105BF000A281B3810D90BC91A02D6D917C91D901B2
:105C00005296ED91FC9124EE34E0AE014F5F5F4F70
:105C100080FD02C045E755E0C4011995BDCD90E077
:105C200080E0BCCD8F929F92AF92BF92CF92DF92D5
:105C3000EF92FF920F931F93CF93DF937C014A0162
:105C40005901C0912C08D0912D08062F660F110B19
:105C5000209709F45CC088858F70863009F055C0A4
:105C600069EE74E0CE010E94F79B6C0182E0881619
:105C7000910449F065E474E0E3E08E16910429F0A4
:105C8000D0E0C0E006C06EEE74E0CE010E94F79B4B
:105C9000EC01C114D104D9F1F60180858F708430F4
:105CA000B1F561857285A801C7010E94AADDA8012E
:105CB00063EF74E0C7010E948CDD209779F188853D
:105CC0008F70843059F569857A85A801C7010E94D3
:105CD0008CDDA80163EF74E0C7010E948CDDA11484
:105CE000B10429F0A801B501C7010E948CDDC701EC
:105CF000DF91CF911F910F91FF90EF90DF90CF90A8
:105D0000BF90AF909F908F900895D0E0C0E0A80121
:105D10006DE777E1C7010E94A7CEC9CFF2E08F16E9
:105D2000910481F083E08816910429F060919B082A
:105D300070919C08CACFA80167E777E1C7010E946C
:105D400089CEC7CFA80164E777E1F8CFCF92DF9281
:105D5000EF92FF920F931F93CF93DF93CDB7DEB7F0
:105D6000C154D1090FB6F894DEBF0FBECDBF6C0190
:105D7000AB0130E020E060E4CE0101967C010E949E
:105D8000122EF70101900020E9F731978F010E19CB
:105D90001F09A801B701C6010E949CDD892B11F0E3
:105DA00010E000E0C801CF5BDF4F0FB6F894DEBF14
:105DB0000FBECDBFDF91CF911F910F91FF90EF905C
:105DC000DF90CF900895CF92DF92EF92FF920F93E2
:105DD0001F93CF93DF93CDB7DEB7C054D1090FB671
:105DE000F894DEBF0FBECDBF8091A2089091A308AA
:105DF000059709F449C06115710509F445C06901A9
:105E00007A018B0140E450E0CE0101960E94AADDA8
:105E10006FE270E0CE0101960E9471DD892B41F4A2
:105E2000980143E050E060E4CE0101960E94122EFA
:105E30004FE350E0B601CE0101960E948CDD0E9436
:105E4000129C882309F18091A2089091A3080697DB
:105E5000D9F480912E08811117C0B701CE010196A7
:105E60000E94D4AA81E090E0C05CDF4F0FB6F894A6
:105E7000DEBF0FBECDBFDF91CF911F910F91FF907D
:105E8000EF90DF90CF90089590E080E0EDCFAF925B
:105E9000BF92CF92DF92EF92FF921F93CF93DF9347
:105EA00000D000D0CDB7DEB76C017C0110E08AE0F5
:105EB000A82EB12C133061F1F701828190E0B0E09F
:105EC000A0E089839A83AB83BC83BE82AD82BE018E
:105ED0006F5F7F4F8EEF9DE00E940F1B62E777E1BF
:105EE0000E94B4891F5FFFEFEF1AFF0A143011F709
:105EF00026960FB6F894DEBF0FBECDBFDF91CF91CF
:105F00001F91FF90EF90DF90CF90BF90AF900895DA
:105F1000F601858190E0B0E0A0E089839A83AB83AD
:105F2000BC83BE82AD82BE016F5F7F4F8EEF9DE06E
:105F30000E940F1B60E777E1D3CF4F925F926F9281
:105F40007F928F929F92AF92BF92CF92DF92EF9209
:105F5000FF920F931F93CF93DF93CDB7DEB7609778
:105F60000FB6F894DEBF0FBECDBFFC0119861A86AE
:105F70001B861C869A859F7090669A87A081B18146
:105F8000109709F4EFC08C91882309F4EBC00081CD
:105F90001181D8019C91992309F4ADC09D3209F477
:105FA000E5C090539A3028F00F5F1F4F1183008394
:105FB000EECFC801DC016D01C81AD90A2D91022E5D
:105FC000000C330B205331092A303105A0F37F0137
:105FD0006EE270E0C8010E9471DDFC01009709F4D7
:105FE00048C0DC015D01AE1ABF0A11968C91119771
:105FF000082E000C990BC09711960A9798F32181EF
:10600000022E000C330B205331092A30310508F0E1
:1060100075C02A30310514F029E030E037FF02C0A6
:1060200030E020E0032E000C440B550BAAE0B0E05A
:106030000E94D1D82B013C018281082E000C990BC3
:10604000C0978A30910588F48A30910514F089E070
:1060500090E097FF02C090E080E0092E000CAA0BB0
:10606000BB0B480E591E6A1E7B1EA114B10409F019
:1060700049C0C8010E9422CE2A852F70206A2A8733
:106080002B013C016CE270E0D7018D919C910E9444
:1060900071DD009709F061C0F701118210824D8611
:1060A0005E866F86788A88E0FE013996DE01119659
:1060B00001900D928A95E1F729813A814B815C81AB
:1060C0006D817E818F81988560960FB6F894DEBFD2
:1060D0000FBECDBFDF91CF911F910F91FF90EF9039
:1060E000DF90CF90BF90AF909F908F907F906F90F8
:1060F0005F904F900895D12CC12C69CF20E030E003
:10610000A90194CFC801B3E0AB16B104ECF4E8E008
:10611000CE16D104CCF40E9422CE4B015C01A4E641
:10612000B0E0AC019B010E94D1D8B7FE08C07094CA
:10613000609450944094411C511C611C711C460E8B
:10614000571E681E791E9ECF0E9400CE2B013C0177
:106150008A858F7080678A8795CF0196D7018D9346
:106160009C939DCF412C512C320199CFC8010196AF
:1061700021CFEF92FF920F931F93CF93DF93EC0108
:10618000A881B981109761F18C91882349F1088128
:106190001981F8018081882351F08D3241F08053BC
:1061A0008A3028F00F5F1F4F19830883F0CFC80192
:1061B0000E9404CE7C016CE270E0C8010E9471DD97
:1061C000009751F419821882C701DF91CF911F9176
:1061D0000F91FF90EF900895019699838883F4CFF3
:1061E000F12CE12CF1CF61E173E18EEF9DE00E9493
:1061F000B4896EEF72E18EEF9DE00E94B48960EF8A
:1062000072E18EEF9DE00E94B48968EE72E18EEF3C
:106210009DE00E94B4898EEF9DE00E941E8868ED8B
:1062200072E18EEF9DE00E94B4896CEC72E18EEF1A
:106230009DE00E94B48964EA72E18EEF9DE00E94C5
:10624000B48967E972E18EEF9DE00E94B48962E84B
:1062500072E18EEF9DE00E94B48963E772E18EEFF8
:106260009DE00E94B4896BE672E18EEF9DE00E9492
:10627000B48960E672E18EEF9DE00E94B48966E524
:1062800072E18EEF9DE00E94B4896EE472E18EEFC0
:106290009DE00E94B48962E472E18EEF9DE00E946D
:1062A000B48968E272E18EEF9DE00E94B48969E0F2
:1062B00072E18EEF9DE00E94B48964EF71E18EEF90
:1062C0009DE00E94B4896CED71E18EEF9DE00E942B
:1062D000B4896EEC71E18EEF9DE00E94B48962ECAE
:1062E00071E18EEF9DE00E94B4896AEB71E18EEF5F
:1062F0009DE00E94B4896FEA71E18EEF9DE00E94FB
:10630000B48962EA71E18EEF9DE00E94B4896AE986
:1063100071E18EEF9DE00E94B4896FE871E18EEF2C
:106320009DE00E94B48960E871E18EEF9DE00E94DB
:10633000B48967E771E18EEF9DE00E94B48969E658
:1063400071E18EEF9DE00E94B4896BE571E18EEF03
:106350009DE00E94B4896EE471E18EEF9DE00E94A1
:10636000B4898EEF9DE00C941E880F931F93CF93FA
:10637000DF9300D000D0CDB7DEB70E94F33069EFD5
:106380007BE08EEF9DE00E94B489CE0101960E94D1
:10639000B929CE0101960E94472F02E314E01A8327
:1063A00009838091740D9091750DA091760DB09137
:1063B000770D8B839C83AD83BE83CE0101960E94B3
:1063C000472F1A8309831B821C821D821E8280E54F
:1063D00091E00E9440A544E050E0BE016D5F7F4F18
:1063E00081E090E00E94B692CE0101960E94472F74
:1063F0001A8309831B821C821D821E8280E591E024
:106400000E9440A544E050E0BE016D5F7F4F85E0F3
:1064100090E00E94B692CE0101960E94472F6FE154
:106420007CE08EEF9DE00E94B48988EC90E0269697
:106430000FB6F894DEBF0FBECDBFDF91CF911F9195
:106440000F910895009789F0FC0120852F70253069
:1064500061F40E946C9C009741F0FC0120852F7034
:10646000243019F481859285089590E080E00895A4
:10647000CF92DF92EF92FF920F931F93CF93DF9310
:1064800000D000D0CDB7DEB780912B0881119AC023
:106490008091A2089091A30802970CF493C0809178
:1064A000060790910707009709F48CC067EF74E026
:1064B0000E94F79B8C01009709F484C00E94819C84
:1064C000E82EF12CE114F10409F47CC070E060E0E6
:1064D000C8010E9422326C01EA94EF2809F481C0BD
:1064E00061E0C8010E946C9CFC0101851285CE010F
:1064F00001960E94B929CE0101960E9443A56AEE39
:106500007BE08EEF9DE00E94B489B6018EEF9DE0A6
:106510000E944E896DE775E08EEF9DE00E944E89E6
:10652000B8018EEF9DE00E94799C6DE775E08EEFDB
:106530009DE00E944E8964EE79E08EEF9DE00E941E
:106540004E898EEF9DE00E941E8862E072E08DE42D
:106550009FE00E944017D092430FC092420F1093C9
:10656000450F0093440F84EE99E0892BE9F585EF00
:1065700094E09093470F8093460F80919D089091EF
:106580009E08009741F070E060E00E9422329093F4
:106590009C0880939B0880919B0890919C08009791
:1065A00031F19093490F8093480F10924B0F109246
:1065B0004A0F81E080932B0861ED7BE08EEF9DE038
:1065C0000E94B48926960FB6F894DEBF0FBECDBFE9
:1065D000DF91CF911F910F91FF90EF90DF90CF90BF
:1065E000089502E012E083CF84EE99E0C2CF8BE3FE
:1065F00093E0892B19F485EF94E0D3CF8BE393E0FC
:10660000D0CFCF92DF92EF92FF921F93CF93DF9381
:1066100000D000D0CDB7DEB76CEC7BE08EEF9DE014
:106620000E94B48983EEE82E8DE0F82E10E090E110
:10663000C92ED12CF70181917F01803130F469E8B6
:1066400074E08EEF9DE00E944E89153041F1F70114
:106650003197808190E0B0E0A0E089839A83AB839A
:10666000BC83DE82CD82BE016F5F7F4F8EEF9DE0E7
:106670000E940F1B6AEC7BE00E94B4891F5F1630FA
:10668000C9F626960FB6F894DEBF0FBECDBFDF91D8
:10669000CF911F91FF90EF90DF90CF900895809160
:1066A000E80D90E0B0E0A0E089839A83AB83BC83DF
:1066B000DE82CD82BE016F5F7F4F8EEF9DE00E9434
:1066C0000F1B0E941E88DACFEF92FF920F931F9349
:1066D000CF93DF9300D000D01F92CDB7DEB77B0100
:1066E000CE0107969F938F9301979F938F93019766
:1066F0009F938F9301979F938F9301979F938F936E
:1067000001979F938F938E010F5F1F4F1F930F93DE
:106710008EEF94E09F938F93DB0113968C911397E8
:106720008F9312968C918F930E9431DE0FB6F8945E
:10673000DEBF0FBECDBF0697ECF463EC7FE088E0D0
:106740009EE00E94B489D70112966D917C9188E0F9
:106750009EE00E944E8980E991E027960FB6F8945A
:10676000DEBF0FBECDBFDF91CF911F910F91FF9084
:10677000EF9008958091DB0D9091DC0D892B09F449
:106780004BC00E94BA9C882309F446C0A091DB0D3F
:10679000B091DC0D52961C921E92519754961C9209
:1067A0001E92539784E890E01D969C938E931C97BD
:1067B0001E961C921E9780E090E350969C938E93B9
:1067C0001F97ED91FC9111970088F189E02D64E00D
:1067D00070E0CD0119958091DB0D9091DC0DDC010D
:1067E000ED91FC910280F381E02D46E050E0B8018C
:1067F000199586E0F801A3EEBDE001900D928A950F
:10680000E1F78091DB0D9091DC0DDC01ED91FC91C5
:106810000488F589E02D19950E94013365ED7FE02C
:106820008EEF9DE00E94B48988EC90E096CFEF92C5
:10683000FF920F93CF93DF93CDB7DEB7A0970FB63C
:10684000F894DEBF0FBECDBF7C0100E020E033E056
:1068500040E250E0BE016F5F7F4F0E946720BE01A3
:106860006F5F7F4F8FE29FE00E944E896CEB7AE072
:106870008FE29FE00E94B489F701618162956F7099
:106880004AE050E08FE29FE00E94228865EB7AE0C8
:106890008FE29FE00E94B489F70161816F704AE046
:1068A00050E08FE29FE00E9422888FE29FE00E94EA
:1068B0001E88A0960FB6F894DEBF0FBECDBFDF9145
:1068C000CF910F91FF90EF900895AF92BF92CF922A
:1068D000EF92FF920F931F93CF93DF9300D000D0DE
:1068E0001F921F92CDB7DEB75C0109831A832B83F9
:1068F0003C834D835E836F8378876CE477E18FE21E
:106900009FE00E94B489CE0101960E941734E114E1
:10691000F10439F065E477E1C7010E9470CE009779
:1069200021F1F5010281138101151105E1F0898141
:1069300081115BC08A818F70813009F45BC038F1AE
:10694000823019F1082F10E068E277E18FE29FE0D2
:106950000E94B489B8018FE29FE00E94799C8FE287
:106960009FE00E941E8890E080E028960FB6F89481
:10697000DEBF0FBECDBFDF91CF911F910F91FF9072
:10698000EF90CF90BF90AF900895CC20C1F060E021
:10699000CE0101960E94E212892B09F444C0C8017D
:1069A0000E94E81B672B682B692BE1F480E00E94B2
:1069B0005218AB01BC01C8010E94B82513C0C80120
:1069C0000E94271D8D3060F48A3010F4813051F41C
:1069D00060E0CE0101960E94E212892B19F0DFCF10
:1069E0008E30B1F381E090E0C0CF8230E1F0B0F4BE
:1069F0008130A9F268E377E18FE29FE00E94B489D9
:106A00004AE050E069818FE29FE00E9422888FE295
:106A10009FE00E941E8801E010E096CF8A508530EA
:106A200008F4BDCFE7CF40E050E0BA01C8010E94B2
:106A3000B82560E0C5010E94341DD4CFCF92DF920B
:106A4000FF920F931F93CF93DF93F12C6115710584
:106A500009F463C06A01EB018C01CB010E946C1444
:106A6000F82E882309F459C0D0FE05C0D8016C91D6
:106A7000CE010E94F51CD1FE47C0F801448155812A
:106A800066817781818182958F70873030F089307F
:106A9000E0F08A50823008F449C0CE010E94781498
:106AA000EC81FD81309781F180858F709EEF980F8A
:106AB000923010F0811128C0D80111969C91907FDE
:106AC00080858F70892B80871FC0EC81FD81309776
:106AD000D9F080858F709EEF980F923010F0811161
:106AE00013C04187528763877487EC81FD8180855D
:106AF000807F83608087EC81FD818085982F907FE7
:106B00008F7080679036F9F26EEA7AE08FE29FE04C
:106B10000E94B489C8010E9417348F2DDF91CF9154
:106B20001F910F91FF90DF90CF900895CE010E94AA
:106B30007814EACFCF92DF92EF92FF920F931F93D8
:106B4000CF93DF936115710509F460C06A017B0181
:106B50008C01CB010E946C14D82F882389F1D701B6
:106B600014968D919C91009709F43FC0FC01C0855B
:106B70002C2F2F703EEF320F323010F021112AC02F
:106B8000C595C595C595C595D0FE5EC0C7010E9447
:106B9000271DF8018083CC2351F1C295C07F8181EC
:106BA0008F70C82BC183D7011496ED91FC9181851C
:106BB0009285A385B485F80184839583A683B783E2
:106BC0008D2FDF91CF911F910F91FF90EF90DF906C
:106BD000CF900895253049F460E00E946C9C0097A6
:106BE00021F0DC011896CC91CBCFC0E0CDCFD701FE
:106BF0001496ED91FC9180858295807F8595859591
:106C000085958595823021F0833081F0D0E0D8CF12
:106C10004185528563857485F80181818F70806A12
:106C200081834483558366837783CACF41855285A8
:106C300063857485F80181818F70806781834483C7
:106C4000558366837783BCCFCC2389F2C295C07FFE
:106C5000F801A5CF0F931F93CF93DF9300D000D0FF
:106C60001F921F92CDB7DEB719821A821B821C8237
:106C70001D821E821F8218862A812F702A83FC01A2
:106C800002811381C8010E94271D8230D9F085300E
:106C9000C9F08823B9F040E052E0B801CE01019676
:106CA0000E949A3560E0CE0101960E94E212289679
:106CB0000FB6F894DEBF0FBECDBFDF91CF911F910D
:106CC0000F91089590E080E0F2CFCF93DF9300D052
:106CD00000D01F921F92CDB7DEB7FC01862F8F70B8
:106CE0006181607F682B618388E0DE0111960190ED
:106CF0000D928A95E1F729813A814B815C816D8102
:106D00007E818F81988528960FB6F894DEBF0FBEDE
:106D1000CDBFDF91CF910895CF93DF9300D000D006
:106D20001F921F92CDB7DEB7FC01608398E0DE01B1
:106D3000119601900D929A95E1F729813A814B8144
:106D40005C816D817E818F81988528960FB6F8943D
:106D5000DEBF0FBECDBFDF91CF910895AF92BF923E
:106D6000CF92DF92EF92FF920F931F93CF93DF9317
:106D7000CDB7DEB7CD56D1090FB6F894DEBF0FBE42
:106D8000CDBF5C01A7960FAFA797A8961FAFA89796
:106D9000A9962FAFA997AA963FAFAA97AB964FAFE8
:106DA000AB97AC965FAFAC97AD966FAFAD97AE9625
:106DB0007FAFAE9723961FAE1EAE2397FE01ED5B0D
:106DC000FF4F82E1DF011D928A95E9F772961192D9
:106DD000119287E0DF011D928A95E9F7CE018A5969
:106DE0009F4F0E941734F0FE2CC0A796EFADA797D7
:106DF000E83108F04DC1F0E08827EE5FF84C8F4F86
:106E00000C941BD94E381A3745384838483845381D
:106E10001A374838483848381A371A371A371A375D
:106E20001A37483848384838483848384838483891
:106E300048384E3864E17AE0CE018B5A9F4F0E9469
:106E400079CE0E94129C882309F407C180912E08F4
:106E5000811103C1C114D10409F05EC030E020E00B
:106E600043E050E060E4CE0101960E94122ED5016D
:106E7000ED91FC91608171814FE350E0CE0101966C
:106E80000E948CDDF1FE0DC1A7968FADA7978230D1
:106E900009F407C1853009F404C1A8968FADA897FD
:106EA00082958F709FE0980F9F70923018F0883015
:106EB00009F0F7C001E020E032E044E150E0BE011B
:106EC0006F5B7F4FCE018A599F4F0E946720BE01A2
:106ED0006F5B7F4FCE0101960E94D4AA6CEF79E0E0
:106EE0008FE29FE00E94B489BE016F5F7F4F8FE207
:106EF0009FE00E944E8969EF79E08FE29FE00E9457
:106F0000B489BE016F5B7F4F8FE29FE00E944E8984
:106F10008FE29FE00E941E88A8968FADA897807F81
:106F2000870100271071882311F0F1FC04C00115BE
:106F3000110509F4EAC030E020E043E050E060E4ED
:106F4000CE0101960E94122ED501ED91FC91608137
:106F500071814FE350E0CE0101960E948CDDC11497
:106F6000D10469F063EF74E0CE0101960E9466DD02
:106F70004FE350E0B601CE0101960E948CDD63EF35
:106F800074E0CE0101960E9466DD4FE350E06CEEA6
:106F900079E00115110511F468EE79E0CE01019652
:106FA0000E9489CEA8968FADA89782958F70845045
:106FB000823008F096C067E1CE018A599F4F0E9447
:106FC0008C366F962FAF6F97A0963FAFA097A19684
:106FD0004FAFA197A2965FAFA297A3966FAFA3976B
:106FE000A4967FAFA497A5968FAFA597A6969FAFBF
:106FF000A69700E020E033E044E150E0BE016F5B83
:107000007F4FCE018A599F4F0E94672062EE79E040
:107010008FE29FE00E94B489BE016F5F7F4F8FE2D5
:107020009FE00E944E896FED79E08FE29FE00E9421
:10703000B489BE016F5B7F4F8FE29FE00E944E8953
:107040008FE29FE00E941E880E94129C882329F0F4
:1070500080912E08882309F44CC0B701C5010E9415
:10706000B51C90E080E0C359DF4F0FB6F894DEBF47
:107070000FBECDBFDF91CF911F910F91FF90EF9089
:10708000DF90CF90BF90AF90089560E17AE0D4CECA
:1070900062E07AE08FE29FE00E94B489E894F0F821
:1070A000D0CEF0FE39CFBE016B5A7F4FCE01019694
:1070B0000E94D4AA63EF79E08FE29FE00E94B48936
:1070C000BE016F5F7F4F8FE29FE00E944E8960EFAD
:1070D00079E08FE29FE00E94B489BE016B5A7F4F36
:1070E00013CF20E032E0012B11F020E033E000E08C
:1070F00083CFBE016F5B7F4FCE0101960E94D4AA61
:1071000060E072E0C5010E94911CF0FE87C0A79666
:10711000EFADA797E150EE30E0F4F0E08827EC56B1
:10712000F74C8F4F0C941BD91A39A938A938A938B4
:10713000A9381A39A938A938A938A23811391F39FC
:107140001739143965ED79E0CE018B5A9F4F0E94B3
:1071500079CE30E020E043E050E060E4CE010196DB
:107160000E94122ED501ED91FC91608171814FE357
:1071700050E0CE0101960E948CDDC114D10469F06B
:1071800063EF74E0CE0101960E9466DD4FE350E0AC
:10719000B601CE0101960E948CDD63EF74E0CE0152
:1071A00001960E9466DD4FE350E06FEB79E0CE017F
:1071B00001960E9489CE69EB79E08FE29FE00E9400
:1071C000B489BE016F5F7F4F8FE29FE00E944E89BE
:1071D00066EB79E08FE29FE00E94B489BE016B5AB2
:1071E0007F4F8FE29FE00E944E898FE29FE00E94D6
:1071F0001E880E94129C882309F42FCF80912E08AC
:1072000081112BCFBE016B5A7F4FCE0101960E9498
:10721000D4AA60E071E0C5010E94911C81E090E079
:1072200022CF60ED79E090CF6CEC79E08DCF63EC0C
:1072300079E08ACFF5018085853009F08ACF6AED43
:1072400079E082CFDC011196EC911197E295EF7015
:10725000E150EB3008F037C0F0E08827ED5CF64CE9
:107260008F4F0C941BD94539453963393E393E3926
:1072700054394B394B394B393E393E3914966D915F
:107280007D918D919C911797089514966C9170E063
:1072900090E080E0089514966D917D918D919C9180
:1072A00017970E9418DA089514966D917D918D912B
:1072B0009C91179724E630E040E050E00E94B2D85D
:1072C000CA01B901089560E070E0CB0108954F92C2
:1072D0005F926F927F928F929F92AF92BF92CF9266
:1072E000DF92EF92FF920F931F93CF93DF93CDB76F
:1072F000DEB762970FB6F894DEBF0FBECDBF4C016C
:107300000B871C872D873E874F87588B698B7A8B1D
:1073100067EA74E1C7010E9470CEEDE0F0E0892BCE
:10732000F1F061EA74E1C7010E9470CEEFE0F0E095
:10733000892BA9F06BE974E1C7010E9470CEEEE0E1
:10734000F0E0892B61F01F7067E974E1C7010E94CA
:1073500070CEE12FF0E0892B11F4ECE0F0E09B859A
:10736000992309F480C1309731F4EF2809F478C0EB
:107370008FEF9FEF9CC03197EF30F10508F03EC0D2
:107380008827EA53F64C8F4F0C941BD9303AD539E5
:10739000FE39FE39FE39FE39993ADB3AFE39FE39BB
:1073A000FE39FE39E23A263BEE3ACE010B960E94B8
:1073B000223970934407609343079B0120513109A0
:1073C00029313105A8F620EF260F209341079B01B4
:1073D000770F440B550BD4011296ED91FC91139746
:1073E0000190F081E02D60817181ED91FC91068426
:1073F000F785E02D03ED14E0C401199510922F07D5
:1074000081E0809327078DE4809328078FE58093A0
:10741000290786EF99E00E940780F4018281938119
:107420000E94E81B2B013C014114510461047104CA
:1074300091F00E9406AA9B01AC01A12CB12C650120
:1074400014E6E12EF12C00E010E0C301B2010E942D
:107450001C2B882349F345E250E06EE177E022C01F
:1074600091509E3058F6E92FF0E08827E55CF54C06
:107470008F4F0C941BD9493A6E3AFE39FE396E3A59
:10748000493AFE39FE39FE39843A803A783A883AE8
:10749000863A80911C07816080933B074DE050E065
:1074A0006CE172E0C4010E94182681E090E06296CF
:1074B0000FB6F894DEBF0FBECDBFDF91CF911F9105
:1074C0000F91FF90EF90DF90CF90BF90AF909F9083
:1074D0008F907F906F905F904F90089580911C07E0
:1074E0008E7F80933B074DE050E06FE072E0DACF93
:1074F0001092350780911C07816080933B077ECFF7
:1075000081E080933507F6CF82E0FBCF84E0F9CFAE
:1075100083E08093350780911C07816080933B074F
:1075200080913707833009F069CF82E08093370775
:1075300065CF19829031A1F148F49C3089F0CE01D9
:107540000B960E9422396093370713C0913169F17D
:107550009231A9F782E08093370762E874E105C0B1
:1075600083E08093370762E974E1CE0101960E94BF
:1075700079CED4011296ED91FC9113970190F08190
:10758000E02D60817181ED91FC910288F389E02DFD
:1075900029EB34E0AE014F5F5F4FC40119952ECF48
:1075A000109237076DE874E1E0CF81E080933707F0
:1075B00066E874E1DACFCE010B960E94223960931F
:1075C00035071CCF913031F0923009F017CF10926F
:1075D0003A0714CF80E580933A0710CF913049F0F5
:1075E0009230F1F0CE010B960E9422396093390758
:1075F00005CF83E080933907D4011296ED91FC9179
:1076000013970190F081E02D60817181ED91FC91E3
:107610000288F389E02D22EB34E04AE655E0BDCF45
:1076200010923907D4011296ED91FC9113970190B5
:10763000F081E02D60817181ED91FC910288F389E8
:10764000E02D22EB34E045E755E0A7CF913039F04B
:10765000923009F0D3CE80913B07877F4ECF809147
:107660003B0788604ACF8827E75CF44C8F4F0C9427
:107670001BD9B839FE39D539FE39FE39FE39FE3904
:10768000993ADB3AFE39FE39FE39FE39FE39FE39C8
:10769000F23ACF93DF93EC016115710539F48F81D4
:1076A00081708F8381E0DF91CF9108958981982F38
:1076B00092959F7029F180E09430A8F79B01770F95
:1076C000440B550B2959310941095109A4E6B0E091
:1076D0000E94D1D82BE531E040E050E00E94B2D8C2
:1076E00037FF02C030E020E02536310514F024E6F3
:1076F00030E02F5F220F8F818170282B2F83D2CF14
:107700008F7080628983DACF2F923F924F925F927F
:107710006F927F928F929F92AF92BF92CF92DF92A1
:10772000EF92FF920F931F93CF93DF93CDB7DEB706
:1077300068970FB6F894DEBF0FBECDBF1C01098756
:107740001A872B873C874D875E876F87788B22E16E
:10775000E216F10408F035C0F701E55BFC4F30811B
:10776000398BCE0109960E944A1497FD04C0BC01D2
:10777000C1010E94493B9A85892F8F70D1011196D2
:10778000EC911197E07FE82B1196EC931197898586
:107790008C93E295EF70EC3008F063C0F0E088273E
:1077A000EB52F44C8F4F0C941BD9E23DFE3BFE3B59
:1077B000803DE33B0E3E493D8A3D8A3D8A3D493D41
:1077C000493D198ACECFB12C92959F709D3008F01B
:1077D000C9C4E92FF0E08827EF50F44C8F4F0C9488
:1077E0001BD9313C483E683E483E113E113E483E62
:1077F000483EB240B240483E483E153D92959F708B
:107800009D3008F022C1E92FF0E08827E55FF34CB6
:107810008F4F0C941BD9313CE93CDD3C9F3C1B3C19
:10782000183CC03CED3C253D253DAA3CAA3C153DFD
:107830008889F10187838F85D10116968C931697DD
:107840008E8515968C9315978D8514968C93149729
:107850009295907F11968C9111978F70982B11961D
:107860009C93B989BB2309F467C0F101818182959A
:107870008F702B2F30E08217130609F45DC06CE186
:107880007AE08FE29FE00E94B489D10111966C9159
:1078900062956F704AE050E08FE29FE00E9422887C
:1078A00069E17AE08FE29FE00E94B4894AE050E00B
:1078B00069898FE29FE00E94228867E17AE08FE287
:1078C0009FE00E94B489F101008119821A821B8213
:1078D0001C821D821E821F82188689898295807F64
:1078E0009A819F70892B8A830983EE24EA94FE2C67
:1078F0001181228133814481558166817781CE0156
:1079000001960E94843BD1012C9311963C931197D0
:1079100012964C93129713965C93139714966C934C
:10792000149715967C93159716968C931697179621
:107930009C93C1010E94173488E0F10182C18F85B8
:107940009889F1018683878190FB80F987838E85F2
:10795000858387CF8D859E85AF85B8898F3F9105BB
:10796000A105B10529F024F08FEF90E0A0E0B0E090
:10797000B7FF03C080E090E0DC01F101848371CFA8
:107980006D857E858F85988924E630E040E050E063
:107990000E94B2D82F3F31054105510529F024F04E
:1079A0002FEF30E040E050E057FF03C020E030E030
:1079B000A901D10114962C9354CF8F859889F10198
:1079C0008683878190FB80F987838E8585838D856B
:1079D000D5CF8D8514968C9344CFCD84DE84EF84EF
:1079E000F88820E030E0A901C701B6010E9446D71F
:1079F00087FD17C020E030E04FE753E4C701B60130
:107A00000E944EDA181634F4C12CD12CAFE7EA2EBE
:107A1000A3E4FA2EC701B6010E941FDAF1016483C4
:107A200020CFC12CD12C7601F5CFD10111968C91AC
:107A300011978F70806C11968C9311978D859E8510
:107A400015969C938E9314970CCF6CE97AE08FE295
:107A50009FE00E94B4896A8562956F704AE050E0A9
:107A60008FE29FE00E94228869E97AE08FE29FE03E
:107A70000E94B489F101618162956F704AE050E023
:107A80008FE29FE00E9422888FE29FE00E941E8882
:107A9000E8CE92959F70933091F09C3031F24D85F5
:107AA0005E856F857889F10144835583668377838A
:107AB0009295907F81818F70982B9183D2CE60E0D8
:107AC000C1010E94E212D10114968C9314978F8504
:107AD000988916968C93169717968C91179790FB0A
:107AE00080F917968C9317978E8515968C9315971A
:107AF00011968C9111978F70806211968C93B1CEF4
:107B000060E0CE0109960E94E212D10114968C9396
:107B10001497EECF92959F709D3008F066C0E92FC4
:107B2000F0E08827E956F24C8F4F0C941BD9313C7A
:107B3000B23DE13D5F3DE13DE13DA43DD13DD13D63
:107B4000D13DC03DCC3D153D8D859E85AF85B88925
:107B5000F10184839583A683B78381818F708066CA
:107B600081837FCE6D8570E090E080E00E944BD7EE
:107B7000D10114966D937D938D939C93179771CE3D
:107B80006D857E858F8598890E944DD7F10164832C
:107B900075838683978365CE6D857E858F8598896D
:107BA000E5CF9295907FF10181818F70982B918321
:107BB0008D859E85AF85B88984839583A683B78399
:107BC00050CE9295907FD10111968C9111978F7024
:107BD000982B11969C938D859E85AF85B889F10170
:107BE00084839583A683B7833CCE67E87AE08FE2EF
:107BF0009FE00E94B4896A8562956F704AE050E008
:107C00008FE29FE00E94228864E87AE08FE29FE0A2
:107C10000E94B489D10111966C912ECFBB24B394EC
:107C2000D3CD4D855E856F857889F1014483558379
:107C3000668377839295907F81818F70982B918353
:107C400088E0DE01119601900D928A95E1F7298175
:107C50003A814B815C816D817E818F8198856896A8
:107C60000FB6F894DEBF0FBECDBFDF91CF911F914D
:107C70000F91FF90EF90DF90CF90BF90AF909F90CB
:107C80008F907F906F905F904F903F902F900895CE
:107C9000963009F43AC148F46D85913071F06FEF78
:107CA00070E0933051F060E008C0973009F439C1BA
:107CB0009A506D857E859230B0F784E68F878889EB
:107CC0008E7F888B1E868A858F7080628A876D87FB
:107CD0002E8530E0AFEFB0E00E94E4D824E630E03B
:107CE00040E050E00E94B2D869017A01FFEFCF1660
:107CF000D104E104F10429F024F0C12CD12C760147
:107D0000CA9486012D852A8B622E712CBB2009F422
:107D100071C088898695A82FA150BB0B2D01BFEF9C
:107D20004B165B0609F01EC1003811050CF000C1AE
:107D30008FE790E08C199D09869DD001879DB00D3D
:107D4000969DB00D11242FEF30E00E9432D921E82A
:107D50003EE740E050E00E94B2D8F1012783ABE952
:107D6000B0E0A70196010E94D1D8EFE78E2E912CAA
:107D7000A12CB12CA50194010E94B2D889019A01CD
:107D80000C591F4F2F4F3F4FAEEFB1E0A7019601A7
:107D90000E94D1D8A50194010E94B2D8D3010E94BB
:107DA000D1D82FEF30E040E050E00E94B2D8390146
:107DB0002FEF6216710421F01CF066246A94712C76
:107DC00067E77AE08FE29FE00E94B489B8018FE212
:107DD0009FE00E94799C69E67AE08FE29FE00E9432
:107DE000B489B3018FE29FE00E94799C8FE29FE00B
:107DF0000E941E88EAE2FCE1E491F0E0EE0FFF1F32
:107E0000E05FF34E85919491E0E8FCE1E4912F85E9
:107E100038893170AFEFBFEF0E94E4D82DE631E032
:107E200040E050E00E94B2D844275527AAEFB5E0C1
:107E30000E94D1D8DC01CB019058AF4FBF4FCD018C
:107E4000BB2797FDB095AB2F8E3FE1E09E0708F072
:107E500062C1382F8F3F910508F47FC14EEF481B58
:107E600050E03FEFF301319678012FEFE21AF20A6A
:107E7000009510E03E9DC0013F9D900D1124292FDB
:107E80003327200F311FDF010E9432D94B015C01E3
:107E90008824AA24BB245E9D90015F9D300D11248F
:107EA000232F3327200F311F0E9432D9BB27A92F40
:107EB000982F872F882A992AAA2A4E9D90014F9D94
:107EC000300D1124232F3327200F311FDF010E9493
:107ED00032D9B82FA72F962F882788279927BB2715
:107EE00088299929AA29F101A683958384836DE3C2
:107EF0007AE08FE29FE00E94B489C1010E941734AA
:107F000060E080E00E947CA8ACCC6D857E858F858A
:107F1000988924E630E040E050E00E94B2D8B901F0
:107F2000CCCE6D857E858F8598890E9418DAC5CE66
:107F3000A70196012058310941095109ABE9B0E088
:107F40000E94D1D82FE730E040E050E00E94B2D844
:107F500089019A010C591F4F2F4F3F4FD10117969E
:107F60001C922ECF9201AAEBBFEF0E942AD944E6C1
:107F7000842E912CA12CB12CA50194010E94B2D881
:107F8000DA01C9018C599F4FAF4FBF4F8B8B9C8B30
:107F9000AD8BBE8B26E430E0D2010E9432D9A50120
:107FA00094010E94B2D849015A019EE1890E911CA8
:107FB000A11CB11C003811050CF093C08FE790E0B4
:107FC0008C199D09869DD001879DB00D969DB00DA1
:107FD0001124A50194010E94DCD89B01AC01AFEFF4
:107FE000B0E00E94D1D824E63AE640E050E00E949A
:107FF000B2D8D10117962C932B893C894D895E8983
:108000002C0D3D1D4E1D5F1DAEEFB1E00E94D1D87D
:1080100023EE30E040E050E00E94B2D829013A015E
:10802000388F2F8BAFEFB0E0A70196010E94D1D817
:108030002FE730E040E050E00E94B2D88901EA89A1
:10804000AE2FB0E0A30192010E94D1D82FEF30E013
:1080500040E050E00E94B2D839012F3F310521F0B5
:108060001CF066246A94712C63E67AE08FE29FE04C
:108070000E94B4892AE030E04B895C896D897E8951
:108080008FE29FE00E94C4886DE57AE08FE29FE076
:108090000E94B4892AE030E0B501A4018FE29FE09C
:1080A0000E94C48865E57AE08FE29FE00E94B4896F
:1080B000B8018FE29FE00E94799C6DE47AE08FE244
:1080C0009FE00E94B489B3018FE29FE00E94799CF7
:1080D00064E47AE08FE29FE00E94B4896F89788D32
:1080E00081CEA70196012058310941095109ABE918
:1080F000B0E00E94D1D82FE730E040E050E00E948D
:10810000B2D889019A010C591F4F2F4F3F4FD1010F
:1081100017961C92A9CF8C3FF3E09F0768F48D3F20
:1081200022E0920728F452E0580F3FEF40E09ACE49
:108130003CEF381B5FEFFACF8A3F35E0930781F0C1
:108140008B3FE4E09E0728F444E0480F5FEF30E007
:1081500089CE5AEF581B30E001C050E04FEF82CE7D
:1081600050E0F9CF6BE27AE08FE29FE00E94B489A1
:108170006A8562956F704AE050E08FE29FE00E944E
:10818000228868E27AE042CDAF92BF92CF92DF922E
:10819000EF92FF920F931F93CF93DF93CDB7DEB78C
:1081A00068970FB6F894DEBF0FBECDBFFC01098BF8
:1081B0001A8B2B8B3C8B4D8B5E8B6F8B788F8281D8
:1081C0009381009709F49FC024813581232B09F402
:1081D0009AC0CC2009F497C06F0170E060E00E9463
:1081E000041C192FD601ED91FC91028CF38DE02D2A
:1081F000C60119955C018230910509F478C0039796
:1082000009F447C095E0F1E0AF16B10409F091E040
:1082100019861A861B861C861D861E861F86188A4E
:108220009295907F8A858F70892B8A87EE24EA94B5
:10823000FE2C09891A892B893C894D895E896F89B1
:10824000788DCE0109960E94843BF1E0AF16B1040F
:1082500009F44FC082E0A816B10409F045C06F854B
:1082600070E0D60114968C910E94B8A861E070E08D
:10827000C6010E942F1C6E8570E00E94B8A862E0C3
:1082800070E0C6010E942F1C6D8570E00E94B8A8A6
:108290002BC0612F661F6627661FCE0141960E9484
:1082A000E2125C01BC01D60114968C910E94B8A820
:1082B00060EC76E18FE29FE00E94B489F601648170
:1082C00075818FE29FE00E94799C6EEB76E18FE2F0
:1082D0009FE00E94B489B5018FE29FE00E94799CE3
:1082E0008FE29FE00E941E8881E090E00EC094E043
:1082F0008FCF63E070E0C6010E942F1C688970E098
:108300000E94B8A8ACCF90E080E068960FB6F894D1
:10831000DEBF0FBECDBFDF91CF911F910F91FF90B8
:10832000EF90DF90CF90BF90AF900895FC019181C6
:10833000892F82958F7021F0823029F080E0089596
:108340009F70906291839B0177FF02C030E020E034
:108350002E3681E0380714F02DE631E02683878140
:1083600030FB80F9878381E00895AF92BF92CF926E
:10837000DF92EF92FF920F931F93CF93DF9300D082
:1083800000D01F921F92CDB7DEB75C017B0160FF6A
:1083900003C0E894E0F8F3F8F3FC0DC00E94EB1181
:1083A000663971058105910530F08091A2089091A0
:1083B000A3080597F9F4B70166277370C5010E94F9
:1083C000B51C65EA79E08FE29FE00E94B4898FEFE7
:1083D0009FEF28960FB6F894DEBF0FBECDBFDF919A
:1083E000CF911F910F91FF90EF90DF90CF90BF90B2
:1083F000AF90089519821A821B821C821D821E82F0
:108400001F8218868A818F708A8340E053E0B5010D
:10841000CE0101960E949A3560E073E0C5010E948A
:10842000DB1CE82AF92AD12CC12C09811A812B8165
:108430003C814D815E816F817885C5010E94AE3699
:10844000C8CF4F925F926F927F92AF92BF92CF92BE
:10845000EF92FF920F931F93CF93DF9300D000D042
:108460001F921F92CDB7DEB75C0109831A832B835D
:108470003C834D835E836F8378876AE077E08FE289
:108480009FE00E94B489CE0101960E941734898131
:10849000811134C00A810F700130A9F160F10230FE
:1084A00021F010E0053009F041C0D501ED91FC91BB
:1084B000068CF78DE02D09811A812B813C814D813D
:1084C0005E816F817885C501199581E090E02896DD
:1084D0000FB6F894DEBF0FBECDBFDF91CF911F91D5
:1084E0000F91FF90EF90CF90BF90AF907F906F90E3
:1084F0005F904F900895CC24C394D7CF813061F121
:10850000823009F4BCC06DEF76E08FE29FE00E94FC
:10851000B4894AE050E069818FE29FE00E9422889E
:108520008FE29FE00E941E8801E010E06DEE76E091
:108530008FE29FE00E94B489B8018FE29FE00E9421
:10854000799C8FE29FE00E941E88CE0101960E94D6
:10855000173490E080E0BBCF8A8182958F7086309F
:1085600009F474C0D8F481508230E0F16EE170E01B
:10857000CE0101960E94AF13F5016281738140E044
:1085800052E0CE0101960E941E3560E07AE0D501EE
:1085900012968D919C910E94B5411BC0873079F154
:1085A0008A50823018F78D819E81AF81B8858536DB
:1085B0009105A105B10524F084E690E0A0E0B0E0CB
:1085C000B7FF03C080E090E0DC019C01243131055D
:1085D0006CF2D501ED91FC91068CF78DE02DCC2449
:1085E000C39469CF2D8130E0A4E6B0E00E94E4D8C6
:1085F0002FEF30E040E050E00E94B2D8E7CF4D804E
:108600005E806F80788420E030E0A901C301B20170
:108610000E9446D787FD11C020E030E048EC52E4CC
:10862000C301B2010E944EDA181654F4412C512CA9
:1086300088EC682E82E4782E03C0412C512C320144
:10864000C301B2010E9418DA9B01C0CF6D817E8107
:108650008F81988524E630E040E050E00E94B2D857
:10866000253631054105510524F024E630E040E08F
:1086700050E057FFABCF20E030E0A901A7CF1D822B
:108680001E821F821886D501ED91FC91068CF78D14
:10869000E02DCC24C39402E01A812B813C8140E080
:1086A0000FCF0F931F93CF93DF938C01FC01C081F9
:1086B000D1816FE270E0CE010E94B9DD0097D9F060
:1086C000FC011192CF010E941E1AEC0167E977E0CC
:1086D0008FE29FE00E94B489BE018FE29FE00E947A
:1086E000799C8FE29FE00E941E88CE01DF91CF919E
:1086F0001F910F910895CE010E941E1AEC01892B43
:10870000A1F3F80111821082F0CF2F923F924F9285
:108710005F926F927F928F929F92AF92BF92CF9211
:10872000DF92EF92FF920F931F93CF93DF93CDB71A
:10873000DEB7C15CD1090FB6F894DEBF0FBECDBF66
:108740004C01C755DF4F0883C95AD040C655DF4F8B
:108750001883CA5AD040C555DF4F2883CB5AD04022
:10876000C455DF4F3883CC5AD040C355DF4F4883C0
:10877000CD5AD040C255DF4F5883CE5AD040C15554
:10878000DF4F6883CF5AD040C055DF4F7883C05B3E
:10879000D040CF54DF4FF982E882C15BD040CF5345
:1087A000DF4FC882C15CD0400E9406AAC354DF4F8D
:1087B000688379838A839B83CD5BD040C655DF4F26
:1087C0008881CA5AD0408F70282E312CC090A208C0
:1087D000D090A308C554DF4FD982C882CB5BD0406C
:1087E000CF54DF4FE881F981C15BD040309721F051
:1087F000808181110C94E94FD4011B968C918823C0
:1088000041F0C4010B96CF54DF4F99838883C15B3D
:10881000D0402114310411F00C943250CF54DF4F6A
:10882000E881F981C15BD040309711F00C94ED4F95
:10883000F401238C348C2114310411F40C94325043
:10884000C655DF4F8881CA5AD0408F7011F00C9402
:108850003250622DCE0187559F4F0E946536C75614
:10886000DF4F2883C959D040C656DF4F3883CA59D5
:10887000D040C556DF4F4883CB59D040C456DF4F58
:108880005883CC59D040C356DF4F6883CD59D04070
:10889000C256DF4F7883CE59D040C156DF4F888310
:1088A000CF59D040C056DF4F9883C05AD0400C9467
:1088B0003250D4018D919C91009709F406C2B4E026
:1088C0002B16310409F0A8C00E94819C082F10E0EB
:1088D000063011058CF40E94BD91009721F0FC0137
:1088E0002085207F2087BC01D4018D919C910E941E
:1088F00090A00F5F1F4FECCF65E0F4018081918164
:108900000E946C9C8C01892BE9F410E000E0C80106
:10891000CF53DF4F0FB6F894DEBF0FBECDBFDF9150
:10892000CF911F910F91FF90EF90DF90CF90BF906C
:10893000AF909F908F907F906F905F904F903F90FF
:108940002F900895C755DF4F8881C95AD040803194
:10895000E0F6CE0187559F4F0E9422391616170662
:10896000180619062CF4D80118968C918D7089F090
:10897000F80180858F70808762E079E08FE29FE068
:108980000E94B4898FE29FE00E941E8801E010E0FF
:10899000BECF0E9406AA6B017C01CE0187559F4F76
:1089A0000E942239C60ED71EE81EF91ED80119965C
:1089B000CD92DD92ED92FC921C97C755DF4F8881D6
:1089C000C95AD0408295807F826018968C9367EF59
:1089D00078E08FE29FE00E94B489CE0187559F4FD7
:1089E0000E942239AB01BC012AE030E08FE29FE017
:1089F0000E94C48861EF78E08FE29FE00E94B48912
:108A0000F80141855285638574852AE030E08FE264
:108A10009FE00E94C488B6CFC755DF4F1881C95A5E
:108A2000D040143009F4C4C228F4112391F1B12CC0
:108A3000A12C77C288EF810F8230C8F788E0FE0151
:108A4000E755FF4FDE01119601900D928A95E1F7EF
:108A5000C655DF4FE881CA5AD0408E2F807F09F477
:108A600023C3E295EF70E150EB3008F01DC3F0E056
:108A70008827E25CFA4B8F4F0C941BD9424842483E
:108A8000544833483348A948984898489848334848
:108A9000334819821A821B821C821D821E821F8209
:108AA00018868A818F708A83C655DF4F8881CA5A9B
:108AB000D040807F09F4BBCFF9E02F16310409F4D0
:108AC00032C20CF005C12114310409F425C182E041
:108AD0002816310409F0ABCFB12CA12CCD54DF4FB7
:108AE0001882C35BD040DD24DA94B401CE01019634
:108AF0000E94EBA08A81982F92959F70945F9F703F
:108B0000923060F4C655DF4F9881CA5AD040929592
:108B10009F70923019F48F7080628A83D401189606
:108B20009C91973071F4C655DF4F8881CA5AD04066
:108B3000807E803211F0803421F48A818F708062CF
:108B40008A83F401A185B285892F90E0109741F0C6
:108B5000ED91FC911197028CF38DE02DCD011995CB
:108B60007C01C755DF4F0881C95AD040C655DF4F39
:108B70001881CA5AD040C555DF4F2881CB5AD04002
:108B8000C455DF4F3881CC5AD040C355DF4F4881A0
:108B9000CD5AD040C255DF4F5881CE5AD040C15532
:108BA000DF4F6881CF5AD040C055DF4F7881C05B1E
:108BB000D040CE0101960E94843BCF57DF4F2883DF
:108BC000C158D040CE57DF4F3883C258D040CD5720
:108BD000DF4F4883C358D040CC57DF4F5883C45829
:108BE000D040CB57DF4F6883C558D040CA57DF4FBE
:108BF0007883C658D040C957DF4F8883C758D040C4
:108C0000C857DF4F9883C858D040CE0101960E94C4
:108C10001734CD54DF4FC880C35BD040CC2069F1FE
:108C2000C655DF4F8881CA5AD04082958F709FE029
:108C3000980F9F70923020F08A5F8F708230E8F436
:108C40008A8182958F7081508230B8F42D8130E016
:108C5000AFEFB0E00E94E4D824E630E040E050E01E
:108C60000E94B2D82F3F31054105510529F024F06B
:108C70002FEF30E040E050E02D8388E0FE01319698
:108C8000DE01A755BF4F01900D928A95E1F72AE0CA
:108C9000B22AC12CD40118968C911897873009F00C
:108CA0008EC5C954DF4FE881F981C75BD040EE35EE
:108CB000F1400CF068C46BEC78E088E09EE00E9424
:108CC000B48988E09EE00E941E880FEF1FEF1FCE40
:108CD0009AE02916310409F4D0C0ABE02A16310419
:108CE00009F0A5CEB401CE0101960E94EBA0CE0101
:108CF00087559F4F0E944A14BC01CE0101960E94E5
:108D0000493B88E0FE013196DE01A755BF4F019037
:108D10000D928A95E1F702C1C4010E94E1538C01D2
:108D200061E070E01816190614F070E060E08FE260
:108D30009FE00E94799C69E474E08FE29FE00E94CA
:108D40004E89CE0187559F4F0E942239AB01BC014D
:108D50002AE030E08FE29FE00E94C4888FE29FE02B
:108D60000E941E88CE0187559F4F1016110614F0E1
:108D70000C94D74F0E942239672B682B692B09F07E
:108D800073C062E0CE0187559F4F0E948C36CF564C
:108D9000DF4F2883C159D040CE56DF4F3883C259A8
:108DA000D040CD56DF4F4883C359D040CC56DF4F1B
:108DB0005883C459D040CB56DF4F6883C559D04043
:108DC000CA56DF4F7883C659D040C956DF4F8883D3
:108DD000C759D040C856DF4F9883C859D040AA24FD
:108DE000A394BA2CB1E0CD54DF4FB883C35BD0401D
:108DF000DD24D3947ACE61E0CE0187559F4F0E9447
:108E00008C36C757DF4F2883C958D040C657DF4F2D
:108E10003883CA58D040C557DF4F4883CB58D0401D
:108E2000C457DF4F5883CC58D040C357DF4F6883B7
:108E3000CD58D040C257DF4F7883CE58D040C1576D
:108E4000DF4F8883CF58D040C057DF4F9883C05939
:108E5000D040AA24A394BA2CE1E0CD54DF4FE8839C
:108E6000C35BD040D12C41CEB12CA12CF1E0CD542C
:108E7000DF4FF883C35BD040BBCFB401CE01019676
:108E80000E94EBA0C255DF4F8881CE5AD0409A8114
:108E900092959F7061F0923071F0B12CA12CCC248E
:108EA000C394CD54DF4F1882C35BD0401CC29A815B
:108EB0009F7090629A8390E08536910514F084E665
:108EC00090E08E8388E0FE013196DE01A755BF4F0A
:108ED00001900D928A95E1F762E0CE0187559F4F90
:108EE0000E946536EA962FAFEA97EB963FAFEB9775
:108EF000EC964FAFEC97ED965FAFED97EE966FAFB8
:108F0000EE97EF967FAFEF97C158DF4F8883CF572B
:108F1000D040C058DF4F9883C058D040A12CBAE051
:108F2000BB2EC12CBECFB401CE0101960E94EBA096
:108F3000C155DF4F6881CF5AD040C055DF4F78818F
:108F4000C05BD0407170CE0101960E949641CD5415
:108F5000DF4F8883C35BD040882309F4A9C288E02F
:108F6000FE013196DE01A755BF4F01900D928A9503
:108F7000E1F762E0CE0187559F4F0E946536E29689
:108F80002FAFE297E3963FAFE397E4964FAFE497B6
:108F9000E5965FAFE597E6966FAFE697E7967FAF0A
:108FA000E797E8968FAFE897E9969FAFE997B6CF36
:108FB000C4010E94E153181619065CF562E0CE0167
:108FC00087559F4F0E948C36AA962FAFAA97AB96D3
:108FD0003FAFAB97AC964FAFAC97AD965FAFAD9749
:108FE000AE966FAFAE97AF967FAFAF97E0968FAF6D
:108FF000E097E1969FAFE197AA24A394BA2CC12CE5
:1090000081E0CD54DF4F8883C35BD040DD24D3940F
:1090100041CE61E0CE0187559F4F0E948C36A296CB
:109020002FAFA297A3963FAFA397A4964FAFA49755
:10903000A5965FAFA597A6966FAFA697A7967FAFA9
:10904000A797A8968FAFA897A9969FAFA997AA248C
:10905000A394BA2CC12C91E0CD54DF4F9883C35B0D
:10906000D040D12C17CEC355DF4F288139814A819A
:109070005B81CD5AD040A4E6B0E00E94D1D82B014C
:109080003C010DC0C355DF4F4880CD5AD040A4E607
:109090004A9E20011124052C000C66087708411413
:1090A00051046104710429F4E5E04E2E512C612C29
:1090B000712C193041F47094609450944094411C88
:1090C000511C611C711CB401CE0187559F4F0E9439
:1090D000EBA060E0CE0187559F4F0E948C366A96C8
:1090E0002FAF6A976B963FAF6B976C964FAF6C97AD
:1090F0006D965FAF6D976E966FAF6E976F967FAF01
:109100006F97A0968FAFA097A1969FAFA197B2E05F
:109110002B16310409F477C02CF52114310409F021
:1091200086CC81E0CD54DF4F8883C35BD04070C0D4
:1091300020E030E048EC52E4C355DF4F688179818C
:109140008A819B81CD5AD0400E94ACD70E9418DA08
:1091500096CFC355DF4F488059806A807B80CD5AB7
:10916000D0409DCFF9E02F16310409F4A6C12AE0C2
:109170002216310409F05BCCC655DF4F8881CA5AEC
:10918000D04082958F70823009F0F2C1C301B201E4
:1091900024E630E040E050E00E94B2D8C255DF4FF4
:1091A0008881CE5AD04090E0280F391F37FF02C087
:1091B00030E020E02536310514F024E630E0C255D9
:1091C000DF4F2883CE5AD04062E0CE0187559F4FB3
:1091D0000E9465362A962FAF2A972B963FAF2B9782
:1091E0002C964FAF2C972D965FAF2D972E966FAF85
:1091F0002E972F967FAF2F9760968FAF60976196CF
:109200009FAF61978BCECD54DF4F1882C35BD040A8
:10921000D40119968D919C911A97009789F518960B
:109220008C9190E060E5A62EB12CC12CD12C85301C
:10923000910549F0A12CB12C6501449721F0A12C96
:10924000B12C6501AA94C655DF4FE881CA5AD040B7
:10925000E295EF70E150EB3008F020C1F0E0882794
:10926000EB5CF64B8F4F0C941BD9484948494E4A4A
:109270004E4A4E4A1B4AE549E549E5497649764951
:10928000DC01ED91FC91028CF38DE02D1995CACF94
:10929000C355DF4F1881CD5AD040C301B20124E637
:1092A00030E040E050E00E94B2D8DA01C901810FFD
:1092B000911DA11DB11DB7FF03C080E090E0DC014E
:1092C0008F3F9105A105B10529F024F08FEF90E0C3
:1092D000A0E0B0E0C355DF4F8883CD5AD040A12C29
:1092E0005AE0B52EC12CDD24DA94D4CCC355DF4F1F
:1092F000E880F9800A811B81CD5AD040B4E64B1634
:10930000510461047104DCF5A4E6B0E0A801970102
:109310000E94D1D8460E571E681E791EA114B104B2
:10932000C104D104B9F0A60195010E94D1D8362F0D
:10933000272FB301A20177FF03C040E050E0BA013C
:10934000432E522E3C01441555056605770514F44D
:109350002A013B01C355DF4F488259826A827B82D2
:10936000CD5AD040C655DF4F8881CA5AD0408F7041
:109370008066C655DF4F8883CA5AD040B0CFC3013C
:10938000B20124E630E040E050E00E94B2D8E20EA4
:10939000F31E041F151FA114B104C104D10461F010
:1093A00017FF03C0E12CF12C8701AE14BF04C006E7
:1093B000D10614F486017501C355DF4FE882F982A6
:1093C0000A831B83CD5AD0408ACFC355DF4F6881B3
:1093D00079818A819B81CD5AD0400E9418DA7B0125
:1093E0008C01C301B20124E630E040E050E00E946D
:1093F000B2D8CA01B9016E0D7F1D801F911FA11443
:10940000B104C104D10461F097FF03C060E070E0D3
:10941000CB01A616B706C806D90614F4C601B501D5
:109420000E944DD7C355DF4F688379838A839B831E
:10943000CD5AD04054CFC355DF4F88819981AA813E
:10944000BB81CD5AD040480E591E6A1E7B1EA11406
:10945000B104C104D104C9F0A4E6B0E0A6019501AD
:109460000E94D1D8362F272FB301A20177FF03C066
:1094700040E050E0BA01432E522E3C014415550500
:109480006605770514F42A013B01C355DF4F488276
:1094900059826A827B82CD5AD04021CF88E0FE017A
:1094A0003196DE01A755BF4F01900D928A95E1F7E5
:1094B000B12CA12CCC24C39416CFC655DF4F888184
:1094C000CA5AD04082958F70823009F051C0C301D2
:1094D000B20124E630E040E050E00E94B2D8C1552D
:1094E000DF4F8881CF5AD040C055DF4F6881C05BC5
:1094F000D040962F9170280F391F2E36E1E03E079D
:109500002CF437FF05C02DE631E002C030E020E04A
:10951000C155DF4F2883CF5AD040C055DF4F8881D7
:10952000C05BD04030FB80F9C055DF4F8883C05B03
:10953000D04062E0CE0187559F4F0E94653662960B
:109540002FAF629763963FAF639764964FAF649770
:1095500065965FAF659766966FAF669767967FAFC4
:10956000679768968FAF689769969FAF6997D6CCD3
:1095700088E0FE013196DE01A755BF4F01900D92A4
:109580008A95E1F78ACCCF53DF4FD880C15CD040B9
:10959000DD20D9F01296ED91FC9190859F70953069
:1095A000A1F4C554DF4F88819981CB5BD0400597EA
:1095B00061F0CF54DF4F48815981C15BD040BE017B
:1095C00067557F4FCF010E942153C755DF4F8881D8
:1095D000C95AD040853009F4CAC020F4833079F1EB
:1095E000C5016CC0863009F47CC08730C9F7C4015E
:1095F0000E94271D182F863009F062C06BEA78E0C0
:109600008FE29FE00E94B48966E070E08FE29FE005
:109610000E94799C8FE29FE00E941E8862E0CE014A
:1096200087559F4F0E948C3629AF3AAF4BAF5CAF46
:109630006DAF7EAF8FAF21969FAF21973CC0C40125
:109640000E94271D853019F003E010E060C96CEB23
:1096500078E08FE29FE00E94B48965E070E08FE2DD
:109660009FE00E94799C8FE29FE00E941E88B401D7
:10967000CE0187559F4F0E94EBA061E0CE01875538
:109680009F4F0E948C3622962FAF229723963FAF92
:10969000239724964FAF249725965FAF259726965C
:1096A0006FAF269727967FAF279728968FAF28977B
:1096B00029969FAF2997C50181609160D12C30C058
:1096C00063E978E08FE29FE00E94B489612F70E047
:1096D0008FE29FE00E94799C8FE29FE00E941E88AB
:1096E000B3CFC4010E94E15318161906CCF1B4019E
:1096F000CE0187559F4F0E94EBA061E0CE018755B8
:109700009F4F0E948C3629AB3AAB4BAB5CAB6DAB39
:109710007EAB8FAB98AFC5018160916046E0D42EDF
:109720005C016894A0F8C655DF4F2881CA5AD04022
:10973000322F3F70323058F4C755DF4F3881C95A45
:10974000D040332321F05C016894A0F8B0F8207F6A
:1097500059F16894B1F801E010E0C110E7C497C274
:109760006FE778E08FE29FE00E94B4896DCFC4017B
:109770000E94E15318161906A4F462E0CE01875541
:109780009F4F0E948C3629A73AA74BA75CA76DA7CD
:109790007EA78FA798ABC5018160916035E0D32E7D
:1097A000BFCF68E678E0DECF40E052E0B401CE0102
:1097B00087559F4F0E949A358111CBCFCCCF9FEF19
:1097C000D912BBC0C4010E94E153DD24D394181602
:1097D00019060CF4B5C0D12C60E678E08FE29FE06A
:1097E0000E94B489ED2C0D2C000CFF08C954DF4FEA
:1097F000F982E882C75BD040B7018FE29FE00E9408
:10980000799C69E578E08FE29FE00E94B489CD54AD
:10981000DF4FF880C35BD0406F2D70E08FE29FE098
:109820000E94799C8FE29FE00E941E88CF54DF4FF8
:10983000E880F980C15BD040E114F10409F48DC0E7
:1098400064E17AE0C7010E9470CE01E010E0892B4C
:1098500009F44BC060E17AE0C7010E9470CE02E0DB
:1098600010E0892B09F441C067EA77E0C7010E9444
:1098700070CE05E010E0892BC1F163EA77E0C70103
:109880000E9470CE06E010E0892B79F165ED79E059
:10989000C7010E9470CE0AE010E0892B31F160ED23
:1098A00079E0C7010E9470CE0BE010E0892BE9F04F
:1098B0006AED79E0C7010E9470CE0CE010E0892BC0
:1098C000A1F063EC79E0C7010E9470CE0DE010E0DA
:1098D000892B59F06CEC79E0C7010E9470CE10E042
:1098E00000E0892B11F40EE010E0C4010E94271D56
:1098F000682E712C6114710431F4C954DF4F6880F3
:109900007980C75BD0400115110509F445C0601688
:109910007106E9F063E478E08FE29FE00E94B48989
:10992000B3018FE29FE00E94799C8FE29FE00E944A
:109930001E880DEF1FEF0C948744DD2009F44CCFF7
:10994000A1E0CD54DF4FA883C35BD04045CFCF54B7
:10995000DF4F19821882C15BD040C755DF4F988115
:10996000C95AD0409F3008F076C1E92FF0E088272F
:10997000E354F34B8F4F0C941BD93F4EED4DD14D1B
:109980000B4D3F4EB04D894D554D3F4E3F4E084E0D
:10999000084E084E084E084ED40119968D919C91A0
:1099A000009711F40C948544DC01ED91FC9104883E
:1099B000F589E02DCD54DF4FC880C35BD040C7553B
:1099C000DF4F0881C95AD040C655DF4F1881CA5AA7
:1099D000D040C555DF4F2881CB5AD040C455DF4F0A
:1099E0003881CC5AD040C355DF4F4881CD5AD04042
:1099F000C255DF4F5881CE5AD040C155DF4F6881E4
:109A0000CF5AD040C055DF4F7881C05BD040199508
:109A10008C010C948744C4010E94271D853009F0F5
:109A200013CE64E378E08FE29FE00E94B48965E0A2
:109A300070E08FE29FE00E94799C8FE29FE00E949D
:109A40001E88B401CE0187559F4F0E94EBA0F40100
:109A500080858530D9F46CE0CE0187559F4F0E94F8
:109A60008C3629A33AA34BA35CA36DA37EA38FA33B
:109A700098A76894A0F8B0F8D12C0FEF1FEFF1E091
:109A8000CD54DF4FF883C35BD04067CE61E0CE0199
:109A900087559F4F0E948C36298F3A8F4B8F5C8F52
:109AA0006D8F7E8F8F8F98A3E4CFC4010E94271DF6
:109AB000182F863059F563E278E08FE29FE00E942C
:109AC000B48966E070E08FE29FE00E94799C8FE2AB
:109AD0009FE00E941E8862E0CE0187559F4F0E9442
:109AE0008C36298B3A8B4B8B5C8B6D8B7E8B8F8B63
:109AF000988F6894A0F8B0F8D12C0FEF1FEF21E0F9
:109B0000CD54DF4F2883C35BD04027CE6BE078E095
:109B1000D9CDD11022C0B401CE0187559F4F0E94EC
:109B2000EBA061E0CE0187559F4F0E948C362987BC
:109B30003A874B875C876D877E878F87988B689481
:109B4000A0F8B0F826E0D22E0FEF1FEF81E0CD5441
:109B5000DF4F8883C35BD04000CE67EF77E002CE53
:109B6000DD20E1F062E0CE0187559F4F0E948C36E8
:109B700029833A834B835C836D837E838F839887AD
:109B80006894A0F8B0F895E0D92E0FEF1FEF91E0A0
:109B9000CD54DF4F9883C35BD040DFCD60EE77E0DC
:109BA000E1CDC655DF4F8881CA5AD0408F708230D0
:109BB00008F05FC0C4010E94271D853009F444CD20
:109BC0006894A0F8B0F8D12C0FEF1FEFA1E0CD54AE
:109BD000DF4FA883C35BD040C0CDC655DF4F88811F
:109BE000CA5AD0408F70823008F0E6C0DD2081F084
:109BF0006DEC77E08FE29FE00E94B48961E0C401E0
:109C00000E94F51C60E079E0C4010E94B5411CCDC2
:109C1000C655DF4F8881CA5AD040282F2F70223076
:109C200008F0D1C0992309F4D5C0807F31F4B40184
:109C3000CE0187559F4F0E94EBA06894A0F8B3E037
:109C4000BB2AD12C0FEF1FEFE1E0CD54DF4FE883AB
:109C5000C35BD04082CDC655DF4F8881CA5AD04001
:109C6000807F19F46894B0F807CF23E0B22AD12C92
:109C70006BCF91E0CD54DF4F9883C35BD040C110D0
:109C800055C2D12C0FEF1FEFA114B10439F0A5017B
:109C9000B401CE0187559F4F0E941E35D4011996FD
:109CA0008D919C91009709F49CC0CF54DF4FE880C0
:109CB000F980C15BD040DC01ED91FC910488F5890D
:109CC000E02DCD54DF4FC880C35BD040C755DF4F78
:109CD0000881C95AD040C655DF4F1881CA5AD040B2
:109CE000C555DF4F2881CB5AD040C455DF4F38814E
:109CF000CC5AD040C355DF4F4881CD5AD040C255D1
:109D0000DF4F5881CE5AD040C155DF4F6881CF5ABE
:109D1000D040C055DF4F7881C05BD04019958C0191
:109D2000F40181859285DC01ED91FC91028CF38D2B
:109D3000E02D1995059711F46894A0F8DD2021F025
:109D40006D2DC4010E94F51CC554DF4FE881F981D7
:109D5000CB5BD040359721F0B501C4010E94B541DD
:109D600063EB77E08FE29FE00E94B489B8018FE255
:109D70009FE00E94799C6CEA77E08FE29FE00E946E
:109D8000B4890E9406AAAB01BC01C354DF4FC8804E
:109D9000D980EA80FB80CD5BD0404C195D096E090B
:109DA0007F092AE08FE29FE00E94D2878FE29FE046
:109DB0000E941E880C948744A1E0CD54DF4FA883F5
:109DC000C35BD0405CCFB1E0CD54DF4FB883C35B01
:109DD000D04055CFE1E0CD54DF4FE883C35BD040A6
:109DE0004ECFF4018085853009F464C0863009F0D7
:109DF000A5CF70E060E0C4010E94041C7C010097C4
:109E000009F49CCF712C612C97FF06C0F194E1946A
:109E1000F10866246394712CC7010197863591057A
:109E200008F08CCFC755DF4F0881C95AD04010E0E9
:109E3000CE2C61E08E2D0E947CA8672859F101305C
:109E4000110521F061E00C30110509F460E0062FE6
:109E500010E08C2D0E944EA868EC77E08FE29FE026
:109E60000E94B489B7018FE29FE00E94799C66EC62
:109E700077E08FE29FE00E94B489B8018FE29FE013
:109E80000E94799C8FE29FE00E941E886894A0F84F
:109E9000B0F886C00130110551F091E080E00C303F
:109EA000110509F090E0092F182F602FD2CF01E0A3
:109EB00010E0FBCFF2E02F16310409F474C023E068
:109EC0002216310429F02A94232809F037CFDECF57
:109ED000C4010E94E81B892B49F4D401ED91FC9147
:109EE0006081718182E195E00E94EFAACE018755E1
:109EF0009F4F0E94031420E030E048EC52E40E949F
:109F0000ACD70E9418DAC954DF4F688379838A83FB
:109F10009B83C75BD040C954DF4F48805980C75BE3
:109F2000D04088E00E945218CD54DF4F6883798377
:109F30008A839B83C35BD040CD54DF4F6880798098
:109F4000C35BD04062EC77E08FE29FE00E94B4896F
:109F5000C954DF4F68817981C75BD0408FE29FE0B1
:109F60000E94799C6DEB77E08FE29FE00E94B489BC
:109F7000CD54DF4F488159816A817B81C35BD040DA
:109F8000662777272AE08FE29FE00E94D2878FE240
:109F90009FE00E941E88B301A201C4010E94B8255F
:109FA00001E010E0CBCE6894A0F8B1F8F9CF0E94A0
:109FB0002239672B682B692B11F00C94FB46B12CCE
:109FC000A12C21E0CD54DF4F2883C35BD0400C94FB
:109FD00032472114310409F045C08081882311F4EF
:109FE0000C941844CE018F549F4F0E9451431C0182
:109FF000C655DF4F8881CA5AD0408F7071F5622DE7
:10A00000CE0187559F4F0E946536CF55DF4F28837D
:10A01000C15AD040CE55DF4F3883C25AD040CD55BB
:10A02000DF4F4883C35AD040CC55DF4F5883C45AC2
:10A03000D040CB55DF4F6883C55AD040CA55DF4F5B
:10A040007883C65AD040C955DF4F8883C75AD0405D
:10A05000C855DF4F9883C85AD0402114310411F4F9
:10A060000C9418440E94EB116B01C954DF4F7983A3
:10A070006883C75BD0406DE379E08FE29FE00E9488
:10A08000B489B6018FE29FE00E94799C66E379E093
:10A090008FE29FE00E94B489D401ED91FC91608130
:10A0A00071818FE29FE00E944E8960E379E08FE248
:10A0B0009FE00E94B489CF54DF4F68817981C15BF2
:10A0C000D0408FE29FE00E944E896EE279E08FE2FD
:10A0D0009FE00E94B489C954DF4FE881F981C75BD2
:10A0E000D04060E279E0E83CF10514F40C945D4660
:10A0F000CE0187559F4F0E941734CF54DF4FE88120
:10A10000F981C15BD040309711F40C94594480819F
:10A11000843211F00C9459446CE079E08FE29FE0B6
:10A120000E94B4898FE29FE00E941E880CEF1FEF0F
:10A130000C9487442F923F924F925F926F927F923E
:10A140008F929F92AF92BF92CF92DF92EF92FF9247
:10A150000F931F93CF93DF93CDB7DEB7A6970FB6BC
:10A16000F894DEBF0FBECDBF5C013B015090EE0600
:10A17000552009F4B8C08091A0088F5F8093A00893
:10A18000E091A408F091A508309709F4A4C0868056
:10A1900097802090A4083090A5082114310409F478
:10A1A00096C08114910409F492C0D40118968C9140
:10A1B0008F70853091F7C4010E94819C823068F3D2
:10A1C000B401CE0101960E94BF23CE0101960E94E8
:10A1D0006C14882309F45EC060E074E0CE0101963F
:10A1E0000E94DB1C892B09F455C01E8E1F8E18A2FD
:10A1F00019A21AA21BA21CA21DA28F8D8F708F8F75
:10A2000040E053E0BE016F5F7F4FCE014E960E944B
:10A210009A3561E879E08FE29FE00E94B48960E0BE
:10A2200074E0CE0101960E94911C8A859B8500975F
:10A2300089F1DC01ED91FC910488F589E02DCC24B5
:10A24000C394F12CE12C0E8D1F8D28A139A14AA1B8
:10A250005BA16CA17DA119958F3F9807D9F0E98189
:10A26000FA8160817181892BE9F48FE29FE00E947D
:10A270004E896FE779E08FE29FE00E94B48967E73B
:10A2800079E08FE29FE00E94B4898FE29FE00E9414
:10A290001E88512CF40182809380CE0101960E9489
:10A2A000A21477CF8FE29FE00E944E8965E779E0A4
:10A2B0008FE29FE00E94B48961E779E08FE29FE03E
:10A2C0000E94B4898FE29FE00E941E88E3CF8FE254
:10A2D0009FE00E941E888091A00881508093A00872
:10A2E00051101092EE0665E0D5018D919C910E946F
:10A2F0006C9C4C01009709F487C0FC018085859512
:10A300008595859585958EA32184328443845484D4
:10A310000E9406AAFEA1FF2309F476C0261A370A76
:10A32000480A590A1E8E1F8E18A219A2FE8F1F8D71
:10A330001F70106A1F8F2AA23BA24CA25DA224E0CC
:10A340006216710449F5D12CC12CE12C90E1F92E53
:10A350000F2F28A139A14AA15BA16CA17DA1C50144
:10A360000E94AE36C201B10128EE33E040E050E079
:10A370000E94B2D8BA01A9012AE030E08FE29FE042
:10A380000E94C48866E979E08FE29FE00E94B48968
:10A390008FE29FE00E941E8857FE36C082E028169A
:10A3A0003104410480E858067CF1D12CC12CE12C09
:10A3B00080E1F82E0E8D1F8D28A139A14AA15BA145
:10A3C0006CA17DA1C5010E94AE3619821A821B8242
:10A3D0001C821D821E821F8218861A811F701A839A
:10A3E000AEA1A983CC24C394F12CE12C0A2F2B819C
:10A3F0003C8140E05E816F817885C5010E94854384
:10A40000F40180858F708087F1E06F167104B9F4D4
:10A4100060E073E0C5010E94DB1C009781F0209191
:10A42000A2083091A3082630310549F4BC01C501CA
:10A430000E94B54160E073E0C5010E94911CD50106
:10A4400019968D919C910097D9F490E080E0A696A2
:10A450000FB6F894DEBF0FBECDBFDF91CF911F9135
:10A460000F91FF90EF90DF90CF90BF90AF909F90B3
:10A470008F907F906F905F904F903F902F900895B6
:10A48000DC01ED91FC910484F585E02D1995892B73
:10A49000E1F2F50181859285DC01ED91FC9104806A
:10A4A000F581E02DB3011995D2CFAF92BF92CF9233
:10A4B000DF92EF92FF920F931F93CF93DF93CDB76D
:10A4C000DEB76D970FB6F894DEBF0FBECDBF0E940A
:10A4D00006AA9B01AC016091000770910107809171
:10A4E000020790910307A12CB12C650118EEE12E13
:10A4F00013E0F12E00E010E00E941C2BF82E8823C0
:10A5000051F00E9406AA60930007709301078093A0
:10A510000207909303078091A0088F5F8093A008A3
:10A52000E091A408F091A5080681178194E0C92E56
:10A53000D12CF11003C082E0C82ED12CA090A40829
:10A54000B090A508A114B10429F10115110511F16C
:10A55000F80180858F708530A9F7C8010E94819C21
:10A56000823080F3B801CE0101960E94BF23CE0154
:10A5700001960E946C14882329F0B601CE01019641
:10A580000E949A50F80102811381CE0101960E9427
:10A59000A214D4CF8091A00881508093A00880910C
:10A5A000A2089091A3080597D9F1FF20C9F110E006
:10A5B00060910807709109076115710589F1111102
:10A5C0002FC0FB0180858F70853091F4CE010196FC
:10A5D0000E94BF2361E070E0CE0101960E949A5074
:10A5E00011E0892B09F410E0CE0101960E94A2141B
:10A5F000E0910807F0910907309791F082819381EB
:10A600009093090780930807892B91F6E091A4089D
:10A61000F091A50886819781909309078093080798
:10A620006D960FB6F894DEBF0FBECDBFDF91CF9110
:10A630001F910F91FF90EF90DF90CF90BF90AF9060
:10A6400008954F925F926F927F928F929F92AF92F6
:10A65000BF92CF92EF92FF920F931F93CF93DF930E
:10A66000CDB7DEB76D970FB6F894DEBF0FBECDBF86
:10A67000009709F4A4C0FC0120852F70253009F053
:10A680009EC02A015B01868097808091A0088F5F21
:10A690008093A0088114910409F48CC0F401808592
:10A6A0008F70843009F082C0618572858091A40822
:10A6B0009091A5080E94F79B3C01009709F476C091
:10A6C000FC0180858F70853009F070C0B301CE0128
:10A6D00001960E94BF23A114B104A9F0CE010196F6
:10A6E0000E946C14882379F0C12C7201F50100815D
:10A6F0001181228133814481558166817781CE0128
:10A7000001960E94854360E0C3010E946C9C009703
:10A71000D1F1FC0120852F702230A9F58185928529
:10A72000A385B4850797A105B10569F561E0C3016B
:10A730000E946C9CA201B5010E942153A114B10496
:10A7400089F5882379F18091A00881508093A00831
:10A75000CE0101960E94A21481E06D960FB6F89486
:10A76000DEBF0FBECDBFDF91CF911F910F91FF9044
:10A77000EF90CF90BF90AF909F908F907F906F9011
:10A780005F904F900895A114B10461F4CE01019639
:10A790000E946C14882331F0CE0101960E94E1538F
:10A7A000892B89F6CE0101960E94A214F4018280C1
:10A7B000938070CF8091A00881508093A00880E0A2
:10A7C000CCCFDF92EF92FF920F931F93CF93DF9343
:10A7D00000D000D01F921F92CDB7DEB77C01198246
:10A7E0001A821B821C821D821E821F8218868A8109
:10A7F0008F708A83D701ED91FC91608171818FE226
:10A800009FE00E944E896FE679E08FE29FE00E9410
:10A81000B489C7010E946C1481111BC066E679E0FF
:10A820008FE29FE00E94B4898FE29FE00E941E8821
:10A830000FEF1FEFC80128960FB6F894DEBF0FBECA
:10A84000CDBFDF91CF911F910F91FF90EF90DF90DF
:10A850000895C7010E94271DD82EF7018185928592
:10A86000009791F0DC01ED91FC910688F789E02DCD
:10A8700019958C0197FD08C081E00115110509F4B7
:10A8800080E00E94C618D6CFF7018085873059F046
:10A89000F5E0DF1689F1FD15F8F081E0D81619F121
:10A8A000A2E0DA1649F140E052E0B701CE0101968C
:10A8B0000E949A35F7018085873009F445C010F56C
:10A8C000833009F46AC0843011F167E579E08FE2E2
:10A8D0009FE00E94B48913C0B6E0DB1621F086EF3A
:10A8E0008D0D833000F767E479E08FE29FE00E94EE
:10A8F000B48901E010E09ECF80E00E94C61810E00D
:10A9000000E098CF883009F448C08930F1F660E063
:10A91000CE0101960E94E2128C016CE479E08FE294
:10A920009FE00E94B489B8018FE29FE00E94799C69
:10A930008FE29FE00E941E8891E080E0012B09F4E5
:10A9400090E0092F182F76CF0280F381E02D8085CB
:10A950008F7010E000E0853001F764E679E08FE267
:10A960009FE00E94B48950E040E070E060E0F701B1
:10A97000828193810E942153F82E082F10E061E616
:10A9800079E08FE29FE00E94B4898F2D0E94C61863
:10A990008FE29FE00E941E884DCFCE0101960E945B
:10A9A00022398B01BACF2F923F924F925F926F92D2
:10A9B0007F928F929F92AF92BF92CF92DF92EF924F
:10A9C000FF920F931F93CF93DF93CDB7DEB76097BE
:10A9D0000FB6F894DEBF0FBECDBF6130710509F42C
:10A9E00095C0DC0112966D917C916115710509F499
:10A9F0008DC04C0119821A821B821C821D821E820C
:10AA00001F8218868A818F708A8340E052E0CE01CF
:10AA100001960E949A3560E0CE0101960E94E212F2
:10AA20001C01F401828193810E94E81B2B013C01EF
:10AA3000D40117962D913D914D915C911A97D101BA
:10AA40000E94DCD82FEF30E040E050E00E9490D828
:10AA500029873A874B875C870E9406AA9B01AC0135
:10AA600089859A85AB85BC850097A105B10509F458
:10AA700068C0A12CB12C65017C018D01C301B2011C
:10AA80000E941C2B89874114510461047104F1F167
:10AA9000D40117968D919D910D90BC91A02D8D871D
:10AAA0009E87AF87B88B0E9406AA9B01AC018D855B
:10AAB0009E85AF85B8890097A105B10561F0A12CED
:10AAC000B12C65017C018D01C301B2010E941C2BD8
:10AAD000882309F451C0D40112966D907C9080E0D7
:10AAE0000E945218AB01BC01C3010E94B825232863
:10AAF00069F0F40184810E943F11D40116969C9163
:10AB0000891304C061E0C4010E94341D90E080E01C
:10AB100060960FB6F894DEBF0FBECDBFDF91CF9128
:10AB20001F910F91FF90EF90DF90CF90BF90AF906B
:10AB30009F908F907F906F905F904F903F902F905D
:10AB4000089591E099879FCFB985BB23F1F060E02C
:10AB5000C4010E94341DF401828193810E94E1535B
:10AB6000892BA1F640E050E0BA01D40112968D91F4
:10AB70009C910E94B825CACFF40184810E943F11A4
:10AB8000D40116969C918913DFCF232809F4BECFF8
:10AB9000F40184810E943F11D40116969C9189137F
:10ABA000B5CFB985B111B2CFADCFCF93DF93EC0163
:10ABB0006BEC76E18FE29FE00E94B4896C817D812D
:10ABC0008FE29FE00E94799C65EC76E18FE29FE046
:10ABD0000E94B4898FE29FE00E941E8861E08C8110
:10ABE0000E947CA86E818C810E944EA88A819B81E4
:10ABF000009729F040E050E0BA010E94B82581E0BA
:10AC000090E09093D8078093D7078A819B810E9418
:10AC1000E153181619065CF40A80DB81C02D80E030
:10AC20000E945218AB01BC01CE010E94B82581E000
:10AC300090E0DF91CF9108952F923F924F925F92D3
:10AC40006F927F928F929F92AF92BF92CF92DF923C
:10AC5000EF92FF920F931F93CF93DF93CDB7DEB7A1
:10AC6000C955D1090FB6F894DEBF0FBECDBF0E9403
:10AC700006AA9B01AC016091FC067091FD068091D3
:10AC8000FE069091FF06A12CB12C650110E3E12E88
:10AC900015E7F12E00E010E00E941C2B882309F438
:10ACA00001C2E091A408F091A508309709F4FAC117
:10ACB0008091A0088F5F8093A0082680378010E0E5
:10ACC0002114310409F434C1F10180858F7085307D
:10ACD000F9F460E0C1010E946C9CFC0181859285C1
:10ACE000A385B4850597A105B10591F4B101CE0105
:10ACF00001960E94BF23CE0101960E946C146696B5
:10AD00008FAF6697811108C0CE0101960E94A214F0
:10AD1000F10122803380D4CF25961CAE1DAE1EAE2D
:10AD20001FAE259729961CAE1DAE1EAE1FAE2997ED
:10AD300040E052E0BE016F5F7F4FCE018F5B9F4FBF
:10AD40000E949A35CE0101960E94E81B6B017C019E
:10AD500069966FAF69976A96DFAE6A9770E060E0B8
:10AD6000CE0101960E94041C4C01CE018F5B9F4FC7
:10AD70000E94031465966CAF7DAF8EAF9FAF659751
:10AD8000CE0101960E94271D182FB601DD0C880BFD
:10AD9000990B0E944DD720E030E048EC52E40E942D
:10ADA000A6D92B013C01CE0101960E94E153689681
:10ADB0009FAF8EAF689769EA73E18FE29FE00E94D0
:10ADC000B48965966CAD7DAD8EAD9FAD65970E94E3
:10ADD0001BA463EA73E18FE29FE00E94B489C30180
:10ADE000B2010E941BA46DE973E18FE29FE00E9413
:10ADF000B489612F70E08FE29FE00E94799CE1149A
:10AE0000F10409F48EC088E00E9452189B01AC0145
:10AE100044275527B70190E080E0AA24AA94BA2CD1
:10AE2000C12CD12C17E2E12E19E0F12E00E010E048
:10AE30000E941C2B882371F1F1016081718188E0EF
:10AE40009EE00E944E896DE873E188E09EE00E94DA
:10AE5000B489F1016081718181E295E00E94EFAADD
:10AE600090E080E0BC0169964FAD69976A965FAD4E
:10AE70006A97CE0101960E94B82562E070E0C40195
:10AE80000E94D01ACE0101960E94A21466961FADB0
:10AE900066973ECF20E030E048E152E4C301B201C2
:10AEA0000E944EDA18163CF4F101608171818DE246
:10AEB00095E00E94EFAA68968EAD9FAD6897892BAA
:10AEC00019F461E070E0DBCF20E030E040E85FE3C0
:10AED00065966CAD7DAD8EAD9FAD65970E9439D9FD
:10AEE0009B01AC01C301B2010E9446D770E060E053
:10AEF00087FDC5CFA301920165966CAD7DAD8EAD8A
:10AF00009FAD65970E9446D71816DCF66EE773E191
:10AF10008FE29FE00E94B4898FE29FE00E941E882A
:10AF2000B1CF64E773E18FE29FE00E94B489AACFBA
:10AF30008091A00881508093A0080E9406AA609387
:10AF4000FC067093FD068093FE069093FF060E9418
:10AF5000EB112B013C010E9406AA6B017C010E94AF
:10AF6000129C882309F466C080912E08811162C06A
:10AF700030E020E041E050E060E4CE0101960E9424
:10AF8000122E40E450E064E879E1CE0101960E947F
:10AF900089CE63EF74E0CE0101960E9466DD40E445
:10AFA00050E06BE473E1CE0101960E9489CEB301BB
:10AFB000A201CE018F5B9F4F0E945611BE016F5BB5
:10AFC0007F4FCE0101960E94D4AA30E020E041E0FC
:10AFD00050E060E4CE0101960E94122E40E450E061
:10AFE00064E879E1CE0101960E9489CE63EF74E0B6
:10AFF000CE0101960E9466DD40E450E064E473E116
:10B00000CE0101960E9489CEC701B60128EE33E039
:10B0100040E050E00E9490D8BA01A901CE018F5BB8
:10B020009F4F0E945611BE016F5B7F4FCE0101966C
:10B030000E94D4AA112309F44FC06EE673E18FE297
:10B040009FE00E94B4890E94EB11AB01BC012AE091
:10B050008FE29FE00E94D28766E673E18FE29FE075
:10B060000E94B4896091A008062E000C770B8FE235
:10B070009FE00E94799C64E573E18FE29FE00E946B
:10B08000B4894091F8065091F9066091FA067091E2
:10B09000FB062AE08FE29FE00E94D2878FE29FE0CA
:10B0A0000E941E88C75ADF4F0FB6F894DEBF0FBE4E
:10B0B000CDBFDF91CF911F910F91FF90EF90DF9067
:10B0C000CF90BF90AF909F908F907F906F905F9048
:10B0D0004F903F902F90089564E673E18FE29FE0D8
:10B0E0000E94B4890E94EB11AB01BC012AE08FE2FF
:10B0F0009FE00E94D2876CE573E1B0CF8F929F9260
:10B10000AF92BF92CF92DF92EF92FF920F931F9375
:10B11000CF93DF93CDB7DEB767970FB6F894DEBF56
:10B120000FBECDBF8C017B014C018BE0880E911CC2
:10B130009F8A8E8AF801128611861386148E138ECA
:10B14000672B09F463C0A090A408B090A508A114CF
:10B15000B10409F45BC06FE270E0C7010E9471DDC9
:10B160006C01892B09F44AC0F701DE01119690E0C9
:10B1700080E0BD012191222341F02F3231F0843152
:10B18000910519F02D930196F5CF860F971FFC01BD
:10B190001082C5010E94F79BF80191838083B6015C
:10B1A0006F5F7F4F4FE050E0C4010E94AADDCE01E7
:10B1B00046960E945143F801948F838F8E899F8910
:10B1C000892B09F41386C8010E946C14882319F096
:10B1D000C8010E94522267960FB6F894DEBF0FBED8
:10B1E000CDBFDF91CF911F910F91FF90EF90DF9036
:10B1F000CF90BF90AF909F908F900895B701C501F9
:10B200000E94F79BF80191838083DDCFF8011182C2
:10B210001082D9CF2F923F924F925F926F927F927E
:10B220008F929F92AF92BF92CF92DF92EF92FF9256
:10B230000F931F93CF93DF93CDB7DEB7C955D109D5
:10B240000FB6F894DEBF0FBECDBF3C01562E6296FE
:10B25000EFAE62976396FFAE639764960FAF649705
:10B2600065961FAF659766962FAF669767963FAF57
:10B27000679768964FAF689769965FAF69976A96C8
:10B28000CFAE6A972D2C4A2C3B2C009709F45CC159
:10B29000FC0180858295807F85958595859585952E
:10B2A000843009F43CC12CF4882309F441C180E0C6
:10B2B0002DC0853009F444C08630C9F76AE375E0D3
:10B2C000C3010E94F79B4C01009709F46FC0B12C99
:10B2D000A12CD12CC12C6296EFAC62976396FFAC87
:10B2E000639764960FAD649765961FAD65976696F4
:10B2F0002FAD669767963FAD679768964FAD689795
:10B3000069965FAD6997652D0E940A59C75ADF4F4C
:10B310000FB6F894DEBF0FBECDBFDF91CF911F9166
:10B320000F91FF90EF90DF90CF90BF90AF909F90E4
:10B330008F907F906F905F904F903F902F900895E7
:10B340008091A0088F5F8093A008868097808114E9
:10B35000910431F1A42CB32C6A96CFAC6A97D22C0D
:10B360006296EFAC62976396FFAC639764960FADFD
:10B37000649765961FAD659766962FAD669767963D
:10B380003FAD679768964FAD689769965FAD6997CF
:10B39000652DC4010E940A59F40182809380D7CFA1
:10B3A0008091A00881508093A00881CF6EE375E062
:10B3B000C3010E94F79B7C0163E475E0C3010E9416
:10B3C000F79B6C01552039F0F1E05F1609F488C055
:10B3D00010E000E00CC068E475E0C3010E94F79B38
:10B3E0004C016DE475E0C3010E94F79B8C01811450
:10B3F000910409F443010115110509F48301E114D5
:10B40000F10421F46A96EFAC6A97F22CC114D104CE
:10B4100011F4C42CD32C8114910409F492C0F401CA
:10B4200080858F70843009F08CC0818492840115EE
:10B43000110509F491C0F80180858F70843009F0FE
:10B440008BC001851285E114F10409F4C9C081148F
:10B45000910409F490C064EA77E18FE29FE00E94D2
:10B46000B489F701618572858FE29FE00E944E8961
:10B470006FE977E18FE29FE00E94B489B4018FE227
:10B480009FE00E944E898FE29FE00E941E88CE01BD
:10B490008F5A9F4F0E941734C114D10409F0F8C08D
:10B4A000F70180858F70843009F0F0C06185728566
:10B4B000CE0101960E947E58CE0101960E946C1426
:10B4C000882349F08114910409F469C0B401CE01C4
:10B4D00001960E9480A1CE0101960E94A214D6C0BE
:10B4E00062E575E0C3010E94F79B4C0167E575E0DA
:10B4F000C3010E94F79B8C018114910409F0CDC017
:10B5000068E475E0C3010E94F79B4C010115110529
:10B5100009F467CF892B09F072CF430170CF10E097
:10B5200000E0912C812CD12CC12CF12CE12C5FCF8F
:10B5300010E000E0912C812CD12CC12CF12CE12CBD
:10B540005ECF912C812C73CFCA2CDB2C6A96EFAC8A
:10B550006A97F22C912C812C00E020E033E040E14E
:10B5600050E0BE016F5B7F4FCE018F5A9F4F0E940C
:10B5700067208C0168CF65E977E18FE29FE00E9448
:10B58000B489F701618572858FE29FE00E944E8940
:10B5900060E977E18FE29FE00E94B48978CFCC2404
:10B5A000C394F12CE12C62960FAD629763961FADA8
:10B5B000639764962FAD649765963FAD65976696E1
:10B5C0004FAD669767965FAD679768966FAD689762
:10B5D00069967FAD6997CE0101960E9485437BCF26
:10B5E000C114D10409F452C00115110509F44EC06B
:10B5F000F60180858F70843009F044C069E877E1F6
:10B600008FE29FE00E94B489F601618572858FE226
:10B610009FE00E944E8964E877E18FE29FE00E94FC
:10B62000B489B8018FE29FE00E944E898FE29FE0CB
:10B630000E941E88F6016185728540E450E0CE01CB
:10B6400001960E94AADD0E94129C8823D9F0809165
:10B650002E08811117C06FE270E0CE0101960E94A2
:10B6600071DD892B51F4F6012185328543E050E0EC
:10B6700060E4CE0101960E94122EB801CE0101961F
:10B680000E94D4AAE114F10409F00ACF81E03ECE71
:10B690000115110509F0ACCF03CF892B09F0AFCE0E
:10B6A000A0CE2F923F924F925F926F927F928F9295
:10B6B0009F92AF92BF92CF92DF92EF92FF920F9341
:10B6C0001F93CF93DF93CDB7DEB7C057D1090FB625
:10B6D000F894DEBF0FBECDBF6F969FAF8EAF6F9752
:10B6E00062960FAF6297912F63961FAF6397649630
:10B6F0002FAF649765963FAF659766964FAF669795
:10B7000067965FAF679768966FAF689769967FAFE8
:10B710006997E196FFAEEEAEE1979F70292F30E07A
:10B72000AB963FAF2EAFAB97002361F1232B09F40B
:10B73000C0C1973039F5013109F493C1023109F4E0
:10B74000B0C10031F9F46FEF70E0CE018F5A9F4F16
:10B750000E94AD122A962FAF2A972B963FAF2B97B8
:10B760002C964FAF2C972D965FAF2D972E966FAFDF
:10B770002E972F967FAF2F9760968FAF6097619629
:10B780009FAF61976F96AEADBFAD6F971496ED9179
:10B79000FC91309709F477C286809780AD961FAEF2
:10B7A0001EAEAD97A5961FAE1EAEA597A1961FAE75
:10B7B0001EAEA197712C612C512C412C8114910447
:10B7C00009F46DC264ED74E0C4010E94F79B1C0192
:10B7D00065EE74E0C4010E94F79B6B969FAF8EAF3D
:10B7E0006B976CE575E0C4010E94F79BAF969FAF25
:10B7F0008EAFAF972114310409F42EC16B96EEADD4
:10B80000FFAD6B97309709F427C1D10118968C9141
:10B810008F70823009F020C180858F70823009F0EE
:10B820001BC160E675E0C4010E94F79BDC0119961C
:10B830002D913D914D915C911C97A9962CAF3DAFF8
:10B840004EAF5FAFA997E196EEADFFADE1973097B0
:10B8500009F4BBC0D401CD90DC90BF01C6010E94A9
:10B860007CDD892B09F0B1C062968FAD62978111A2
:10B8700027C163968FAD6397807FAB96EEADFFAD2A
:10B88000AB97379709F0ACC1882309F478C0CE0193
:10B890008F5A9F4F0E9422396B96EEADFFAD6B978A
:10B8A0000185128523853485672B682B692B09F464
:10B8B000B4C1023011052105310529F00F3F1F4F9A
:10B8C0002F4F3F4F31F562E675E08FE29FE00E9417
:10B8D0004E898FE29FE00E941E8821E030E040E028
:10B8E00050E06B96AEADBFAD6B9719962D933D931F
:10B8F0004D935C931C9761E0CE018F5A9F4F0E943D
:10B900008C3629A33AA34BA35CA36DA37EA38FA37C
:10B9100098A7CE018F5A9F4F0E942239F10161876B
:10B920007287838794878091A2089091A3080597D6
:10B9300031F1D401CD90DC90E12C33E0F32E62960E
:10B940000FAD629763961FAD639764962FAD6497B2
:10B9500065963FAD659766964FAD669767965FAD06
:10B96000679768966FAD689769967FAD69976F9690
:10B97000EEADFFAD6F97828193810E94AE36AF9698
:10B98000EEADFFADAF97309701F1B12CA12CD12CCA
:10B99000C12C6296EFAC62976396FFAC6397649696
:10B9A0000FAD649765961FAD659766962FAD669748
:10B9B00067963FAD679768964FAD689769965FAD9C
:10B9C00069976FEFCF010E940A596B96EEADFFADFC
:10B9D0006B9781859285A385B48582309105A105F9
:10B9E000B105A1F18F3F9F4FAF4FBF4F79F1F101EB
:10B9F00081859285A385B485A7964EAD5FADA79747
:10BA0000849F9001859F300D949F300D1124420E2C
:10BA1000531EAD96EEADFFADAD97AF01FF0F660BB8
:10BA2000770B481759076A077B0784F4AD969FAFD9
:10BA30008EAFAD97A5963FAF2EAFA597A7962EAD2B
:10BA40003FADA797A1963FAF2EAFA197A7964EAD5A
:10BA50005FADA797640E751ED40112968D909C90D1
:10BA6000ADCE60E870E0CE018F5A9F4F0E94AD12BC
:10BA700022962FAF229723963FAF239724964FAF5E
:10BA8000249725965FAF259726966FAF2697279622
:10BA90007FAF279728968FAF289729969FAF299732
:10BAA00071CE6AE070E0CE018F5A9F4F0E94AF13B3
:10BAB00069CE41E050E0AB965FAF4EAFAB9762CE40
:10BAC000482F50E070E060E06B96AEADBFAD6B9775
:10BAD00019964D935D936D937C931C97813009F477
:10BAE0005CC0823009F46CC06B96EEADFFAD6B9715
:10BAF00081859285A385B4850197A105B10501F5DE
:10BB0000F10181859285A385B4854497A105B1058E
:10BB1000BCF42EE130E040E050E0218732874387DB
:10BB200054876EE170E0CE018F5A9F4F0E94AD1294
:10BB300029A73AA74BA75CA76DA77EA78FA798ABAD
:10BB40008091A2089091A308059709F418CFF401F9
:10BB5000C080D180E12C43E0F42E62960FAD629755
:10BB600063961FAD639764962FAD649765963FAD5E
:10BB7000659766964FAD669767965FAD67976896CF
:10BB80006FAD689769967FAD69976F96AEADBFADA3
:10BB90006F9712968D919C91F0CEF101618572851F
:10BBA000CE018F5A9F4F0E94AD1229AF3AAF4BAFD3
:10BBB0005CAF6DAF7EAF8FAF21969FAF219794CFD3
:10BBC00070E060E0CE018F5A9F4F0E94AD1229AB0A
:10BBD0003AAB4BAB5CAB6DAB7EAB8FAB98AF84CF6E
:10BBE000882309F4CCCE60E0CE018F5A9F4F0E948B
:10BBF000E212092E000CAA0BBB0BF1018187928780
:10BC0000A387B4878091A2089091A308059709F4AF
:10BC1000B6CEE12C22E0F22EA0CF02301105210594
:10BC2000310559F10F3F1F4F2F4F3F4F31F16DE657
:10BC300075E08FE29FE00E944E898FE29FE00E94B4
:10BC40001E8822E030E040E050E06B96AEADBFAD24
:10BC50006B9719962D933D934D935C931C9762E0DF
:10BC6000CE018F5A9F4F0E948C36298F3A8F4B8F6F
:10BC70005C8F6D8F7E8F8F8F98A3F1011186128656
:10BC80001386148650CEA5961FAE1EAEA597A1961C
:10BC90001FAE1EAEA197712C612C512C412C61144A
:10BCA000710409F4A0C0C201B3010E9407D98B013D
:10BCB00065E976E18FE29FE00E94B489B3018FE2EB
:10BCC0009FE00E94799C6AE876E18FE29FE00E9403
:10BCD000B489EE24EA94F12CC201B7010E9407D97D
:10BCE0008FE29FE00E94799C63E876E18FE29FE01B
:10BCF0000E94B489B8018FE29FE00E94799C65E7B9
:10BD000076E18FE29FE00E94B489A5968EAD9FAD4B
:10BD1000A597B7010E9407D98FE29FE00E94799C06
:10BD20006EE676E18FE29FE00E94B489A1966EAD47
:10BD30007FADA1978FE29FE00E94799C6AE676E151
:10BD40008FE29FE00E94B4898FE29FE00E941E88EC
:10BD500019821A821B821C821D821E821F821886F3
:10BD60008A818F708A83B801CE0101960E94AD123C
:10BD700029873A874B875C876D877E878F87988B6B
:10BD800061E0012B09F462E0CE0109960E948C3635
:10BD900079018A013B014C01298BFA8A4B8B1C8B60
:10BDA0006D8B7E8A8F8B988E61E776E06F96EEAD15
:10BDB000FFAD6F97848195810E94F79BB12CA12CD8
:10BDC000D12CC12C9301A4016FEF0E940A596F96E8
:10BDD000AEADBFAD6F971496ED91FC913097F1F435
:10BDE00066246394712CC301C059DF4F0FB6F894D9
:10BDF000DEBF0FBECDBFDF91CF911F910F91FF909E
:10BE0000EF90DF90CF90BF90AF909F908F907F90FA
:10BE10006F905F904F903F902F900895868097800D
:10BE2000A1962EAD3FADA197032E000C440B550BF0
:10BE3000A3962CAF3DAF4EAF5FAFA397A5968EAD47
:10BE40009FADA597092E000CAA0BBB0B6D968CAF6E
:10BE50009DAFAEAFBFAF6D978114910409F260E65C
:10BE600075E0C4010E94F79B8C0165E474E0C40195
:10BE70000E94F79B3C0164ED74E0C4010E94F79BB3
:10BE80002C0165EE74E0C4010E94F79B61147104FB
:10BE900009F4C3C04114510409F4BFC0009709F468
:10BEA000BCC0D30118962C912F70223009F0B5C078
:10BEB000F20120852F70223009F0AFC0DC01189606
:10BEC0002C9118972F70223009F0A7C0F801C18477
:10BED000D284E384F484C114D10409F49EC0199679
:10BEE0008D919D910D90BC91A02D82309105A10561
:10BEF000B10509F496C08F3F9F4FAF4FBF4F09F474
:10BF000090C0A5962EAD3FADA597232B09F489C00F
:10BF1000D20119968D919C918C9D80018D9D100D63
:10BF20009C9D100D11242FEF30E0D8010E9432D9D2
:10BF30009601DD0C440B550B0E94B2D8A3966CAD54
:10BF40007DAD8EAD9FADA3970E9480D86D962CAD30
:10BF50003DAD4EAD5FAD6D970E94B2D819012A017B
:10BF6000F401608171818FE29FE00E944E8969E750
:10BF700075E08FE29FE00E944E89C8016FEF70E08C
:10BF80000E9407D98FE29FE00E94799C64E676E1E7
:10BF90008FE29FE00E94B4892AE030E0B201A10163
:10BFA0008FE29FE00E94C4888FE29FE00E941E887B
:10BFB000F30181859285A385B48582159305A40537
:10BFC000B50559F119861A861B861C861D861E86A4
:10BFD0001F86188A8A858F708A87B101CE010996DB
:10BFE0000E94AD1229833A834B835C836D837E83E9
:10BFF0008F839887B12CA12CD12CC12C79018A0177
:10C000009B01AC016FEFC4010E940A59D30119963C
:10C010002D923D924D925C921C97F4018280938008
:10C020001BCF212C312C2101C3CF6F927F928F9295
:10C030009F92AF92BF92CF92DF92EF92FF920F93B7
:10C040001F93CF93DF93CDB7DEB7A0970FB6F894C9
:10C05000DEBF0FBECDBF8C01862E7A01DC018D9133
:10C060009C911197892B09F466C01496ED91FC916F
:10C07000309709F460C080818071BFEF6B135DC0A1
:10C08000B1F481E0A0960FB6F894DEBF0FBECDBF2D
:10C09000DF91CF911F910F91FF90EF90DF90CF90A4
:10C0A000BF90AF909F908F907F906F900895433096
:10C0B000510539F3818082942FE0822263E577E095
:10C0C0008FE29FE00E94B4894AE050E0D8011396C5
:10C0D0006C918FE29FE00E94228861E577E08FE219
:10C0E0009FE00E94B489D8011496ED91FC91618182
:10C0F0006F704AE050E08FE29FE00E9422886EE479
:10C1000077E08FE29FE00E94B4894AE050E0682D1A
:10C110008FE29FE00E9422888FE29FE00E941E88AB
:10C12000D8011496ED91FC9181818F70881207C01F
:10C1300080818F7E808380E0A5CF8111FCCF198E16
:10C140001A8E1B8E1C8E1D8E1E8E1F8E18A28A8D1F
:10C150008F708A8FD8011496ED91FC9181818F7038
:10C160008815A9F1B3E0EB16F10489F16CE477E0EE
:10C170008FE29FE00E94B4894AE050E0F8016381B9
:10C180008FE29FE00E9422886AE477E08FE29FE0DE
:10C190000E94B489D8011496ED91FC9161816F7071
:10C1A0004AE050E08FE29FE00E94228867E477E057
:10C1B0008FE29FE00E94B4894AE050E0682D8FE250
:10C1C0009FE00E9422888FE29FE00E941E88F80173
:10C1D00020813181FCE0F81508F416C1E82DF0E06B
:10C1E0008827EA50FF498F4F0C941BD903614061A7
:10C1F000C161D861E461C1619A61C161E761F261C5
:10C20000AE61F5610162D8011496CD90DC90F60123
:10C2100081818F70853009F4F7C050F48230C1F00D
:10C220006DE875E0C9010E94F79B3C01912C4BC061
:10C230008730D1F08A30A1F766E875E0C9010E9425
:10C24000F79B3C01D6019C9092FA992490F83BC050
:10C2500060E875E0C9010E94F79B3C01D6019C9003
:10C2600090FA992490F82FC06FE775E0C9010E94F9
:10C27000F79B3C01F601908091FA992490F823C035
:10C2800062E975E0C9010E94F79B3C01D801149650
:10C29000ED91FC91808180FB992490F8982F9E7FEE
:10C2A00080FF916090836114710469F461E0CE01B4
:10C2B00049960E948C36298B3A8B4B8B5C8B6D8B0D
:10C2C0007E8B8F8B988FF801A080B1806EE375E034
:10C2D000C5010E94F79B6C0163E475E0C5010E94F3
:10C2E000F79B5C01892B81F4C114D10469F460E0EF
:10C2F000CE0149960E948C3629833A834B835C8316
:10C300006D837E838F839887D8011496ED91FC917D
:10C310006114710409F07CC0898D811179C0B82D38
:10C32000BF708B2E8181807F882A818280818F7E61
:10C330008083A7CE67E975E0C9010E94F79B3C01A5
:10C34000D8011496ED91FC91808181FB992490F89D
:10C35000982F9D7F81FF92609083B5CF6DE975E046
:10C36000C9010E94F79B3C01D8011496ED91FC9104
:10C37000808182FB992490F8982F9B7F82FF9460A4
:10C38000EBCF6DE875E0C9010E94F79B3C01892B5A
:10C3900009F04CCF62E0CE0149960E948C36298785
:10C3A0003A874B875C876D877E878F87988B3ECFD8
:10C3B00063EA75E0C9010E94F79B3C01D80114961D
:10C3C000ED91FC9190804CCF68EA75E0F3CF6EEA76
:10C3D00075E0C9010E94F79B3C01D8011496ED91CC
:10C3E000FC9149CF64EB75E0F4CF6BEB75E0C901CC
:10C3F0000E94F79B3C01D8011496ED91FC9190802E
:10C4000023CF61EC75E0F3CF912C712C612C5BCFC5
:10C4100083E0E816F104B9F0982D9F70892E818190
:10C42000807F882A818280818F7E8083E98CFA8C4C
:10C430000B8D1C8D2D8D3E8D4F8D58A1692DC30107
:10C440000E940A591ECE81818F70881509F419CE79
:10C45000829490EF8922882A81828081806168CFCE
:10C460008F929F92AF92BF92CF92DF92EF92FF9204
:10C470000F931F93CF93DF93CDB7DEB7CD55D1097F
:10C480000FB6F894DEBF0FBECDBF8C016B016115F6
:10C49000710519F041155105D1F468EC7BE08FE28C
:10C4A0009FE00E94B4896FEB7BE08FE29FE00E94E7
:10C4B000B489B8018FE29FE00E944E896DEB7BE06A
:10C4C0008FE29FE00E94B4898FE29FE030C0460F68
:10C4D000571FDA011C920E94EB114B016BEB7BE0C2
:10C4E0008FE29FE00E94B489B4018FE29FE00E9436
:10C4F000799C68EB7BE08FE29FE00E94B489B801F1
:10C500008FE29FE00E944E8965EB7BE08FE29FE027
:10C510000E94B489BAE38B16B1E09B06F4F468EA92
:10C520007BE088E09EE00E94B48988E09EE00E9463
:10C530001E88C35ADF4F0FB6F894DEBF0FBECDBFC3
:10C54000DF91CF911F910F91FF90EF90DF90CF90EF
:10C55000BF90AF909F908F90089566EA7BE08FE246
:10C560009FE00E94B489B6018FE29FE00E944E894D
:10C5700064EA7BE08FE29FE00E94B4898FE29FE053
:10C580000E941E881A821982FE0133968EE3DF0113
:10C590001D928A95E9F78091A2089091A3080597CA
:10C5A000D9F563E070E0C8010E94A62E7C01892BBA
:10C5B00009F045C0E091820DF091830D808180FFEC
:10C5C000B8CF62E070E0C8010E94A62E892BD9F096
:10C5D00064E270E0C8010E94B9DD892B09F0A9CF9F
:10C5E0006CE87BE08FE29FE00E94B489B8018FE2A3
:10C5F0009FE00E944E898FE29FE00E941E88C80142
:10C600000E94ABA696CF61E070E0C8010E94A62E02
:10C61000892B09F48ECFDCCF61E070E0C8010E9465
:10C62000A62E7C01892B21F562E070E0C8010E94F2
:10C63000A62E7C0161E87BE0892B09F441CFE00E56
:10C64000F11E68E77BE0C7010E9470CE892BC1F420
:10C65000F60101900020E9F73197EC19FD093297B6
:10C6600078F0C8010E94ABA6C6010E94F18E61CF8E
:10C670004FE350E0B801CE0101960E94AADDDFCF62
:10C6800064E270E0C8010E94B9DD892B09F051CF46
:10C69000B701CE018F5B9F4F0E947E58CE018F5B0A
:10C6A0009F4F0E946C14882339F1B601CE018F5B35
:10C6B0009F4F0E9480A118161906F4F489818823DF
:10C6C000D9F08091A2089091A3080597A9F060E69F
:10C6D0007BE08FE29FE00E94B489BE016F5F7F4FD5
:10C6E0008FE29FE00E944E898FE29FE00E941E88A9
:10C6F000CE0101960E94ABA6CE018F5B9F4F0E9498
:10C70000A21417CF3F924F925F926F927F928F92B7
:10C710009F92AF92BF92CF92DF92EF92FF920F93D0
:10C720001F93CF93DF93CDB7DEB7CE56D1090FB6A7
:10C73000F894DEBF0FBECDBFDC0114962D913C9165
:10C74000232B09F421C69B012250310922303105E7
:10C7500008F091C23B014C01FC018281803409F454
:10C76000F7C208F04AC0843008F085C28091ED0617
:10C770008F5F8093ED06A3016FEFC4010E941560E7
:10C78000D40112960C9112970695017013961C9184
:10C7900013978AEC810F803108F043C068EC75E094
:10C7A0008D919C910E94F79B7C010097D1F1FC0137
:10C7B00080858F708530A9F58091780D181324C07D
:10C7C0008091790D803401F580917A0D90917B0DE7
:10C7D0005C01990FCC08DD0860E0C7010E946C9CE9
:10C7E000FC0181859285A385B485A816B906CA0681
:10C7F000DB060CF065C0512C3EC0823409F4A8C29F
:10C8000008F439C28058AFCF1093780D80E480933C
:10C81000790D812F0E948FA990937B0D80937A0DC3
:10C82000D7CF212F30E0F901EA52F34E8491F9017C
:10C83000E058F34E1491F901E65DF34EF490FF20B9
:10C8400009F43BC081110E94E7A7EF2DF0E0EE0F45
:10C85000FF1FE35DF84FA591B491EC911E2331E0E9
:10C8600020E009F430E0832F922F552453940817C9
:10C87000190609F0C0CFF3E06F16710409F488C0FF
:10C88000D4011496ED91FC91E181EF70E150EC3010
:10C8900008F07EC0F0E08827EF5AFB498F4F0C94D8
:10C8A0001BD97264EE65A864DE64EE65F764EE651C
:10C8B0002B6558657165B365D56590E080E0D5CF8F
:10C8C00061E0C7010E946C9C55245394FC01818552
:10C8D0009285A385B4858A159B05AC05BD050CF032
:10C8E000CACF89CF0E9406AA9B01AC0144275527D5
:10C8F000D4011496ED91FC916281738190E080E007
:10C90000AA24AA94BA2CC12CD12C18EEE12E13E043
:10C91000F12E00E010E00E941C2B8823C9F1F401E5
:10C920000081118163EA75E0C8010E94F79B892BA1
:10C9300041F468EA75E0C8010E94F79B892B09F46D
:10C940000EC142E050E063E0C4010E94156020C0C7
:10C950000E9406AA9B01AC0144275527D4011496D6
:10C96000ED91FC916281738190E080E0AA24AA9409
:10C97000BA2CC12CD12C1CE2E12EFF24F39400E050
:10C9800010E00E941C2B42E050E064E0811184C062
:10C99000D4011496ED91FC91808183FB992790F945
:10C9A000951509F4D2C1982F907E09F439C1982FBA
:10C9B000907E90528F71892B808358C10E9406AA65
:10C9C0009B01AC0144275527D4011496ED91FC91AD
:10C9D0006281738190E080E0AA24AA94BA2CC12CD1
:10C9E000D12C16E9E12EF12C00E010E0CACF0E9414
:10C9F00006AA9B01AC0144275527D4011496ED915A
:10CA0000FC916281738190E080E0AA24AA94BA2C00
:10CA1000C12CD12C18EEE12E13E0F12E00E010E035
:10CA20000E941C2B882309F4B3CFF40100811181EB
:10CA30006EEA75E0C8010E94F79B892B41F464EB14
:10CA400075E0C8010E94F79B892B09F488C042E079
:10CA500050E068E079CF0E9406AA9B01AC01442710
:10CA60005527D4011496ED91FC916281738190E079
:10CA700080E0AA24AA94BA2CC12CD12C1CE2E12E6D
:10CA8000FF24F39400E010E00E941C2B42E050E0F1
:10CA900069E0882309F47CCFC4010E9415600E94DC
:10CAA00006AAD4011496ED91FC917383628370CF32
:10CAB0000E9406AA9B01AC0144275527D401149675
:10CAC000ED91FC916281738190E080E0AA24AA94A8
:10CAD000BA2CC12CD12C16E9E12EF12C00E010E08B
:10CAE000D3CF0E9406AA9B01AC0144275527D4014D
:10CAF0001496ED91FC916281738190E080E0AA240C
:10CB0000AA94BA2CC12CD12C18EEE12E13E0F12EF0
:10CB100000E010E00E941C2B882309F439CFF401B7
:10CB2000008111816BEB75E0C8010E94F79B892B96
:10CB300039F461EC75E0C8010E94F79B892B21F064
:10CB400042E050E06BE000CF6DE975E0C8010E9463
:10CB5000F79B42E050E066E0892B09F4F5CE42E015
:10CB600050E06DE0F1CE0E9406AA9B01AC01442783
:10CB70005527D4011496ED91FC916281738190E068
:10CB800080E0AA24AA94BA2CC12CD12C1CE2E12E5C
:10CB9000FF24F39400E010E00E941C2B882309F48A
:10CBA000F7CE42E050E06CE077CF0E9406AA9B01EE
:10CBB000AC0144275527D4011496ED91FC91628174
:10CBC000738190E080E0AA24AA94BA2CC12CD12CC5
:10CBD00016E9E12EF12C00E010E0DECF0E9406AA5B
:10CBE0009B01AC0144275527D4011496ED91FC918B
:10CBF0006281738190E080E0AA24AA94BA2CC12CAF
:10CC0000D12C18E5E12E12E0F12E00E010E00E9498
:10CC10001C2B882309F4BCCE42E050E060E094CEA7
:10CC20000E9406AAD4011496ED91FC911597738386
:10CC30006283E181EF70552009F445C0E230F1F0E4
:10CC400050F4EE23E9F1D4011496ED91FC9180812A
:10CC500050FA83F9B1CEE53089F0A3016AE0E730FC
:10CC600091F7C4010E9415608111EDCF8091ED060E
:10CC700081508093ED0690E080E088C3F40100814C
:10CC8000118167E975E0C8010E94F79B892BA9F41F
:10CC90006EEA75E0C8010E94F79B892B71F464EB82
:10CCA00075E0C8010E94F79B892B39F46FE775E0A6
:10CCB000C8010E94F79B892B19F0A30166E0D1CF30
:10CCC000A30161E0CECFE150ED3008F0BCCFF0E041
:10CCD0008827E259F9498F4F0C941BD97B6623664C
:10CCE0007E667E66236681662366A266A266A2666B
:10CCF000A266A2667E66A30162E0B3CFA30165E0EF
:10CD0000B0CF0D911C9167E975E0C8010E94F79BB7
:10CD1000892BA9F46EEA75E0C8010E94F79B892B64
:10CD200071F464EB75E0C8010E94F79B892B39F41C
:10CD30006FE775E0C8010E94F79B892B19F0A301EA
:10CD400067E08FCFA30160E08CCF8F71806434CE19
:10CD5000B3E06B16710409F48ECF68EC75E0F40152
:10CD6000808191810E94F79B8C01D40113968C9154
:10CD70009091780D8913EBC09091790D903409F062
:10CD8000E6C080917A0D90917B0D3C010115110553
:10CD900009F40DC1F80120852F70253009F007C175
:10CDA000C8010E94819C382EF3E0F81708F0DBC020
:10CDB00063E0C8010E946C9CDC0119968D919C91E6
:10CDC0003AE0E32EE89E6001E99ED00C1124A39680
:10CDD000DFAECEAEA39762E0C8010E946C9CDC017E
:10CDE00019968D919C91E89E2001E99E500C11248A
:10CDF0006201052C000CEE08FF08AF96CCAEDDAE4C
:10CE0000EEAEFFAEAF9761E0C8010E946C9C5C0182
:10CE100060E0C8010E946C9CDC011996CD90DD9009
:10CE2000ED90FC901C97A796CCAEDDAEEEAEFFAEBB
:10CE3000A7979301072C000C440B550B2C193D09A7
:10CE40004E095F09A396CEACDFACA397B601DD0C0B
:10CE5000880B990BAF96CCACDDACEEACFFACAF97CA
:10CE60006C197D098E099F090E9480D8D5011996F9
:10CE70002D913D914D915C911C97A796CCACDDAC6A
:10CE8000EEACFFACA7972C193D094E095F09A79698
:10CE90002CAF3DAF4EAF5FAFA7970E94B2D8AF9611
:10CEA000ACACBDACCEACDFACAF97A20EB31EC41E13
:10CEB000D51E45E0E42E3E1409F468C081E090E000
:10CEC000A396EEACFFACA397A701FF0C660B770B04
:10CED0004A155B056C057D050CF461C0B601A50122
:10CEE0006201052C000CEE08FF084C155D056E056F
:10CEF0007F050CF459C06A017B0122E032126BC03D
:10CF00006301770CEE08FF0860E0C8010E946C9C8A
:10CF1000FC0181859285A385B485C816D906EA06E9
:10CF2000FB060CF44CC261E0C8010E946C9CFC0141
:10CF300081859285A385B4858C159D05AE05BF05B9
:10CF40000CF099CE81E090E0A0E0B0E03BC280938D
:10CF5000780D90E49093790D0E948FA990937B0DAA
:10CF600080937A0D12CF8AE0869D5001879DB00C88
:10CF700011240B2C000CCC08DD08512C412C20E096
:10CF800038E2A3963FAF2EAFA39798CF64E0C801D5
:10CF90000E946C9CDC0119968D919C9191CF662426
:10CFA0006A9423E0722E9CCF712C612CA6CF2AE0CC
:10CFB000289F6001299FD00C11240D2C000CEE0835
:10CFC000FF08512C412C20E038E2A3963FAF2EAF52
:10CFD000A39781E090E0D4011496ED91FC916281D9
:10CFE0007381A301461B570B57FF03C05195419511
:10CFF0005109841795070CF4BFC08081982F929532
:10D0000096959770963008F0BAC09F5F9295990FE9
:10D01000907E8F71892BB2C0F70161857285DB012B
:10D020008C9181115EC2A114B10409F472C0D501C2
:10D0300018968C9118978F70843009F06AC01996F1
:10D040006D917C91CE0101960E947E58CE01019691
:10D050000E946C14882309F458C06114710409F407
:10D060005FC0E114F10431F0F70180858F708430E6
:10D0700009F441C025961CAE1DAE1EAE1FAE25970D
:10D0800029961CAE1DAE1EAE1FAE299723961FAD6E
:10D0900023971F7023961FAF239781E022968FAFAF
:10D0A0002297CC24C394F12CE12C01E024962FADDF
:10D0B000249725963FAD259740E027965FAD2797AB
:10D0C00028966FAD289729967FAD2997CE010196B6
:10D0D0000E9485431AC00115110529F0F8018085C9
:10D0E0008F70843019F065E775E0FBC1618572854A
:10D0F000FB01808196CF61857285FB018081882349
:10D1000021F0CE0101960E9480A1CE0101960E94DD
:10D11000A214D4011496ED91FC9173826282ABCD7E
:10D120000115110531F0D80118968C918F7084305B
:10D13000E9F025961CAE1DAE1EAE1FAE25972996B2
:10D140001CAE1DAE1EAE1FAE299723961FAD2397B2
:10D150001F7023961FAF239782E022968FAF2297EE
:10D16000CC24C394F12CE12C02E0A0CFF80161851E
:10D170007285DB018C91C3CF80818F718083808128
:10D18000803AB8F0C201550CAA0BBB0BC816D906E1
:10D19000EA06FB0671F0A396EEADFFADA397CF01B3
:10D1A000FF0FAA0BBB0BC816D906EA06FB0609F04F
:10D1B00062CD6616770609F45ECD6D961CAE1DAE87
:10D1C0001EAE1FAE6D976B968FAD6B978F7080669E
:10D1D0006B968FAF6B976D968CAD9DADAEADBFADC1
:10D1E0006D9765968CAF9DAFAEAFBFAF6597AAE068
:10D1F000B0E0A70196010E94D1D869966CAF7DAFCF
:10D200008EAF9FAF69976CE177E08FE29FE00E945D
:10D21000B4894AE050E0D40113966C918FE29FE00C
:10D220000E9422886AE177E08FE29FE00E94B48941
:10D23000CE018F5A9F4F0E9417346AE375E0F401C4
:10D24000808191810E94F79BB12CA12CD12CC12C03
:10D250006296EFAC62976396FFAC639764960FADEE
:10D26000649765961FAD659766962FAD669767962E
:10D270003FAD679768964FAD689769965FAD6997C0
:10D280006FEF0E940A59D4010D911C916EE375E075
:10D29000C8010E94F79B7C0163E475E0C8010E940D
:10D2A000F79B8C010097E1F1FC0180858F70843041
:10D2B000B9F56185728540E450E0CE0101960E9487
:10D2C000AADD6FE270E0CE0101960E9471DD892B2C
:10D2D00059F4D80119962D913C9143E050E060E457
:10D2E000CE0101960E94122E00E020E032E040E1E3
:10D2F00050E0BE016F5B7F4FCE018F5A9F4F0E945F
:10D3000067200E94129C882359F080912E08811179
:10D3100007C0BE016F5B7F4FCE0101960E94D4AA69
:10D32000E114F10409F4F5CEF70180858F708430A3
:10D3300009F0EFCE61857285CE0101960E947E587C
:10D34000CE0101960E946C14882309F4DECECC2411
:10D35000C394F12CE12C62960FAD629763961FADDA
:10D36000639764962FAD649765963FAD6597669613
:10D370004FAD669767965FAD679768966FAD689794
:10D3800069967FAD6997A2CE8FEF9FEFC259DF4FAD
:10D390000FB6F894DEBF0FBECDBFDF91CF911F91C6
:10D3A0000F91FF90EF90DF90CF90BF90AF909F9044
:10D3B0008F907F906F905F904F903F90089580E0A6
:10D3C00090E0DC01F40124813581F901428153812F
:10D3D000052E000C660B770B84179507A607B70779
:10D3E00009F449CC3C01D4010D911C916EE375E028
:10D3F000C8010E94F79B5C0163E475E0C8010E94CC
:10D40000F79B6C01A114B10419F4892B09F481CEA6
:10D4100062E975E0C8010E94F79B7C016DE875E048
:10D42000C8010E94F79B8C0162E277E08FE29FE0E7
:10D430000E94B4894AE050E0F40163818FE29FE0EA
:10D440000E94228860E277E08FE29FE00E94B48928
:10D45000B3018FE29FE00E94799C8FE29FE00E94DF
:10D460001E88C114D10409F4DECDD60118968C9122
:10D4700018978F70843009F0D6CD19966D917C91F4
:10D4800040E450E0CE0101960E94AADD0E94129C69
:10D49000882309F4C8CD80912E088111C4CD6FE294
:10D4A00070E0CE0101960E9471DD892B51F4F601E6
:10D4B0002185328543E050E060E4CE0101960E9470
:10D4C000122E6114710409F406CEE114F10439F04E
:10D4D000D70118968C918F70843009F49DCD6AE63F
:10D4E00075E0CE0101960E94D4AA9DCD8F929F92A5
:10D4F000AF92BF92CF92DF92EF92FF920F931F9362
:10D50000CF93DF9300D000D0CDB7DEB720910407D2
:10D5100030910507232B09F4C5C02091F70621118E
:10D52000C1C04C018091F7068F5F8093F706809110
:10D53000A0088F5F8093A0080E9406AA9B01AC01FF
:10D540006091F3067091F4068091F5069091F606CD
:10D55000A12CB12C65011BE0E12EF12C00E010E0C4
:10D560000E941C2B882309F452C0E0910407F0911B
:10D5700005070681178101151105B9F1F8018085AC
:10D580008F70863071F56AE375E0C8010E94F79BE1
:10D590000097D1F0FC0120852F702530A9F4E6809A
:10D5A000F780E114F104E9F0FA82E982B801CE01D2
:10D5B00001960E941F1BB401CE0101960E94826356
:10D5C000F701E280F380EDCF1A83098370E060E019
:10D5D000CE0101960E941F1BB401CE0101960E944C
:10D5E0008263F80102811381C6CFF3E08F169104A4
:10D5F00051F00E9406AA6093F3067093F40680939C
:10D60000F5069093F6061092780D1092790D83E04E
:10D6100088169104E9F10E9406AA9B01AC01609171
:10D62000EF067091F0068091F1069091F206A12C20
:10D63000B12C650118E8E12E13E1F12E00E010E0B5
:10D640000E941C2B882321F1E0910407F09105072B
:10D65000068117810115110589F0F80180858F7009
:10D66000863041F41A83098370E060E0CE010196B0
:10D670000E941F1BF80102811381ECCF0E9406AAB1
:10D680006093EF067093F0068093F1069093F20694
:10D690008091A00881508093A0088091F706815066
:10D6A0008093F70626960FB6F894DEBF0FBECDBF67
:10D6B000DF91CF911F910F91FF90EF90DF90CF906E
:10D6C000BF90AF909F908F9008954F925F926F920E
:10D6D0007F92AF92BF92CF92DF92EF92FF920F9321
:10D6E0001F93CF93DF93CDB7DEB76D970FB6F89446
:10D6F000DEBF0FBECDBF67E374E18FE29FE00E9403
:10D70000B4898FE29FE00E941E880E9406AA2B0126
:10D710003C018091A008882351F10E9406AA9B0138
:10D72000AC01A12CB12C650110E1E12E17E2F12E24
:10D7300000E010E0C301B2010E941C2B811117C050
:10D740000E94728F8091A2089091A308059741F0E2
:10D750008091A4089091A508892B11F00E94555240
:10D760000E941C5682E090E00E94766AD2CF80919F
:10D77000A008FF24F394882359F064E174E188E061
:10D780009EE00E94B48988E09EE00E941E88F12CF1
:10D790006EEF73E18FE29FE00E94B4898FE29FE019
:10D7A0000E941E8880910A078F5F80930A07E0918C
:10D7B000A408F091A508309781F106811781011521
:10D7C000110559F1D80118968C918F708530B9F7F1
:10D7D000C8010E94819C882391F3F80160817181C6
:10D7E000CE0101960E947E58CE0101960E946C14D3
:10D7F000882359F08A859B85009739F0DC01ED91EB
:10D80000FC910284F385E02D1995CE0101960E94CA
:10D81000A214F80102811381D2CF1092090710924D
:10D82000080766EF73E18FE29FE00E94B4898FE200
:10D830009FE00E941E8864E670E080E090E00E9415
:10D84000D4A910922B081092A1086EED73E18FE21B
:10D850009FE00E94B4890E94EB11AB01BC012AE059
:10D860008FE29FE00E94D287809106079091070780
:10D870000E94F0A410920707109206071092050765
:10D88000109204071092A5081092A40810922D0877
:10D8900010922C0810929E0810929D0810929C08DD
:10D8A00010929B0869ED73E18FE29FE00E94B489BA
:10D8B0000E94EB11AB01BC012AE08FE29FE00E94C5
:10D8C000D2878FE29FE00E941E8810929F0880916D
:10D8D0000A07815080930A078F2D6D960FB6F89432
:10D8E000DEBF0FBECDBFDF91CF911F910F91FF9093
:10D8F000EF90DF90CF90BF90AF907F906F905F9050
:10D900004F90089580912E088F5F80932E08A895E0
:10D9100083E090E00E94766A0E94728F80912E08C8
:10D92000815080932E080895CF92DF92EF92FF925C
:10D93000CF93DF93EC018C85883068F40E946E975A
:10D940000E9406AA6B017C018C850E948A97811136
:10D9500009C088E08C87DF91CF91FF90EF90DF9036
:10D96000CF9008950E94826C61E070E080E090E0CA
:10D970000E94D4A90E9406AAAB01BC014C195D0902
:10D980006E097F098D859E85B0E0A0E04817590794
:10D990006A077B07C8F28C850E947C97DACFCF920A
:10D9A000DF92EF92FF921F93CF93DF93EC017B0105
:10D9B0006A018C85883048F40E948A97882319F080
:10D9C0008C850E946E9788E08C87F7018281938115
:10D9D000A481B5810097A105B10551F490E080E0E4
:10D9E000DF91CF911F91FF90EF90DF90CF9008953E
:10D9F0008F3F9F4FAF4FBF4F89F370E060E081E2F0
:10DA00000E94C597182F8C87883040F780E591E0F9
:10DA10000E9440A5A7014E5F5F4F24E030E06CE01C
:10DA200070E0812F0E943B27B601812F0E949997B9
:10DA300064E070E0812F0E94A6920E9406AA6B010A
:10DA40007C018C850E948A97873121F18C3111F1FC
:10DA5000882321F20E9406AAAB01BC014C195D0982
:10DA60006E097F098D859E85B0E0A0E0841795073B
:10DA7000A607B70748F00E94826C61E070E080E082
:10DA800090E00E94D4A9DDCF8C850E947C9788E02D
:10DA90008C87A4CF81E090E0A3CF8F929F92BF921A
:10DAA000CF92DF92EF92FF920F931F93CF93DF936A
:10DAB000CDB7DEB7A3970FB6F894DEBF0FBECDBFCC
:10DAC0008091060790910707892B09F44AC280913B
:10DAD000A008811146C28091A0088F5F8093A008A2
:10DAE0006DEC7EE08EEF9DE00E94B4898EEF9DE0AC
:10DAF0000E941E8800910607109107076CEC75E0E4
:10DB0000C8010E94F79B9093A5088093A40862ED3A
:10DB100075E0C8010E94F79B90932D0880932C0814
:10DB200063E376E0C8010E94F79B9093050780931A
:10DB3000040769ED75E0C8010E94F79B90939E0869
:10DB400080939D080E9438321092090710920807AE
:10DB5000E091A408F091A508309709F4F2C0E6809E
:10DB6000F7800091A4081091A5080115110509F48A
:10DB7000E1C0E114F10409F4DDC0D70118968C91DD
:10DB80008F70853091F7C7010E94819C823068F3C5
:10DB9000B701CE0101960E94BF23CE0101960E94DB
:10DBA0006C14882309F464C08A859B85009769F505
:10DBB00070E060E0CE0101960E94041C8C01912C63
:10DBC000812C97FF06C01195019511098824839433
:10DBD000912CCE0101960E94271DC82ED12C89853B
:10DBE000853009F44EC0863009F042C0B02E61E0A5
:10DBF000802F0E947CA861E0892809F479C0CA942A
:10DC0000CD2809F079C060E077C0DC01ED91FC918E
:10DC10000484F585E02D1995892B49F08A859B852B
:10DC2000DC01ED91FC910284F385E02D19958A8544
:10DC30009B85DC01ED91FC910680F781E02D199523
:10DC4000892BB1F0CE0101960E94271D882331F067
:10DC500060E071E0CE0101960E94B51C8D819E812D
:10DC6000892B31F060E072E0CE0101960E94B51C74
:10DC7000D7011296ED90FC90CE0101960E94A2145D
:10DC800070CFCD2829F462E0CE0101960E94F51CE8
:10DC900060E071E0CE0101960E94B51C8D819E81ED
:10DCA000892B31F060E072E0CE0101960E94B51C34
:10DCB00061E0802F0E947CA860E0802F0E944EA827
:10DCC00065EC7EE08FE29FE00E94B489B8018FE2AC
:10DCD0009FE00E94799C60EC7EE08FE29FE00E94D2
:10DCE000B4896EEB7EE08FE29FE00E94B489C0CFE2
:10DCF000CA94CD2809F087CFC62ED12C8B2D0E9437
:10DD00004EA869EB7EE08FE29FE00E94B489B801E3
:10DD10008FE29FE00E94799C67EB7EE08FE29FE0BC
:10DD20000E94B489B6018FE29FE00E94799C65EB66
:10DD30007EE0D9CFF801868197819093090780937F
:10DD400008078FE29FE00E941E88E0910407F0918F
:10DD50000507309709F48AC08091A0088F5F8093EF
:10DD6000A008068117810115110509F47AC0D801B0
:10DD700018968C918F70863009F069C01F8F0E8FB6
:10DD800070E060E0CE014E960E941F1B8AA19BA10D
:10DD9000892B09F45CC08091060790910707892BB5
:10DDA00009F455C0EE8CFF8CF70180858F708630AA
:10DDB00099F56AE375E0C7010E94F79B0097F1F0BF
:10DDC000DC0118962C9118972F702530B9F416960F
:10DDD000CD90DC90C114D104F9F0DA82C982B70188
:10DDE000CE0101960E941F1BED81FE8110821182DF
:10DDF00012821382F601C280D380ECCFFA82E982CC
:10DE000070E060E0CE0101960E941F1B62E070E0AE
:10DE1000CE0101960E948263EAA1FBA110821182C9
:10DE20001282138288A1843068F462E0823008F0A4
:10DE300060E089A10E947CA8EAA1FBA18181807F8A
:10DE4000818305C0803441F060E0823431F0D80134
:10DE500012960D911C9187CF62E089A10E947CA847
:10DE6000F6CF8091A00881508093A00868EA7EE0F8
:10DE70008EEF9DE00E94B48960EA7EE08EEF9DE027
:10DE80000E94B48981E02091A4083091A508232B39
:10DE900009F480E00E94B01867E97EE08EEF9DE013
:10DEA0000E94B48981E02091040730910507232B5B
:10DEB00009F480E00E94B01860E97EE08EEF9DE0FA
:10DEC0000E94B48981E020919D0830919E08232B07
:10DED00009F480E00E94B01867E87EE08EEF9DE0D4
:10DEE0000E94B48980912B080E94B0188EEF9DE0AB
:10DEF0000E941E8862E87EE08EEF9DE00E94B48959
:10DF00000E94EB11AB01BC012AE08EEF9DE00E9464
:10DF1000D2878EEF9DE00E941E8881E08093A10849
:10DF20008CEC9DE00E94A517882351F08CEC9DE0BD
:10DF30000E94946C84E090E09093A3088093A208E0
:10DF40008091A2089091A308079731F484E090E0B3
:10DF50009093A3088093A2088091A0088150809399
:10DF6000A008A3960FB6F894DEBF0FBECDBFDF9119
:10DF7000CF911F910F91FF90EF90DF90CF90BF90C6
:10DF80009F908F900895EF92FF920F931F93CF93DE
:10DF9000DF9300D01F92CDB7DEB78C017B01FB0170
:10DFA00084858830A8F082E394E0F801918380832F
:10DFB0001282138214821582C8010F900F900F9065
:10DFC0000F90DF91CF911F910F91FF90EF900895E7
:10DFD00080E591E00E9440A524E030E0AE014F5F73
:10DFE0005F4F6CE070E0F70184850E946A28BE01F3
:10DFF0006F5F7F4FC8010E94EA89DECFEF92FF92E8
:10E000000F931F93CF93DF93CDB7DEB764970FB60F
:10E01000F894DEBF0FBECDBF0D871E872F87388BCC
:10E02000498B5A8B6B8B7C8B64E276E18FE29FE0AD
:10E030000E94B489CE010D960E9417349E85892FC7
:10E040008F70082F10E02D85222309F4A8C0011538
:10E05000110509F474C0813009F471C08130A0F158
:10E060008230C1F18C3009F081C092959F7069892E
:10E070007A899C3011F070E060E0CE0101960E9438
:10E0800035876FE476E0C7010E947CDD892B09F0BB
:10E090003FC0BE016F5F7F4FCE0107960E942C8765
:10E0A000CE0107960E94F4A6BC0180E39CE00E948A
:10E0B000A689CE0107960E94F98601E010E0CE0104
:10E0C00001960E94F98616C063E176E18FE29FE037
:10E0D0000E94B4896FEF75E18FE29FE00E94B489DE
:10E0E0008FE29FE00E941E888E85807F01E010E015
:10E0F00009F400E0C80164960FB6F894DEBF0FBEC5
:10E10000CDBFDF91CF911F910F91FF90EF900895B8
:10E110006FE576E0C7010E947CDD00E0892B71F697
:10E12000BE016F5F7F4FCE0107960E942C87CE0104
:10E1300007960E94F4A6BC0183E19BE0B8CF213092
:10E1400031F1223049F162EF75E18FE29FE00E94E8
:10E15000B4894AE050E06D858FE29FE00E942288FA
:10E160008FE29FE00E941E8801E010E062EE75E100
:10E170008FE29FE00E94B489B8018FE29FE00E9485
:10E18000799C8FE29FE00E941E8800E003C02093EC
:10E19000290201E010E0AECF10922902FACF8130BF
:10E1A00009F05CCFD0CFAF92BF92CF92DF92EF92C7
:10E1B000FF920F931F93CF93DF93CDB7DEB7CA596A
:10E1C000D1090FB6F894DEBF0FBECDBF8E010F5B35
:10E1D0001F4FD8011D921C92FE01ED5BFF4F8EE197
:10E1E000DF011D928A95E9F78091DB0D9091DC0D9E
:10E1F000892B09F49FC10E94BA9C882309F49AC113
:10E20000A091DB0DB091DC0D52961C921E9251979D
:10E2100054961C921E92539784E890E01D969C930E
:10E220008E931C971E961C921E9780E090E350964A
:10E230009C938E931F97ED91FC9111970088F18923
:10E24000E02D60E270E0CD0119954FE150E0B8019A
:10E250008091DB0D9091DC0D0E94119D7C018091DD
:10E26000DB0D9091DC0DDC01ED91FC910488F589CA
:10E27000E02D1995E114F10409F45CC1F801EE0DEB
:10E28000FF1D10828091E80D1F928F938091E70D02
:10E290001F928F938091E60D1F928F938091E50DD1
:10E2A0001F928F938091E40D1F928F938091E30DC5
:10E2B0001F928F938EED95E09F938F931F9280E432
:10E2C0008F93FE0131966F01FF93EF930E94C4DD9F
:10E2D00060E171E18EEF9DE00E94B489B8018EEF9C
:10E2E0009DE00E944E89B6018EEF9DE00E944E890E
:10E2F0008EEF9DE00E941E887E01F1E6EF0EF11C7C
:10E30000D70113961C921E92129788EE93E0A0E01C
:10E31000B0E0F70184839583A683B78388E0848780
:10E3200088EE93E0968785878CEB93E091838083DA
:10E33000108A1786128B018B148A138A80E590E06D
:10E34000968B858B118E6FE370E18FE29FE00E94C8
:10E35000B4896DED7DE0CE0185589F4F0E942C87DA
:10E36000BE0165587F4F8FE29FE00E94A6898FE231
:10E370009FE00E941E88CE0185589F4F0E94F9861B
:10E380006DE076E0CE0183579F4F0E9435876DE0A8
:10E3900076E0CE0185589F4F0E943587BE016558B3
:10E3A0007F4FCE018B579F4F0E942C876DED7DE0F4
:10E3B000CE018B579F4F0E949586BE0163577F4FBA
:10E3C0000E949586BC01CE018D569F4F0E942C87DE
:10E3D000CE018B579F4F0E94F986CE0185589F4FE3
:10E3E0000E94F986CE0183579F4F0E94F9868FE0E5
:10E3F00096E0CB57DF4F99838883C558D040C757E5
:10E40000DF4F19821882C958D040C557DF4F198293
:10E410001882CB58D040CD56DF4F88819981C3599F
:10E42000D040C957DF4F99838883C758D0406AE0EE
:10E4300071E18FE29FE00E94B4890E94EB11AB0171
:10E44000BC012AE08FE29FE00E94D2878FE29FE02A
:10E450000E941E8864E670E080E090E00E94D4A9EB
:10E4600085E19BE7D70150969C938E931F9769E2B5
:10E4700078E880EF91E90E9458CF8C010FB6F894AC
:10E48000DEBF0FBECDBF892BA1F183E090E00E94DB
:10E4900034CBD8011D969C938E931C97FC01F1827E
:10E4A000E0821282C7010E94A517882319F0C701D4
:10E4B0000E94946CD70153966D917C915497559618
:10E4C000AD90BC906115710509F44BC0CE01855823
:10E4D0009F4F0E94EA89A501BE0165587F4FC70181
:10E4E0000E94CF6C181619060CF489C1C8010E944D
:10E4F000C99161EA70E18FE29FE00E94B489EE2445
:10E50000EA94FE2CCE018D569F4F0E94F986C701DA
:10E51000C656DF4F0FB6F894DEBF0FBECDBFDF91FA
:10E52000CF911F910F91FF90EF90DF90CF90BF9010
:10E53000AF90089540E250E062E471E1C8010E94AA
:10E54000A7CE64E271E18EEF9DE00E94B489B8012C
:10E550008EEF9DE00E944E898EEF9DE00E941E8806
:10E5600091CEF70161897289A501C7010E94C71781
:10E57000B9CF8AE990E19F938F931F930F930E94E5
:10E58000DFCFD70158961C921E925797D8011C9640
:10E59000ED91FC91A080B1800F900F900F900F90A3
:10E5A00093E3C92ED12CD501ED91FC910084F18526
:10E5B000E02DC501199541975CF4B1E0CB1AD10863
:10E5C00039F064E170E080E090E00E94D4A9EBCFE4
:10E5D0006E01E9E9CE0ED11CDF92CF928AE490E180
:10E5E0009F938F931F930F930E94FCCF0F900F90D8
:10E5F0000F900F900F900F900197D1F4D6018D914D
:10E600009C91F701908F878B61E776E0CE0183576D
:10E610009F4F0E94358780E0C12CFAE0CF1272C074
:10E620008A3009F073C0CE0183579F4F0E94F9864C
:10E63000D7015796ED90FC90B8ECEB16F10409F079
:10E64000BCC06EEF70E18EEF9DE00E94B48964EF74
:10E6500071E080E090E00E94D4A9EF961FAE1EAE5C
:10E66000EF97C158DF4F19821882CF57D0408FEFF4
:10E670009FEFCF57DF4F99838883C158D0408CE0FC
:10E6800093E0ED969FAF8EAFED97CD57DF4F198397
:10E690000883C358D040F8948091060790910707EB
:10E6A000892B11F00E94656BCE0185589F4F0E9407
:10E6B00022A590930707809306077894C8010E94CB
:10E6C000C9918091060790910707892B09F063C0D3
:10E6D00061E776E0CE0183579F4F0E943587CE01D8
:10E6E00083579F4F0E9434B0CE0183579F4F0E94A3
:10E6F000F98667EE70E188E09EE00E94B489F12C13
:10E70000E12C00CF9DE0C91201C0C82EC8010E94B3
:10E71000A3CFD82ED7011F96AD90BC90A114B10401
:10E7200099F1BAE08B1779F0EDE08E1761F0FFEF09
:10E730008F1749F0682FCE0183579F4F0E94EB85BA
:10E740008C2DCD2C6ACFCF56DF4F88819981C1594E
:10E75000D040892B91F0BE0163577F4FCE01855881
:10E760009F4F0E942C87CE0185589F4FF501199528
:10E77000CE0185589F4F0E94F98661E776E0CE0171
:10E7800083579F4F0E94C986FFEFDF12D9CFC80180
:10E790000E94C99148CF0E944D6D8091A1088823A5
:10E7A00029F00E94AD9F67FF0E949B1B60EE70E105
:10E7B0008EEF9DE00E94B489A5CEE0E3EE16E1E085
:10E7C000FE0651F46CEC70E18EEF9DE00E94B4897E
:10E7D000C8010E94C99196CE64EB70E188E09EE08A
:10E7E0000E94B489C8010E94C991B70188E09EE0E7
:10E7F0000E94799C88E09EE00E941E8883CED7010B
:10E800005196BC9051975296AC90DF92CF928DE981
:10E8100090E19F938F931F930F930E94DFCFDF921E
:10E82000CF9288E990E19F938F931F930F930E945B
:10E83000DFCFD8011C96ED91FC9181E08283DF92BD
:10E84000CF9285E990E19F938F931F930F930E943E
:10E85000DFCFD8011C96ED91FC911282AF92BF924E
:10E860008FE590E19F938F931F930F930E94DFCFCB
:10E870000FB6F894DEBF0FBECDBFB12C86E5C82E13
:10E8800080E1D82E8B2D94E08902F0011124A5E8B7
:10E89000B0E0AC0FBD1FEA0FFB1F80819181009794
:10E8A00009F467CE2281338121153105C1F33F93ED
:10E8B0002F939F938F93DF92CF921F930F930E947A
:10E8C000DFCFB3940FB6F894DEBF0FBECDBFDACF63
:10E8D0000F931F93CF93DF93EB0102970CF49DC02E
:10E8E0000A811B8161E370E1C8010E9452CE892B2D
:10E8F00051F481E00E9470A088EC90E0DF91CF910C
:10E900001F910F9108956DE270E1C8010E9452CEEF
:10E91000892B11F480E0EECF6DE070E18EEF9DE089
:10E920000E94B4890E94AD9F63FB662760F981E075
:10E93000682770E08EEF9DE00E94799C8EEF9DE04D
:10E940000E941E888091DB0D9091DC0D892B09F4CB
:10E9500054C00A811B810E94BA9C882309F44DC0CF
:10E96000F80101900020E9F73197E01BF10BB09717
:10E9700008F043C0A091DB0DB091DC0D52961C92C3
:10E980001E92519754961C921E92539784E890E0E1
:10E990001D969C938E931C971E961C921E9780E04A
:10E9A00090E350969C938E931F97ED91FC91119755
:10E9B0000088F189E02D60E270E0CD011995B80181
:10E9C0008091DB0D9091DC0D0E944E898091DB0DD2
:10E9D0009091DC0DDC01ED91FC910190F081E02D36
:10E9E00060E019958091DB0D9091DC0DDC01ED91DB
:10E9F000FC910488F589E02D19956A817B818EEF61
:10EA00009DE00E944E8966E070E18EEF9DE00E94DD
:10EA1000B4898EEF9DE00E941E888091A20890919B
:10EA2000A30802977CF10E94D370883C910539F4C9
:10EA300024E030E03093A3082093A2085FCF8F3FFB
:10EA40009807C9F46BEE7FE08FE29FE00E94B489E3
:10EA50008FE29FE00E941E8810929F0883E090E062
:10EA60009093A3088093A2088CEC9DE00E94946C84
:10EA700089EC90E043CF2091A1082111D9CF2FE05C
:10EA800030E0D8CF6EED7FE088E09EE00E94B48950
:10EA900088E09EE00E941E8884EF91E02FCFCF9304
:10EAA000DF93CDB7DEB72E970FB6F894DEBF0FBE5B
:10EAB000CDBF8091A00881116BC06AE17FE08EEF2D
:10EAC0009DE00E94B4898EEF9DE00E941E88109206
:10EAD000FB0D1092FA0D80E090E19093F60D80937B
:10EAE000F50D84E890E09093FD0D8093FC0D81E09E
:10EAF0008093F70D80E090E29093F90D8093F80DEC
:10EB000089EE9DE00E948D268B37910509F0C4C0E7
:10EB10001C821B8282E293E09A83898389EE9DE0C6
:10EB20009E838D838FEF9FEF98878F838091060759
:10EB300090910707892B11F00E94656BCE01019619
:10EB40000E9422A5909307078093060789EE9DE017
:10EB50000E94B9148091060790910707892BD9F478
:10EB60006EE07FE088E09EE00E94B48988E09EE04D
:10EB70000E941E8861E776E0CE0109960E943587E3
:10EB8000CE0109960E9434B0CE0109960E94F98602
:10EB900090E080E014C06BEF7EE08EEF9DE00E947D
:10EBA000B4898EEF9DE00E941E880E944D6D809179
:10EBB000DB0D9091DC0D892B59F481E090E02E96CD
:10EBC0000FB6F894DEBF0FBECDBFDF91CF91089591
:10EBD0000E94BA9C882389F3A091DB0DB091DC0DD3
:10EBE00052961C921E92519754961C921E925397C5
:10EBF00084E890E01D969C938E931C971E961C9221
:10EC00001E9780E090E350969C938E931F97ED9112
:10EC1000FC9111970088F189E02D60E670E0CD014C
:10EC200019956091DB0D7091DC0D40E0CE010996E5
:10EC30000E947887BE01675F7F4F8DED9DE00E9447
:10EC4000FF85CE0109960E94F9868091DB0D909197
:10EC5000DC0DDC01ED91FC910488F589E02D19951E
:10EC60006DED7EE08FE29FE00E94B4896DED7DE066
:10EC7000CE0109960E942C87BE01675F7F4F8FE20D
:10EC80009FE00E94A6898FE29FE00E941E88CE012D
:10EC900009960E94F98691CF89EE9DE00E94D214D8
:10ECA000892BA1F089EE9DE00E94FC1461E776E0DB
:10ECB000CE0101960E943587CE0101960E9434B0A4
:10ECC000CE0101960E94F9860E94A8AF89EE9DE0D0
:10ECD0000E94B9146AEE7EE08EEF9DE00E94B48936
:10ECE0008EEF9DE00E941E8853CF0E944F75892BA6
:10ECF00049F486EF9FEF9093A3088093A20884EFD6
:10ED000091E0089588EC90E00895BF92CF92DF9251
:10ED1000EF92FF920F931F93CF93DF9300D000D019
:10ED2000CDB7DEB78C016B01FB0184819581892B06
:10ED3000D9F1E080F1806FE370E0C7010E9471DDDE
:10ED4000009791F19C012E193F09790137FD2CC0E4
:10ED500061E776E0CE0101960E943587F601848155
:10ED600095810097B9F08E159F0508F47C01F60196
:10ED700060817181FB01EE0DFF1DB0801082CE011C
:10ED800001960E94D386F60180819181E80EF91EDA
:10ED9000F701B082BE016F5F7F4FC6010E94FF8501
:10EDA000CE0101960E94F9866DE176E0C6010E94CF
:10EDB0007A85882319F1F801128A118A80E090E19E
:10EDC0009587848784E890E0948B838B81E08687A5
:10EDD00080E090E2908B878781E090E026960FB6E6
:10EDE000F894DEBF0FBECDBFDF91CF911F910F9181
:10EDF000FF90EF90DF90CF90BF9008956AE276E0A9
:10EE0000C6010E947A85882369F0F801128A118A66
:10EE1000148A138A84E890E095878487168680E0B8
:10EE200090E3D8CF90E080E0D9CFDF92EF92FF92CD
:10EE30000F931F93CF93DF9300D000D0CDB7DEB7F1
:10EE40008C017B0163EC75E1CE0101960E94FE8688
:10EE5000BE016F5F7F4FC7010E948F85D82ECE0104
:10EE600001960E94F986DD2019F1D8011296ED91E4
:10EE7000FC9113970190F081E02D60817181ED91FB
:10EE8000FC910288F389E02D26E336E04FEB55E054
:10EE9000C801199526960FB6F894DEBF0FBECDBFF8
:10EEA000DF91CF911F910F91FF90EF90DF90089528
:10EEB00068EA75E1CE0101960E94FE86BE016F5F91
:10EEC0007F4FC7010E948F85D82ECE0101960E94E8
:10EED000F986DD20A1F0D8011296ED91FC911397EF
:10EEE0000190F081E02D60817181ED91FC910288AB
:10EEF000F389E02D26E336E042EB55E0C9CF6DE81B
:10EF000075E1CE0101960E94FE86BE016F5F7F4FC4
:10EF1000C7010E948F85F82ECE0101960E94F986C6
:10EF2000FF2009F4B7CFD8011296ED91FC91139709
:10EF30000190F081E02D60817181ED91FC9102885A
:10EF4000F389E02D26E336E048E956E0A1CF6F9241
:10EF50007F928F929F92AF92BF92CF92DF92EF9269
:10EF6000FF920F931F93CF93DF93CDB7DEB72C970C
:10EF70000FB6F894DEBF0FBECDBF4C0180E39CE01E
:10EF80000E946B7F892B39F180E00E9452186093B8
:10EF9000CF077093D0078093D1079093D20780E377
:10EFA0009CE00E94497F682E8DE290E09A838983DD
:10EFB00069824FE350E0BE016F5F7F4F85E497E0C9
:10EFC0000E948CDD8091CD079091CE0701969093A1
:10EFD000CE078093CD0783E19BE00E946B7F892B56
:10EFE00039F180E00E9452186093C9077093CA07F4
:10EFF0008093CB079093CC0783E19BE00E94497FED
:10F00000782E8DE290E09A83898379824FE350E0F5
:10F01000BE016F5F7F4F87E897E00E948CDD809193
:10F02000C7079091C80701969093C8078093C707B8
:10F030008091CF079091D007A091D107B091D207CE
:10F04000892B8A2B8B2B09F0C7C08AE26812DEC09D
:10F050001092CF071092D0071092D1071092D207CA
:10F060001092CE071092CD0765E477E0CE010796A7
:10F070000E94358710924507CE0107960E948D8425
:10F080008B859C85892B09F4DEC16DE376E0CE018A
:10F0900001960E943587BE016F5F7F4FCE010796B4
:10F0A0000E945F85182FCE0101960E94F9861123D8
:10F0B00021F0809129028823A1F0BE01695F7F4F72
:10F0C000CE0101960E942C87CE0101960E94F4A6E3
:10F0D000BC0183E19BE00E94A689CE0101960E94BB
:10F0E000F986BE01695F7F4FCE0101960E942C8791
:10F0F000BE016F5F7F4FC4010E941577CE0101965C
:10F100000E94F98666E476E0CE0101960E9435877A
:10F11000BE016F5F7F4FCE0107960E945F85182F5B
:10F12000CE0101960E94F986112309F44FC1BE0158
:10F13000695F7F4F88E69FE00E948F85811183C1C0
:10F14000BE01695F7F4F88E69FE00E94E2864F81A3
:10F150005885D4011296ED91FC9113970190F0819E
:10F16000E02D60817181ED91FC910288F389E02DA1
:10F170002CE436E0C40119958091850790918607AB
:10F18000892B09F460C16EED75E18FE29FE00E946A
:10F19000B48910E000E0F0E1EF2EF12CB801CE01CF
:10F1A00007960E944D85FC018081882309F447C1A0
:10F1B0008B859C850817190708F041C18091850748
:10F1C000909186078130910509F442C1029709F4B4
:10F1D0006AC10F5F1F4FE2CF0E9406AA9B01AC01DC
:10F1E0006091CF077091D0078091D1079091D2079D
:10F1F000A12CB12C65011AE0E12EF12C00E010E009
:10F200000E941C2B882309F420CF22CFADE06A1680
:10F2100009F41ECF8091CD079091CE0780349105DF
:10F2200008F016CF8091C9079091CA07A091CB072B
:10F23000B091CC07892B8A2B8B2B09F040C1BAE205
:10F240007B1257C11092C9071092CA071092CB07C0
:10F250001092CC071092C8071092C70767E877E0B2
:10F26000CE0107960E94358710928707CE01079638
:10F270000E948D848B859C85892B09F49AC16DE34E
:10F2800076E0CE0101960E943587BE016F5F7F4F09
:10F29000CE0107960E945F85182FCE0101960E942D
:10F2A000F986112321F0809129028823A1F0BE0163
:10F2B000695F7F4FCE0101960E942C87CE01019697
:10F2C0000E94F4A6BC0180E39CE00E94A689CE01C6
:10F2D00001960E94F986BE01695F7F4FCE010196BB
:10F2E0000E942C87BE016F5F7F4FC4010E9415777B
:10F2F000CE0101960E94F98666E476E0CE01019681
:10F300000E943587BE016F5F7F4FCE0107960E9436
:10F310005F85182FCE0101960E94F986112309F40A
:10F320000BC1BE01695F7F4F84E79FE00E948F851C
:10F3300081113FC1BE01695F7F4F84E79FE00E945A
:10F34000E2864F815885D4011296ED91FC91139776
:10F350000190F081E02D60817181ED91FC91028836
:10F36000F389E02D2CE536E0C401199580918507DD
:10F3700090918607892B09F41CC160EE75E18FE23C
:10F380009FE00E94B489912C812C00E110E0B4012F
:10F39000CE0107960E944D85FC018081882309F4E7
:10F3A00004C18B859C858816990608F0FEC0809163
:10F3B0008507909186078130910509F4FFC0029777
:10F3C00009F427C1BFEF8B1A9B0AE1CF61E576E014
:10F3D000CE0101960E943587BE016F5F7F4FCE013F
:10F3E00007960E945F85182FCE0101960E94F9862C
:10F3F000112309F4C1CEBE01695F7F4F8EE69FE005
:10F400000E948F8581111FC0BE01695F7F4F8EE60C
:10F410009FE00E94E2864F815885D4011296ED91BB
:10F42000FC9113970190F081E02D60817181ED9145
:10F43000FC910288F389E02D27E536E09BCE8FE230
:10F440009FE00E941E88CE0107960E94F986EACEB0
:10F45000B801CE0107960E944D85DC018C9161E7D1
:10F4600076E0803114F469E874E08FE29FE00E9456
:10F470004E89B801CE0107960E944D85FC0180811E
:10F48000082E000C990BAA0BBB0B89839A83AB83C4
:10F49000BC83FE82ED82BE016F5F7F4F8FE29FE0F3
:10F4A0000E940F1B96CEB801CE0107960E944D8593
:10F4B000DC016C918FE29FE00E94BD888ACE0E94A1
:10F4C00006AA9B01AC016091C9077091CA0780919F
:10F4D000CB079091CC07A12CB12C65011AE0E12E4D
:10F4E000F12C00E010E00E941C2B882309F4A7CE29
:10F4F000A9CEEDE07E1609F4A5CE8091C7079091C4
:10F50000C8078034910508F09DCE81E090E02C96EC
:10F510000FB6F894DEBF0FBECDBFDF91CF911F9124
:10F520000F91FF90EF90DF90CF90BF90AF909F90A2
:10F530008F907F906F90089561E576E0CE010196FF
:10F540000E943587BE016F5F7F4FCE0107960E94F4
:10F550005F85182FCE0101960E94F986112309F4C8
:10F5600005CFBE01695F7F4F8AE79FE00E948F85CC
:10F5700081111FC0BE01695F7F4F8AE79FE00E9433
:10F58000E2864F815885D4011296ED91FC91139734
:10F590000190F081E02D60817181ED91FC910288F4
:10F5A000F389E02D21E636E0DFCE8FE29FE00E9476
:10F5B0001E88CE0107960E94F986A7CFB401CE011E
:10F5C00007960E944D85DC018C9161E776E08031E1
:10F5D00014F469E874E08FE29FE00E944E89B40160
:10F5E000CE0107960E944D85FC018081082E000CFB
:10F5F000990BAA0BBB0B89839A83AB83BC831E83B5
:10F600000D83BE016F5F7F4F8FE29FE00E940F1B53
:10F61000D9CEB401CE0107960E944D85DC016C91D4
:10F620008FE29FE00E94BD88CDCEFF920F931F9383
:10F63000CF93DF9300D000D0CDB7DEB78C01BC01F3
:10F64000CE0101960E942C87BE016F5F7F4F8FE233
:10F650009FE00E94A6898FE29FE00E941E88CE0153
:10F6600001960E94F98668E370E1CE0101960E943E
:10F67000FE86BE016F5F7F4FC8010E945F85F82E36
:10F68000CE0101960E94F986FF2069F0B801CE01F3
:10F6900001960E942C87CE0101960E9434B0CE01C3
:10F6A00001960E94F98626960FB6F894DEBF0FBE2B
:10F6B000CDBFDF91CF911F910F91FF9008955F9281
:10F6C0006F927F928F929F92AF92BF92CF92DF9272
:10F6D000EF92FF920F931F93CF93DF93CDB7DEB7D7
:10F6E000CF56D1090FB6F894DEBF0FBECDBF4C0187
:10F6F0008B01F42E4AE050E06F2D8FE29FE00E94D4
:10F7000022886EE57BE08FE29FE00E94B489B80119
:10F71000CE0101965C010E942C87B5018FE29FE02B
:10F720000E94A6898FE29FE00E941E88C5010E9468
:10F73000F98692E0F9126BC26CE57BE0C5010E948C
:10F74000FE86B501C8010E948F85F82EC5010E9472
:10F75000F986FF2009F4D0C220E04DE251E0B40167
:10F760008AEA9DE00E94C38EE0909B08F0909C087E
:10F7700065E57BE0CE0186599F4F0E94FE866EE4D0
:10F780007BE0CE018C599F4F0E94FE86CE01885AA5
:10F790009F4F0E94B9296E961FAD6E976D960FAD63
:10F7A0006D976C96DFAC6C976B96CFAC6B9761E7FF
:10F7B00076E0CE0181960E943587BE016F5D7F4F56
:10F7C000C5010E942C876C2DC5010E944A8666E601
:10F7D00076E00E947B866D2D0E944A8666E676E082
:10F7E0000E947B86602F0E944A8666E676E00E9431
:10F7F0007B86612F0E944A86BC01CE01825A9F4FB0
:10F800000E942C87C5010E94F986CE0181960E9434
:10F81000F98669E47BE0CE018E5A9F4F0E94FE86F6
:10F8200061E776E0CE01845B9F4F0E9435870BED48
:10F830001DE0D80118966C9170E084E0759567958D
:10F840008A95E1F7C5010E948E9C4D815E81698198
:10F850007A81CE01845B9F4F0E94BF85C5010E94C3
:10F86000F986F80160856F7070E0C5010E948E9C7A
:10F870004D815E8169817A81CE01845B9F4F0E94B8
:10F88000BF85C5010E94F9860F5F1F4FFDE0013E55
:10F890001F0779F663E47BE0CE018A5B9F4F0E94ED
:10F8A000FE8662E27BE0CE0181960E94FE86BE016A
:10F8B0006F5D7F4FCE01CE960E942C87BE016A5BA2
:10F8C0007F4FCE01CE960E949586BE01645B7F4F2E
:10F8D0000E949586BE016E5A7F4F0E949586BE019A
:10F8E000625A7F4F0E949586BE016C597F4F0E94DD
:10F8F00095868C014AE0B50180E590E00E94ECCE4F
:10F90000F50101900020E9F73197AF014A195B0931
:10F91000B501C8010E94BF85811103C0C8010E94C2
:10F920003886BE0166597F4FC8010E949586B7018F
:10F930000E947B86BC01C4010E94A689C4010E946A
:10F940001E88CE01CE960E94F986CE0181960E9435
:10F95000F986CE018A5B9F4F0E94F986CE01845BB7
:10F960009F4F0E94F986CE018E5A9F4F0E94F986C2
:10F97000CE01825A9F4F0E94F986CE018C599F4F2B
:10F980000E94F986CE0186599F4F0E94F986C401D4
:10F990000E941E8864E670E080E090E00E94D4A996
:10F9A000D401ED91FC910488F589E02DC4011995ED
:10F9B00001E010E088C028966EAD7FAD2897CE019B
:10F9C00081960E9480A1892B09F450C122961CAE19
:10F9D0001DAE1EAE1FAE229726961CAE1DAE1EAEED
:10F9E0001FAE26978FAD8F708FAF40E053E0BE0102
:10F9F0006F5D7F4FCE01CE960E949A3500E020E0E9
:10FA000033E040E250E0B501CE01CE960E9467207F
:10FA1000BC01C6010E94D38608EC10E129C1EE208A
:10FA200009F4F3C046E050E070E060E0C8010E94D5
:10FA3000EA84D8016D917C91CE0181960E947E5816
:10FA4000CE0181960E946C1400E911E08823B9F17F
:10FA500089A5873061F4CE0181960E94E15361E06F
:10FA6000892B09F462E0CE0181960E94F51C229652
:10FA70001CAE1DAE1EAE1FAE229726961CAE1DAE4E
:10FA80001EAE1FAE26978FAD8F708FAF40E053E054
:10FA9000BE016F5D7F4FCE01CE960E949A3500E089
:10FAA00020E033E040E250E0B501CE01CE960E9466
:10FAB0006720BC01C6010E94D38608EC10E1CE018C
:10FAC00081960E94A214C801C159DF4F0FB6F89465
:10FAD000DEBF0FBECDBFDF91CF911F910F91FF9081
:10FAE000EF90DF90CF90BF90AF909F908F907F90DE
:10FAF0006F905F900895F801608171810E94F79B7B
:10FB00007C01892B09F040C104E911E0DCCFEE2033
:10FB100009F47BC049E050E070E060E0C8010E9459
:10FB2000EA844AE0B401C5010E94788741E050E0D0
:10FB300069E474E0C8010E94BF854D815E816981DE
:10FB40007A81C8010E94BF856EEF7AE08FE29FE064
:10FB50000E94B489B801CE0181960E942C87BE0113
:10FB60006F5D7F4F8FE29FE00E94A6898FE29FE04A
:10FB70000E941E88CE0181960E94F98666EF7AE087
:10FB8000CE0181960E94FE86F801848195812DA187
:10FB90003EA182179307E1F4892BA1F1E080F18067
:10FBA00069A07AA0D7018D917D01882359F1082E93
:10FBB000000C990B0E9401DD6C01F30181913F0162
:10FBC000082E000C990B0E9401DDC816D90651F3CE
:10FBD000CE0181960E94F986552041F021E048EC43
:10FBE00050E0B4018AEA9DE00E94C38ED8018D9155
:10FBF0009C910E94F18E009711F484E991E08C01B0
:10FC0000C5013DC055245394E3CF01E97ECFB1E057
:10FC1000FB1270C06BE17BE0C5010E94FE86B5015E
:10FC2000C8010E945F85582EC5010E94F9865520A3
:10FC300049F1EE2051F346E050E070E060E0C80189
:10FC40000E94EA844AE0B401CE018A5B9F4F0E9481
:10FC50007887F80160817181CE0181960E947E587B
:10FC6000CE0181960E946C148111A5CE00E911E0AD
:10FC7000CE0181960E94A214CE018A5B9F4F0E9402
:10FC8000F98621CF64E07BE0C5010E94FE86B501C4
:10FC9000C8010E945F85F82EC5010E94F986F11007
:10FCA00036CF69EE7AE0C5010E94FE86B501C80133
:10FCB0000E945F85182FC5010E94F98600E011237C
:10FCC00009F401CF80E00E9470A061EC7AE08EEF31
:10FCD0009DE00E94B4898EEF9DE00E941E8861E73E
:10FCE00076E0C5010E943587C5010E9434B0C50188
:10FCF0000E94F98600E05DCE64E17BE0C5010E94D0
:10FD0000FE86B501C8010E945F85F82EC5010E94DC
:10FD1000F986F11084CE6EE07BE0C5010E94FE867C
:10FD2000B501C8010E945F85F82EC5010E94F986C1
:10FD3000FF2001F3EE2009F468CF45E050E070E0C9
:10FD400060E0C8010E94EA8466E676E0C8010E948D
:10FD50007A85882339F0E090A408F090A508E11492
:10FD6000F10491F461E776E0C8010E947A8581117F
:10FD700007C08091A4089091A508009709F0BBCE18
:10FD8000E0900607F090070720E048EC50E2B4014D
:10FD90008AEA9DE00E94C38EC4010E941E881C82D4
:10FDA0001B8282E293E09A8389839E828D828FEF09
:10FDB0009FEF98878F83B701C5010E94B88FEACD66
:10FDC0000895FC01248135816217730748F480810E
:10FDD0009181009729F0860F971FFC01808108957B
:10FDE00080E008950895AF92BF92CF92DF92EF9294
:10FDF000FF920F931F93CF93DF936C017B018B01D5
:10FE0000040F151FEB015E01AE18BF08C017D10724
:10FE100059F06991D601ED91FC910190F081E02DAE
:10FE2000C6011995892B79F7C501DF91CF911F91F3
:10FE30000F91FF90EF90DF90CF90BF90AF9008951B
:10FE4000FC01A089B1898C91A689B78982FD0FC078
:10FE50009C91818D8F5F8F77228D821749F0A18DC4
:10FE6000AE0FBF2FB11D5D969C93818F08958C912D
:10FE70000895FC01538D448D252F30E0842F90E0B0
:10FE8000821B930B541718F081589F4F08950197C8
:10FE90000895FC01918D828D981761F0A28DAE0FAF
:10FEA000BF2FB11D5D968C91928D9F5F9F77928F32
:10FEB00090E008958FEF9FEF0895FC01918D828D62
:10FEC000981731F0828DE80FF11D858D90E008952F
:10FED0008FEF9FEF0895FC01918D228D892F90E087
:10FEE00080589F4F821B91098F779927089586EF3D
:10FEF00099E00E946B7F21E0892B09F420E0822F9A
:10FF0000089583E19BE00E946B7F21E0892B09F437
:10FF100020E0822F089580E39CE00E946B7F21E027
:10FF2000892B09F420E0822F089582E19EE00E944F
:10FF30006B7F21E0892B09F420E0822F0895FC01DA
:10FF4000A48DA80FB92FB11DA356BF4F2C91848D3E
:10FF500090E001968F779927848FA689B7892C9393
:10FF6000A089B1898C9180648C93938D848D981332
:10FF700006C00288F389E02D80818F7D80830895FB
:10FF8000EF92FF920F931F93CF93DF93EC0181E0E9
:10FF9000888F9B8D8C8D981316C0E889F989808194
:10FFA00085FF11C0EE89FF896083E889F989808126
:10FFB0008064808381E090E0DF91CF911F910F9169
:10FFC000FF90EF900895F62E0B8D10E00F5F1F4FFE
:10FFD0000F771127E02E8C8D8E110CC00FB607FC09
:10FFE000FACFE889F989808185FFF5CFCE010E949B
:10FFF0009F7FF1CFEB8DEC0FFD2FF11DE356FF4FEF
:020000021000EC
:10000000F0820B8FEA89FB8980818062D2CFCF9307
:10001000DF93EC01888D8823B9F0AA89BB89E88930
:10002000F9898C9185FD03C0808186FD0DC00FB6D6
:1000300007FCF7CF8C9185FFF2CF808185FFEDCF54
:10004000CE010E949F7FE9CFDF91CF91089580E09C
:1000500090E0892B29F00E94957F81110E94000079
:1000600080E090E0892B29F00E948B7F81110E9413
:10007000000080E090E0892B29F00E94817F8111AF
:100080000E94000080E090E0892B29F00E94777F99
:1000900081110C94000008950F931F93FC01628559
:1000A0007385848595850281138124813581601B48
:1000B000710B820B930B0685178520893189601B94
:1000C000710B820B930B1F910F910895DC01ED9141
:1000D000FC910190F081E02D19948FEF9FEF08952E
:1000E000FC0162897389848995890895EF920F9341
:1000F0001F93CF93DF93FC01248D222341F0213005
:1001000051F1DF91CF911F910F91EF9008952289C6
:1001100033894489558986899789A08DB18D821B41
:10012000930BA40BB50B892F9A2FAB2FBB278C01F8
:100130000F5F1F4F6281738184819581CFB7F894DF
:10014000DCB7E1E0ECBFEE24E394E2E0FEEF1995CA
:10015000DCBFCFBFD6CFF0E0E0E0DF91CF911F91C1
:100160000F91EF901994FC01138E128E41110CC067
:1001700082899389A489B589868B978BA08FB18F4B
:10018000148E81E090E0089590E080E00895CF9291
:10019000DF92EF92FF92CF93DF93DC01CB01642FCC
:1001A000CFB7F8946D01EE24FF24CBBEDCB741E05D
:1001B0004CBFA901E1E0FEEF1995DCBFCFBFDF9195
:1001C000CF91FF90EF90DF90CF900895CF93DF9382
:1001D000FC01248D211110C0EC01828D938D892B9F
:1001E00049F066897789808D918D30E020E045E087
:1001F0000E94C7801B8E1A8EDF91CF9108951F93A6
:10020000CF93DF93FC01248D211145C0162FEC0103
:10021000828D938D892B49F466897789808D918DA4
:1002200030E020E043E00E94C7804A8D5B8DCA0128
:1002300081709927FE01E80FF91F158F892B69F04E
:100240002D8D3E8D6E897F89888D998D640F751FE8
:10025000811D911D41E00E94C7808A8D9B8D019672
:100260009B8F8A8F81159140B1F46E897F89888D2B
:10027000998D30E020E045E00E94C7801B8E1A8EE9
:100280008E899F89A88DB98D9F5FAF4FBF4F8E8B91
:100290009F8BA88FB98F81E090E0DF91CF911F9164
:1002A0000895DC01ED91FC910280F381E02D40E0A6
:1002B0001994FB012481358142815381241735072C
:1002C00050F4A081B181A20FB31F8C9384819581DA
:1002D00001969583848380E00895CF93DF93EC01AA
:1002E000E881F9810284F385E02DCE01199501960C
:1002F000B9F7DF91CF910895CF92DF92EF92FF92FD
:100300000F931F93CF93DF937C016A018B01D0E0A1
:10031000C0E0CC15DD0581F0D701ED91FC910284A0
:10032000F385E02DC70119958F3F980729F0F80153
:1003300081938F012196EDCFCE01DF91CF911F9157
:100340000F91FF90EF90DF90CF900895CF93C62F3D
:10035000DC01ED91FC910088F189E02D1995DC011B
:10036000ED91FC910190F081E02D6C2FCF911994CB
:10037000062E000C770BFC01778366830895CF93DC
:10038000DF93EC018E819F81019611F5E881F9815F
:100390000088F189E02DCE011995DC01ED91FC91E9
:1003A0000084F185E02D1995892BB1F0E881F98160
:1003B0000284F385E02DCE0119958132910534F345
:1003C000E881F9810684F785E02D682FCE01199523
:1003D00081E0DF91CF91089580E0FBCFFC01208187
:1003E0002EBD9B012150310941F051810DB407FE12
:1003F000FDCF4EB55EBD4193F5CF61507109860FBB
:10040000971F0DB407FEFDCF2EB5FC012083089584
:10041000E091A708F091A80880819091A608892B07
:1004200080830895E091A708F091A80890818091B9
:10043000A60880958923808308958EBD00000DB4A1
:1004400007FEFDCF8EB5089590E02091E309233398
:1004500039F40C96982F990F990F990F80E0089511
:100460004896F8CFEF92FF920F931F93CF93DF93AD
:10047000EC018B017A010E9406AA688B798B8A8B2A
:100480009B8B8C819D81DC01ED91FC910280F3813D
:10049000E02DA701B801DF91CF911F910F91FF903F
:1004A000EF9019941F93CF93DF93EC01162F0E94C6
:1004B00006AA688B798B8A8B9B8B8C819D81DC0152
:1004C000ED91FC910190F081E02D612FDF91CF91B2
:1004D0001F911994CF92DF92EF92FF92CF93DF9307
:1004E000EC018E819F818F3F980759F02FEF3FEFEE
:1004F0003F832E83DF91CF91FF90EF90DF90CF90DD
:1005000008950E9406AA6B017C01A4EFCA0EA1E027
:10051000DA1EE11CF11CE881F9810088F189E02DE7
:10052000CE011995DC01ED91FC910084F185E02D5F
:100530001995892B39F40E9406AA6C157D058E0544
:100540009F0548F3E881F9810088F189E02DCE010B
:100550001995DC01ED91FC910284F385E02DDF918A
:10056000CF91FF90EF90DF90CF9019940E94FCDC28
:100570000F931F93CF93DF93EC01888199810097AC
:1005800059F02A813B812617370730F081E0DF914F
:10059000CF911F910F9108958B016F5F7F4F0E9444
:1005A0001BDC009759F0998388831B830A832C8175
:1005B0003D81232B59F7FC011082E8CF80E0E7CF83
:1005C000CF92DF92EF92FF920F931F93CF93DF931F
:1005D0006C018B0186E090E00E9434CBEC0190939B
:1005E000280980932709F60101900020E9F7CF013F
:1005F0008C199D090E9434CB7C01B6010E9485DDD7
:10060000F60101900020E9F73197EC19FD09EE0D94
:10061000FF1D1082F982E8821B830A8380912A09D8
:1006200090912B099D838C83D0932B09C0932A0929
:10063000DF91CF911F910F91FF90EF90DF90CF90BE
:100640000895FC01868197818F3F980729F02FEF4D
:100650003FEF378326830895808591850C94A3CF3F
:100660007F928F929F92AF92BF92CF92DF92EF9242
:10067000FF920F931F93CF93DF93CDB7DEB7A6976B
:100680000FB6F894DEBF0FBECDBF8C01762E942E30
:10069000852E20E2A22ECE0101967C01DC01EA2DFE
:1006A0001D92EA95E9F76801F3E4CF0ED11C82E3CD
:1006B00094E09AA389A38FEF8BA38CA38DA38EA321
:1006C00043E450E0BE016F5D7F4FC6010E94FC28ED
:1006D000019609F4BFC081E089838A8386E0B82E41
:1006E000BB821C82D80114966D917D918D919C9155
:1006F00017970E9423D96D837E838F83988789867D
:100700009A8680E890E09C878B874CE150E0B701A7
:10071000C6010E949128FE0137968AE1DF011D92F1
:100720008A95E9F74801B8E08B0E911CF401D701D6
:1007300001900D92BA94E1F740E150E0B701C60193
:100740000E949128F7011192AA94E9F796E0A92E48
:10075000B12C40E250E0B701C6010E949128F1E0BF
:10076000AF1AB108B1F783E6898392E89A8393E5DB
:100770009B838C8385E38D8381E08E837F829DE3E1
:10078000988797E099878A8786E0F401DE011B96B7
:1007900001900D928A95E1F78CE0898B8A8B68E64F
:1007A00076E0CE0143960E9485DDD8011B966C91C0
:1007B000CE0149960E9486A5F8016485CE014B962C
:1007C0000E9486A5D8011D966C91CE014D960E947F
:1007D00086A54EE150E0B701C6010E949128B3E022
:1007E0007B121EC082E3898384E08A83F8019685A8
:1007F0009B8397859C8390899D8391899E8396E3B3
:100800009F838887828D8987838D8A87848D8B8754
:10081000858D8C874CE050E0B701C6010E9491287D
:1008200087E3898386E08A8391E09B8393E09C83BE
:100830008D838FE08E838AE38F838BE388878FEFAE
:10084000898749E050E0B701C6010E949128C6019E
:100850000E94CB28A6960FB6F894DEBF0FBECDBF80
:10086000DF91CF911F910F91FF90EF90DF90CF908C
:10087000BF90AF909F908F907F90089590E080E020
:100880000C946927CF93DF93C4E1D0E00E943E84AB
:10089000882361F061E070E080E090E00E94D4A9DC
:1008A0002197A1F780E0DF91CF91089581E0FBCF00
:1008B000FF920F931F93CF93DF931F921F92CDB799
:1008C000DEB7F82E22E030E0AE014F5F5F4F66E208
:1008D00070E00E946A2809811A81102701271027D9
:1008E00022E030E0AE014F5F5F4F66E270E08F2D97
:1008F0000E946A2889819A81982789279827081752
:10090000190749F4C8010F900F90DF91CF911F9103
:100910000F91FF9008958C01E3CFAF92BF92CF92D9
:10092000DF92EF92FF920F931F93CF93DF93DC013F
:10093000CD90DC901197C114D10439F01496CD916B
:10094000DC918C017601209761F4DF91CF911F91AA
:100950000F91FF90EF90DF90CF90BF90AF900895F0
:1009600075015701BFEFAB1ABB0AF7018081082E52
:10097000000C990B0E9449CE892B91F72197CC0D41
:10098000DD1D8881082E000C990B0E9449CE892B11
:1009900029F0CE15DF0510F02197F3CFAE014F5FA0
:1009A0005F4F4E195F09D80115965C934E931497CB
:1009B000CE14DF0420F4B701C6010E9438DDD8014F
:1009C000ED91FC91119714968D919C91E80FF91F70
:1009D0001082BBCFCF93DF93DC011496ED91FC9195
:1009E0006E177F0728F54115510511F19F01261B50
:1009F000370B4217530708F49A01DB01EC01888199
:100A00009981E21BF30BFD83EC83AF01461B570B6F
:100A1000260F371FBC01620F731F8A0F9B1F0E9496
:100A2000AADDE881F9818C819D81E80FF91F108290
:100A3000DF91CF910895DF92EF92FF920F931F9372
:100A4000CF93DF93FC01E480F580E114F10451F4CD
:100A50008FEF9FEFDF91CF911F910F91FF90EF905C
:100A6000DF900895EC010190F081E02DEE0DFF1D67
:100A7000D080108208811981062E000C770BC801E6
:100A80000E94B9DD0E0D1F1DF801D082009701F301
:100A900028813981821B930BDDCFFC0124813581B4
:100AA0006217730720F480819181009729F41092D6
:100AB000290989E299E00895860F971F0895FB019F
:100AC00044815581FC01248135812417350778F054
:100AD00080819181009759F0FB01608171816115DE
:100AE000710529F00E949CDD21E0892B09F020E0AE
:100AF000822F0895FC0124813581232B39F421E0D4
:100B0000FB018081882349F020E007C0808191812A
:100B10000E947CDD21E0892BB9F7822F0895FC012A
:100B200024813581FB014481558124173507E1F487
:100B3000FC0180819181FB01608171810097D1F07E
:100B400061157105A1F4232BC1F0FC01808190E0B7
:100B500008C0232B91F0FB01808190E09195819555
:100B6000910921E0892B09F020E0822F08950E944D
:100B70007CDDF7CF6115710561F721E0F6CFEF92CB
:100B8000FF920F931F93CF93DF936115710541F48B
:100B900080E0DF91CF911F910F91FF90EF9008952A
:100BA00041155105B1F07B01EC010C811D81040F51
:100BB000151FB8010E94B882882351F3288139811A
:100BC0008C819D81B701820F931F0E9485DD1D835B
:100BD0000C8381E0DECFCF93DF931F921F92CDB7BE
:100BE000DEB769831A8241E050E0BE016F5F7F4F3C
:100BF0000E94BF850F900F90DF91CF9108950F93C2
:100C00001F93CF93DF938C01EB01FC0180819181D5
:100C10000097E1F06881798161157105A9F0428141
:100C200053812C813D814217530770F00E9485DD6E
:100C30008C819D81F801958384831D821C82DF91C4
:100C4000CF911F910F9108950E94D0CB88819981F7
:100C5000F801918380838A819B81938382838C8135
:100C60009D8195838483198218821B821A82E5CF25
:100C7000CF93DF93EC0188819981009711F00E9456
:100C8000D0CB198218821D821C821B821A82DF91AE
:100C9000CF910895EF92FF920F931F93CF93DF931D
:100CA00000D01F92CDB7DEB77C01862F4AE08E01BF
:100CB0000F5F1F4FB80190E00E94ECCEF801019049
:100CC0000020E9F73197AF01401B510BB801C70174
:100CD0000E94BF85811103C0C7010E943886C701E9
:100CE0000F900F900F900F90DF91CF911F910F9168
:100CF000FF90EF900895CF93DF93EC01611571059C
:100D000039F4CE010E943886CE01DF91CF9108954B
:100D1000FB0101900020E9F73197AF01461B570B0B
:100D20000E94BF85882369F3EFCFCF93DF93EC0157
:100D3000FB0144815581608171810E94BF858111D1
:100D400003C0CE010E943886CE01DF91CF91089575
:100D5000EF92FF920F931F93CF93DF93EC017B01F0
:100D60008A01BA010E94B88281110BC0CE010E9493
:100D70003886CE01DF91CF911F910F91FF90EF90B8
:100D800008951D830C83B701888199810E9485DDB8
:100D9000F0CFFB0101900020E9F73197AF01461B2E
:100DA000570B0C94A886CF93DF93EC016115710566
:100DB00031F00E94C986CE01DF91CF9108950E9443
:100DC0003886F9CFCF93DF93EC01FB0186179707A5
:100DD00049F0608171816115710541F0448155814F
:100DE0000E94A886CE01DF91CF9108950E94388697
:100DF000F9CFFC01808191810C94D0CBEF92FF92CE
:100E00000F931F93CF93DF93EC018B01198218820C
:100E10001B821A821D821C82CB010E9480CE7C0123
:100E2000BC01CE010E94B882811109C0CE01DF91C0
:100E3000CF911F910F91FF90EF900C943886FD8217
:100E4000EC82B80188819981DF91CF911F910F9138
:100E5000FF90EF900C9479CEFC01118210821382E6
:100E60001282158214820C94E286FC011182108297
:100E700013821282158214826115710551F0FB01F3
:100E800001900020E9F73197AF01461B570B0C94F6
:100E9000A88608950F931F93CF93DF93EC010E94D0
:100EA00006AA688779878A879B87E881F981028407
:100EB000F385E02DCE01199597FF15C00E9406AA73
:100EC000088519852A853B85601B710B820B930B66
:100ED0000C811D812E813F81601771078207930766
:100EE00020F38FEF9FEFDF91CF911F910F91089526
:100EF000EF92FF920F931F93CF93DF93EC017B014F
:100F0000042F61E776E00E943587C7010E944A8777
:100F1000002E000C110B97FD0BC00817190741F0AC
:100F2000682FCE010E94EB85C7010E944A87F3CF4C
:100F3000CE01DF91CF911F910F91FF90EF90089517
:100F4000CF92DF92EF92FF920F931F93CF93DF9395
:100F50006C017A018B01D0E0C0E0C6010E944A8793
:100F600097FD07C0F80181938F012196EC16FD06CD
:100F7000A1F7CE01DF91CF911F910F91FF90EF90DC
:100F8000DF90CF900895FB0101900020E9F73197A1
:100F9000AF01461B570BDC01ED91FC910280F38100
:100FA000E02D19948F929F92AF92BF92EF92FF9291
:100FB0000F931F93CF93DF93CDB7DEB7A1970FB6F3
:100FC000F894DEBF0FBECDBF7C01FA01CB0119A2A0
:100FD000223008F42AE08E010F5D1F4F822E912CE3
:100FE000B12CA12CBF01A50194010E9490D8F90158
:100FF000CA016A300CF5605DD8016E938D01232B18
:10100000242B252B79F790E080E0109721F0BD018B
:10101000C7010E94C387A1960FB6F894DEBF0FBE2A
:10102000CDBFDF91CF911F910F91FF90EF90BF90B7
:10103000AF909F908F900895695CDECF6FE676E069
:101040000C94C387242F462F50E070E060E00C948E
:10105000D287EF92FF920F931F93CF93DF93009766
:1010600051F4CFEFDFEFCE01DF91CF911F910F91C0
:10107000FF90EF900895DC011C96ED90FC90F70135
:1010800000811181D801ED91FC910688F789E02D4E
:10109000C8011995882329F3D801ED91FC910084AA
:1010A000F185E02DC8011995D801ED91FC91892BAE
:1010B00061F30284F385E02DC8011995EC010196D6
:1010C00081F2F801818D882339F04AE050E06C2FDD
:1010D00082E19EE00E942288D70112968C9188239B
:1010E00011F2C532D10509F0BECFD801ED91FC91C6
:1010F0000084F185E02DC801199502975CF0D801B4
:10110000ED91FC910688F789E02DC80119958111B0
:10111000ECCFA7CFD1E0C0E0D801ED91FC910284E3
:10112000F385E02DC80119958F3F980709F499CFF1
:101130009C01215431092A31310570F48D2F82959B
:10114000807F829FC00D1124D11104C00C2E000C91
:10115000DD0B89CFD0E0E0CF9C01215631092A3147
:10116000310560F3C0978A30910570F79D2F9295F5
:10117000907F989FC00D1124E7CFDC01ED91FC9189
:101180000190F081E02D1994CF92DF92EF92FF92BF
:101190000F931F93CF93DF932115310581F4DC0169
:1011A000ED91FC910190F081E02D642FDF91CF91C2
:1011B0001F910F91FF90EF90DF90CF9019942A30FC
:1011C000310501F52AE077FF1DC06A017B01EC01C2
:1011D0006DE20E94BD888C0144275527BA014C1945
:1011E0005D096E097F092AE0CE010E94D287800F37
:1011F000911FDF91CF911F910F91FF90EF90DF90A2
:10120000CF900895DF91CF911F910F91FF90EF90B4
:10121000DF90CF900C94D2878F929F92AF92BF9223
:10122000CF92DF92EF92FF920F931F93CF93DF93B2
:101230007C018B014C0182E0880E911C5701E5E096
:10124000AE0EB11CD0E0C0E0F40161914F014AE064
:1012500050E0C8010E9422886C016EE2C8010E9421
:10126000BD888C0D9D1DC80FD91F8A149B0461F782
:101270004AE050E0F7016581C8010E9422888C0F86
:101280009D1FDF91CF911F910F91FF90EF90DF9005
:10129000CF90BF90AF909F908F900895611571058A
:1012A00011F00C94C38790E080E008950F931F9392
:1012B000CF93DF93EC018B016DE076E00E944E89C5
:1012C00001151105C1F1F80161918F01662399F1B2
:1012D000603240F0623231F06C3521F0CE010E9474
:1012E000BD88F1CF6CE5CE010E94BD88F801319731
:1012F00080818C30D1F044F48930D9F08A30B9F053
:10130000883009F762E6EACF823259F024F462E7C6
:101310008D3021F3D8CF8F3231F06CE58C35F1F27E
:10132000D2CF62E2DBCF6FE2D9CF66E6D7CF6EE6EF
:10133000D5CF64E7D3CF62E2CE010E94BD8890E0B2
:1013400080E0DF91CF911F910F910895DB011496FA
:101350004D915C9115976D917C91DC01ED91FC9123
:101360000280F381E02D1994EF92FF920F931F9367
:10137000CF93DF938C017B01D0E0C0E0F701EC0F4D
:10138000FD1F6491662361F0D801ED91FC910190FD
:10139000F081E02DC8011995892B11F02196EECF2F
:1013A000CE01DF91CF911F910F91FF90EF900895A3
:1013B0000F931F93CF93DF93EC010E94B4898C01AC
:1013C000CE010E941E88800F911FDF91CF911F9147
:1013D0000F910895DC0182E394E08D939D9384E066
:1013E000FB0101900D928A95E1F708953F924F928B
:1013F0005F926F927F928F929F92AF92BF92CF92A5
:10140000DF92EF92FF920F931F93CF93DF93CDB7AD
:10141000DEB7EA970FB6F894DEBF0FBECDBF7C01F2
:101420002A013B0169010E9406AA4B015C01870168
:101430000D5B1F4FC8010E94711618161906ACF0FB
:101440000E9406AA681979098A099B094616570657
:101450006806790608F468C10E94826C61E070E059
:1014600080E090E00E94D4A9E5CF42E250E0BE01C6
:101470006F5F7F4FC8010E94FC1589818230D1F0D7
:10148000312C832DEA960FB6F894DEBF0FBECDBF88
:10149000DF91CF911F910F91FF90EF90DF90CF9050
:1014A000BF90AF909F908F907F906F905F904F9084
:1014B0003F900895F801848995898334910501F757
:1014C0006D817E818F8198850E9423D94B015C01BB
:1014D000F60180829182A282B38246E050E0B70199
:1014E000685F7F4FCE014D960E942BDD892B41F620
:1014F000F70180819181A281B38188169906AA069D
:10150000BB0608F4BDCF84819581A681B78188157B
:101510009905AA05BB0508F4B3CF89899A89AB89D7
:10152000BC8986879787A08BB18B4EEC50E070E02A
:1015300060E0C8010E94FC15312CC701829698AB6F
:101540008FA7F701B696FAABE9AB08969CAB8BABCD
:1015500067019AE1C90ED11CBD96FEABEDABC70188
:10156000429698AF8FABFD97FAAFE9AF4701FEE126
:101570008F0E911CF801818D928D181619060CF0B2
:1015800080CFC8010E941B168333910509F4B2C0B5
:1015900014F58130910509F464C044F4892B51F3AA
:1015A000C8010E941B16AC01552775C083309105F8
:1015B00009F462C00697A1F7C8010E941B16B82E55
:1015C00044E050E0B401C8010E94FC15EB2DE4504A
:1015D000FF0BAF0160C08A33910509F45FC084F549
:1015E00085339105B1F1C697D9F6C8010E941B1643
:1015F0005C01B601CE0189960E94EA898BA59CA563
:10160000ADA5BEA5892B8A2B8B2BB1F0EDA9FEA928
:101610004080518062807380B601CE0183960E9423
:10162000EA898DA19EA1AFA1B8A5A50148165906CA
:101630006A067B0609F0B8CF44E050E0B60118C056
:101640008B33910509F440C08F3F910509F492CF87
:10165000A7CFC8010E941B16C8010E941B16382E76
:1016600089CFC8010E941B1644E050E06FA978ADF5
:10167000C8010E94FC157ECFC8010E941B16B82E1F
:1016800044E050E069AD7AADC8010E94FC158B2D95
:101690008450990BAC0170E060E0EACFC8010E9471
:1016A0001B1644E050E069A97AA9C8010E94FC1504
:1016B000F70166A177A180A591A50E9423D966A311
:1016C00077A380A791A756CFC8010E941B1644E0BC
:1016D00050E06BA97CA9C8010E94FC15F70162A526
:1016E00073A584A595A50E9423D962A773A784A793
:1016F00095A740CFC8010E941B1644E050E06FA59B
:1017000078A9C8010E94FC15F70162A173A184A108
:1017100095A10E9423D962A373A384A395A366A76E
:1017200077A780AB91AB26CF33243A94AACE2F92E1
:101730003F924F925F926F927F928F929F92AF9261
:10174000BF92CF92DF92EF92FF920F931F93CF93AE
:10175000DF9300D000D0CDB7DEB78C010E94A5CCBE
:101760002FEC37E040E050E00E94B2D8DC01CB0122
:101770000196A11DB11DF80184839583A683B783CB
:1017800080839183A283B3835801F3E4AF0EB11C2D
:10179000C5010E94C61564E470E0C5010E944017AF
:1017A000882309F445C10E9406AA2B013C01480187
:1017B00082E4880E911C48EEC42E43E0D42EE12C26
:1017C000F12C52E0252E1E821D82D4018C91833093
:1017D000B1F1811166C0F80184819581A681B7813C
:1017E0000196A11DB11D84839583A683B7830E94B2
:1017F00006AA6419750986099709A70196010E942E
:1018000090D8A90161E0C8010E94308381E0D40131
:101810008C938D819E810197C1F20E9406AA641962
:10182000750986099709D801D6962D913D914D915C
:101830005C91D997261737074807590720F6C50145
:101840000E94C615F80184819581A681B781019611
:10185000A11DB11D84839583A683B7830E9406AA28
:10186000F801FE9660837183828393838D819E81CC
:1018700026960FB6F894DEBF0FBECDBFDF91CF9195
:101880001F910F91FF90EF90DF90CF90BF90AF909E
:101890009F908F907F906F905F904F903F902F9090
:1018A00008958430F1F4F80184819581A681B7818F
:1018B0000196A11DB11D84839583A683B7830E94E1
:1018C00006AA6419750986099709A70196010E945D
:1018D00090D8A90163E0C8010E943083D4012C9202
:1018E00098CF813051F5F80142AD53AD64AD75AD7F
:1018F0009E012F5F3F4FC8010E94F689382EF2E00B
:101900008F1390C089819A81AB81BC81F801848357
:101910009583A683B7830E9406AA64197509860970
:101920009709A70196010E9490D8A90163E0C80118
:101930000E943083D4013C926CCF823009F069CF91
:10194000F80142AD53AD64AD75AD9E012F5F3F4FC1
:10195000C8010E94F689382EF5E08F135DC0E3E0E0
:10196000D401EC93F80182A193A1A4A1B5A1892B84
:101970008A2B8B2B41F484E893E0A0E0B0E082A3B3
:1019800093A3A4A3B5A3F80186A197A1A0A5B1A58F
:10199000892B8A2B8B2B61F482A193A1A4A1B5A1E1
:1019A000B695A7959795879586A397A3A0A7B1A766
:1019B000F80182A593A5A4A5B5A5892B8A2B8B2B0D
:1019C000A9F482A193A1A4A1B5A1AC01BD0123E01A
:1019D00076956795579547952A95D1F7841B950B72
:1019E000A60BB70B82A793A7A4A7B5A7F80186A15A
:1019F00097A1A0A5B1A586A797A7A0ABB1AB82A5DB
:101A000093A5A4A5B5A582AB93ABA4ABB5AB81E080
:101A100090E09E838D83FDCE96E0891303C0D401B0
:101A20001C92F7CEBFEF3B12F4CEF4011082F1CE40
:101A30001E821D821BCF1F920F920FB60F92112490
:101A40000BB60F922F933F934F935F936F937F93B8
:101A50008F939F93AF93BF93EF93FF9386EF99E09C
:101A60000E949F7FFF91EF91BF91AF919F918F91C6
:101A70007F916F915F914F913F912F910F900BBE8E
:101A80000F900FBE0F901F9018951F920F920FB6D8
:101A90000F9211240BB60F922F933F934F935F93A6
:101AA0006F937F938F939F93AF93BF93EF93FF9326
:101AB00086EF99E00E94207FFF91EF91BF91AF9157
:101AC0009F918F917F916F915F914F913F912F9156
:101AD0000F900BBE0F900FBE0F901F9018951F9286
:101AE0000F920FB60F9211240BB60F922F933F93C4
:101AF0004F935F936F937F938F939F93AF93BF9316
:101B0000EF93FF9383E19BE00E949F7FFF91EF9112
:101B1000BF91AF919F918F917F916F915F914F9105
:101B20003F912F910F900BBE0F900FBE0F901F9003
:101B300018951F920F920FB60F9211240BB60F92A9
:101B40002F933F934F935F936F937F938F939F93C5
:101B5000AF93BF93EF93FF9383E19BE00E94207FBD
:101B6000FF91EF91BF91AF919F918F917F916F9175
:101B70005F914F913F912F910F900BBE0F900FBE31
:101B80000F901F9018951F920F920FB60F9211246D
:101B90000BB60F922F933F934F935F936F937F9367
:101BA0008F939F93AF93BF93EF93FF9380E39CE05A
:101BB0000E949F7FFF91EF91BF91AF919F918F9175
:101BC0007F916F915F914F913F912F910F900BBE3D
:101BD0000F900FBE0F901F9018951F920F920FB687
:101BE0000F9211240BB60F922F933F934F935F9355
:101BF0006F937F938F939F93AF93BF93EF93FF93D5
:101C000080E39CE00E94207FFF91EF91BF91AF9114
